:020000040800F2
:1000000000040020A51F0008F71F0008F71F0008C4
:10001000F71F0008F71F0008F71F00080000000086
:10002000000000000000000000000000F71F0008B2
:10003000F71F000800000000F71F0008E11E02087B
:100040006D2002086F200208712002087520020846
:10005000952002089720020899200208BD20020876
:10006000E120020805210208292102084D21020889
:100070004F2102085121020853210208552102088C
:1000800057210208592102085B210208F71F0008C6
:10009000F71F0008F71F0008F71F00085D2102087E
:1000A000A9210208AB210208AD210208AF210208F4
:1000B000B1210208B5210208E121020851220208FB
:1000C0005322020855220208572202085922020828
:1000D0005D220208CD230208F522020891240208BD
:1000E00055250208192602081B2602081D260208AB
:1000F00021260208892602088B2602088D2602087E
:100100008F260208912602089326020895260208E7
:10011000992602086D2702086F2702087127020836
:100120007D2802087F280208812802088328020807
:1001300000000000000000000000000000000000BF
:1001400000000000000000000000000000000000AF
:10015000000000000000000000000000000000009F
:10016000000000000000000000000000000000008F
:10017000000000000000000000000000000000007F
:10018000000000000000000000000000000000006F
:10019000000000000000000000000000000000005F
:1001A000000000000000000000000000000000004F
:1001B000000000000000000000000000000000003F
:1001C000000000000000000000000000000000002F
:1001D000000000000000000000000000000000001F
:0401E0005FF8E0F1F3
:1001E800032A70B404460D4626D941EA000313F0E9
:1001F800030F13D020782B78984208BF294606D0E1
:100208001EE014F8010F11F8013F984218D1012A95
:1002180002F1FF32F5D1002070BC70470B4604464E
:1002280051F8045B50F8046BAE4204D1043A04461A
:10023800032A0B46F2D81D461046002ADAD1EBE70E
:10024800C01AE9E7032A2DE9F00109D82AB10023E9
:10025800CC5CC45401339342FAD1BDE8F001704735
:100268000B468218014603E02478013301F8014B5C
:1002780011F0030F1C46F7D113F003055DD06E4251
:10028800C5F1040CED009B594FEACC0C08E004348E
:10029800A7593B4607FA0CF748EA070741F8047BD9
:1002A800571A23FA05F8032FF1DC03E014F8013B91
:1002B80001F8013B8A42F9D8CFE753F8404C41F89E
:1002C800404C53F83C4C41F83C4C53F8384C41F8FE
:1002D800384C53F8344C41F8344C53F8304C41F80E
:1002E800304C53F82C4C41F82C4C53F8284C41F81E
:1002F800284C53F8244C41F8244C53F8204C41F82E
:10030800204C53F81C4C41F81C4C53F8184C41F83D
:10031800184C53F8144C41F8144C53F8104C41F84D
:10032800104C53F80C4C41F80C4C53F8084C41F85D
:10033800084C53F8044C41F8044C561A1D460C4618
:10034800403340313F2EB8DC2B460FE053F8101CE9
:1003580044F8101C53F80C1C44F80C1C53F8081CE7
:1003680044F8081C53F8041C44F8041C161B2146C6
:100378001D46103410330F2EE8DC2B4602E02468AB
:1003880041F8044B551A1C46032D03F10403F6DC0F
:1003980090E700BF032AC9B270B408D82AB103464F
:1003A800121803F8011B9342FBD170BC70478218E6
:1003B800044601E004F8011B14F0030FFAD14FF0D2
:1003C800013303FB01F31FE044F8403C44F83C3C94
:1003D80044F8383C44F8343C44F8303C44F82C3C6D
:1003E80044F8283C44F8243C44F8203C44F81C3C9D
:1003F80044F8183C44F8143C44F8103C44F80C3CCD
:1004080044F8083C44F8043C161B254640343F2E6B
:10041800DADC2C4607E044F8103C44F80C3C44F87D
:10042800083C44F8043C161B254610340F2EF2DC19
:1004380001E045F8043B541B032CFADC01E005F805
:10044800011B9542FBD3B0E710F0030F38B5044603
:1004580012D10368A3F1013222EA030313F0803FAB
:100468000AD1031D184653F8042BA2F1013525EAD9
:10047800020212F0803FF5D003782BB1431C1846D6
:1004880013F8012B002AFAD100F076F9204638BD7E
:10049800C9B2F0B4002950D010F0030F10D003787F
:1004A800002B79D0994246D0431C05E013F8012B64
:1004B800002A3FD091423ED013F0030F1846F5D1E1
:1004C800036841EA01270646A3F1013247EA0747D4
:1004D80022EA030212F0803F1DD187EA0303A3F149
:1004E800013222EA030313F0803F14D1043002E002
:1004F80012F0803F0FD1064650F8043BA3F10135B6
:1005080087EA030225EA0303A2F1013413F0803FCE
:1005180024EA0202ECD033783046002B3CD09942D2
:1005280009D0731C01E0914205D0184613F8012B3D
:10053800002AF8D11046F0BC704710F0030F0CD019
:100548000378002BF7D0431C03E013F8012B002A93
:10055800F1D013F0030F1846F7D102680346A2F151
:10056800013121EA020212F0803F0AD10430034629
:1005780050F8042BA2F1013121EA020212F0803F67
:10058800F5D01A781846002AD5D00133184613F842
:10059800012B002AFAD1CEE71846CCE780EA0102FF
:1005A80012F0030F3AD110F0030220F0030021F0FB
:1005B800030150F804CB08BF51F8043B0DD082F07A
:1005C80003024FEAC2026FF07F4323FA02F251F8A6
:1005D800043B4CEA020C43EA020300BFACF10132CF
:1005E8009C4501BF22EA0C0212F0803F50F804CB70
:1005F80051F8043BF2D04FEA0C604FEA1C2C01285A
:1006080028BFB0EB036F08BF1B0AF4D003F0FF0349
:100618004FEA1060A0EB0300704700BF10F0030F13
:100628000AD010F8012B11F8013B012A28BF9A4281
:10063800F4D0A2EB030070474DF8045D4DF8044D6B
:100648004FF0010242EA022242EA024201F0030CA0
:1006580021F0030150F8044B51F8045BBCF1020F80
:1006680026D04BD824F07F4CBCEB152FA4EB02030B
:1006780023EA04030DD113EAC21308BF51F8045B3F
:100688000AD18CEA040CBCEB056F0CD150F8044B72
:10069800E8E74FEA15255CE033F07F4352D10D7847
:1006A8004FEA146C55E04FEA146C05F0FF0550E072
:1006B8004FEA044CA4EB02034FEA1C4C23EA040360
:1006C800BCEB154F17D113EAC21308BF51F8045BEE
:1006D80007D18CEA040CBCEB054F08D150F8044B49
:1006E800E6E71B042ED10D884FEA144C31E04FEA9F
:1006F80005454FEA144C4FEA15452AE004F0FF0C73
:10070800BCEB156FA4EB020323EA04030DD113EA33
:10071800C21308BF51F8045B0AD18CEA040CBCEB85
:10072800052F0AD150F8044BE8E74FEA156510E0A9
:1007380014F0FF0F06D051F8045B4FEA142C25F093
:100748007F4506E04FF000005DF8044B5DF8045B60
:1007580070470CF0FF0205F0FF00012828BF904207
:1007680004BF4FEA1C2C2D0AF3D0A2EB00005DF861
:10077800044B5DF8045B704780EA0102844612F07E
:10078800030F4FD111F0030F32D14DF8044D11F082
:10079800040F51F8043B0BD0A3F101329A4312F035
:1007A800803F04BF4CF8043B51F8043B16D100BF0E
:1007B80051F8044BA3F101329A4312F0803FA4F19F
:1007C80001320BD14CF8043BA24312F0803F04BF26
:1007D80051F8043B4CF8044BEAD023460CF8013B93
:1007E80013F0FF0F4FEA3323F8D15DF8044B70473D
:1007F80011F0010F06D011F8012B0CF8012B002A7B
:1008080008BF704711F0020FBFD031F8022B12F069
:10081800FF0F16BF2CF8022B8CF8002012F47F4F24
:10082800B3D1704711F8012B0CF8012B002AF9D12C
:10083800704700BF20F0030110F00300C0F1000072
:1008480051F8043B00F1040C4FEACC0C6FF00002A5
:100858001CBF22FA0CF213434FF0010C4CEA0C2C8B
:100868004CEA0C4CA3EB0C0222EA030212EACC126B
:1008780004BF51F8043B0430F4D013F0FF0F1FBF3E
:10088800013013F47F4F013013F47F0F18BF01308C
:10089800704700BFF0B4002A46D041EA000313F0C5
:1008A80003032CD1032A07460E4643D904680D6872
:1008B800AC423FD1043A37D0A4F1013525EA04040B
:1008C80014F0803F18BF18462CD1041D0D1D0EE0F2
:1008D80054F8043B55F8041BA3F101308B4220EA7D
:1008E800030027D1043A1FD010F0803F1ED1032AFD
:1008F80027462E46ECD820462946002A1DD00478E3
:10090800013A0D78AC420CD172B18CB1002302E0EF
:1009180093420BD064B1013310F8014FCD5CAC4267
:10092800F6D0601BF0BC70471046FBE70020F9E7E3
:100938002046F7E738463146E1E724782D78F0E796
:1009480041EA000313F0030F0B4670B414BF0024F0
:100958000124032A94BF002404F001040546D4B9F5
:10096800BAB10E782B46013A03F8016B56B1AC1CAC
:100978007AB111F8015F2346013A04F8015C0134A9
:10098800002DF5D12AB19A18002103F8011B9342D2
:10099800FBD170BC7047194653F8044BA4F10136DB
:1009A80026EA040616F0803FDAD1043A45F8044BEB
:1009B800032A1946EFD8D3E701232DE9F0071D468E
:1009C80000264FF0FF37AC1900EB070C8C420DD214
:1009D8001CF805C010F80480E0452ED201252646F3
:1009E800E31BAC198C4200EB070CF1D34FF0010963
:1009F80000264D464FF0FF3C1360AC1900EB0C0885
:100A0800A1420ED918F8058010F804A0C2451AD9D9
:100A180001252646CCEB0409AC19A14200EB0C08D1
:100A2800F0D80CF101000137B8423CBF994638466E
:100A3800C2F80090BDE8F00770470BD00123374695
:100A48001D46F618BFE709D04FF00109B4464D46D8
:100A58004E44D2E79D4205D00135B4E74D4505D057
:100A68000135CAE72B4626460125ACE7A9462646A6
:100A78000125C2E72DE9F04FADF5826D81B014462E
:100A8800074610460DF580628B460C3219461D4606
:100A9800FFF792FF03AE04A901F57E72331F0090A1
:100AA80043F8045F9342FBD14DB1681E0023E25C1A
:100AB800C11A013303AEAB4246F82210F7D1DDF874
:100AC8000C142046009A6118FFF78AFB002877D19A
:100AD8000099814605F1FF380646C1F101020192ED
:100AE8005A46AB4609EB0B0501F1FF3AB81800214D
:100AF800AA1A00F0E5F900284FD1002D00F0C080B7
:100B08007B1903A913F8013C51F82330002B4CD171
:100B1800009B9E4228BF334698450FD903EB090135
:100B2800E05C7A18795C884205D038E012F8011F39
:100B3800E05C884233D101339845F7D8009A964251
:100B480080F0A48007EB090214F80A10534612F843
:100B58000A20914204BF0AEB0901791807D095E0F1
:100B680014F802C011F8010D844503D113465A1E2A
:100B7800B342F5D101369E4200F28D80DDF80C6457
:100B88002A46B144C6EB0B0609EB0B05B818002141
:100B9800AA1A00F095F90028AFD0002071E0019A58
:100BA8000026914499442A46EEE7002EFAD0DDF853
:100BB8000C2493423CBFC2EB0B0306469944F2E770
:100BC800009E4FF000080099AB1BB34238BF334674
:100BD800C1F101026E1E019201F1FF3A5A4689469F
:100BE800AB460133CDF80C3408EB0B05B8180021DF
:100BF800AA1A00F065F90028CFD1002D40D07B1942
:100C080003A913F8013C51F82330002B30D1B1452A
:100C180013D208EB090314F80910FA18FB5C99427F
:100C280018BF4B4627D14B4604E012F8011FE05C81
:100C3800884220D10133B342F7D3BAF1FF3F53467C
:100C48002CD007EB080C14F80A101CF80A20914263
:100C58000CD10AEB0802BA1804E0E05C12F8011D96
:100C6800884203D1013BF8D260460AE0DDF80C3433
:100C780098442A46B8E701992A4688449844B3E735
:100C8800284605B00DF5806DBDE8F08F009B013654
:100C98009E427FF673AF07EB0900F2E707EB080CFB
:100CA8006046EEE72DE9F04F8346037885B00C46A1
:100CB800002B00F0F9800A78A2B106460131012024
:100CC80002E011F8012B8AB1934214BF002000F012
:100CD800010016F8013F0D46002BF2D12B782BB1FD
:100CE8004FF0000B584605B0BDE8F08F0028F9D149
:100CF8000BF101002178FFF7CBFB2D1BA5F10102B9
:100D0800534243EB0203002808BF43F001030746A0
:100D180083B90BEB0508404594BFC0EB08084FF0BA
:100D280001081F2D08D9414622462B46FFF7A2FE8F
:100D38008346D7E78346D5E7294603AA2046FFF727
:100D48003BFE03996118814620464A46FFF748FA58
:100D580000284FD109F1FF33C9F10102064601927B
:100D680082464246C84699460AEB050BB818002148
:100D7800C2EB0B0200F0A4F80028B1D1BBF1000FC0
:100D8800B0D046452CBF334643469D420FD903EBAE
:100D98000A01E05C7A18795C884205D075E012F89F
:100DA800011FE05C884270D101339D42F7D1B04504
:100DB8007DD907EB0A0214F809104B4612F80920EE
:100DC800914202BF09EB0A01AC46791806D06EE0E1
:100DD800A55C11F8010D854203D113465A1EB34292
:100DE800F6D1654601369E4267D8039E5A46B244FC
:100DF800AE1BB9E7C9F10101C9EB0503424600265C
:100E080009F1FF3A88464B4538BF4B4601330393F7
:100E180006EB050BB8180021C2EB0B0200F050F8E6
:100E280000287FF45DAFBBF1000F3FF45BAF4D4589
:100E380012D906EB090314F80910FA18FB5C994259
:100E480008BF4B4605D026E012F8011FE05C884237
:100E580022D101339D42F7D1BAF1FF3F534628D042
:100E680007EB060C14F80A101CF80A20914217D157
:100E78000AEB0602BA1804E0E05C12F8011D884289
:100E88000ED1013BF8D2E3462CE7019A00269244A2
:100E98005A469A4468E74B4646445A46F618B7E716
:100EA800039B5A46F618B3E70D46012016E743465A
:100EB80098E707EB060CE34614E707EB0A0B11E784
:100EC80010F0030F034670B4C9B211D0002A22D023
:100ED80003788B421DD0013A013005E0DAB110F8F1
:100EE800014B013A8C4218D010F0030F0346F5D19C
:100EF800032A14D87AB1187888420ED0541E5D1C83
:100F080003E015F8016B8E4203D0013C2846F8D265
:100F1800002070BC70471046FBE71846F9E741EA25
:100F2800012646EA0646184653F8044B86EA0404A6
:100F3800A4F1013525EA040414F0803F03D1043AF2
:100F48001846032AEFD80346D4E700BF0000000084
:100F5800C1F30A5C0246ACF57E7C2DE9F84FACF192
:100F68000704132C0B4606460F468946804627DCA5
:100F7800002C52DB4FF6FF7CC0F20F0C4CFA04FA3F
:100F88000AEA0105054317D037A3D3E9002300F087
:100F980075F80022002300F0B3FC002856D0002F7B
:100FA80005DD4FF4801353FA04F407EB040929EA2A
:100FB8000A0900264B46324610461946BDE8F88F06
:100FC800332C07DDB4F5806FF6D100F057F80246F0
:100FD8000B46F1E74FF0FF3BACF11B0C2BFA0CFB77
:100FE8001BEA000FE8D020A3D3E9002300F046F85D
:100FF8000022002300F084FC40B3002F0ADD142CEB
:1010080006D00126C4F13404A64016EB080601D325
:1010180007F1010926EA0B0619E013A3D3E9002317
:1010280000F02CF80022002300F06AFC78B1002FB1
:1010380013DB46EA07054FF000094D45C3F6F07982
:101048000CBF2E46002608BFA94600E0B9464B460D
:10105800324610461946BDE8F88F00264FF0004981
:10106800F5E700BFAFF300809C7500883CE4377E4D
:1010780081F0004102E000BF83F0004330B54FEA41
:1010880041044FEA430594EA050F08BF90EA020FAE
:101098001FBF54EA000C55EA020C7FEA645C7FEA41
:1010A800655C00F0E2804FEA5454D4EB5555B8BF64
:1010B8006D420CDD2C4480EA020281EA030382EAD5
:1010C800000083EA010180EA020281EA0303362D67
:1010D80088BF30BD11F0004F4FEA01314FF4801C3A
:1010E8004CEA113102D0404261EB410113F0004F4C
:1010F8004FEA03334CEA133302D0524263EB430303
:1011080094EA050F00F0A780A4F10104D5F1200EA0
:101118000DDB02FA0EFC22FA05F2801841F10001FB
:1011280003FA0EF2801843FA05F359410EE0A5F1CF
:1011380020050EF1200E012A03FA0EFC28BF4CF000
:10114800020C43FA05F3C01851EBE37101F00045B6
:1011580007D54FF0000EDCF1000C7EEB00006EEBC3
:101168000101B1F5801F1BD3B1F5001F0CD349084D
:101178005FEA30004FEA3C0C04F101044FEA4452A4
:1011880012F5800F80F09A80BCF1004F08BF5FEA2B
:10119800500C50F1000041EB045141EA050130BD0B
:1011A8005FEA4C0C404141EB010111F4801FA4F1AE
:1011B8000104E9D191F0000F04BF01460020B1FA03
:1011C80081F308BF2033A3F10B03B3F120020CDA3B
:1011D8000C3208DD02F1140CC2F10C0201FA0CF019
:1011E80021FA02F10CE002F11402D8BFC2F1200C7E
:1011F80001FA02F120FA0CFCDCBF41EA0C01904034
:10120800E41AA2BF01EB0451294330BD6FEA04047C
:101218001F3C1CDA0C340EDC04F11404C4F1200267
:1012280020FA04F001FA02F340EA030021FA04F379
:1012380045EA030130BDC4F10C04C4F1200220FAD0
:1012480002F001FA04F340EA0300294630BD21FA0E
:1012580004F0294630BD94F0000F83F4801306BFD4
:1012680081F480110134013D4EE77FEA645C18BFC8
:101278007FEA655C29D094EA050F08BF90EA020F5F
:1012880005D054EA000C04BF1946104630BD91EA57
:10129800030F1EBF0021002030BD5FEA545C05D15A
:1012A8004000494128BF41F0004130BD14F5800499
:1012B8003CBF01F5801130BD01F0004545F0FE410D
:1012C80041F470014FF0000030BD7FEA645C1ABF42
:1012D800194610467FEA655C1CBF0B46024650EA79
:1012E800013406BF52EA033591EA030F41F40021A5
:1012F80030BD00BF90F0000F04BF0021704730B52B
:101308004FF4806404F132044FF000054FF00001FF
:1013180050E700BF90F0000F04BF0021704730B5C0
:101328004FF4806404F1320410F0004548BF404295
:101338004FF000013EE700BF42004FEAE2014FEAEA
:1013480031014FEA02701FBF12F07F4393F07F4FC5
:1013580081F06051704792F0000F14BF93F07F4FF7
:10136800704730B54FF4607401F0004521F000413A
:1013780020E700BF50EA010208BF704730B54FF0C0
:1013880000050AE050EA010208BF704730B511F0C5
:10139800004502D5404261EB41014FF4806404F1FD
:1013A80032045FEA915C3FF4DCAE4FF003025FEA7F
:1013B800DC0C18BF03325FEADC0C18BF033202EB07
:1013C800DC02C2F1200300FA03FC20FA02F001FA61
:1013D80003FE40EA0E0021FA02F11444C1E600BF00
:1013E80070B54FF0FF0C4CF4E06C1CEA11541DBFB3
:1013F8001CEA135594EA0C0F95EA0C0F00F0DEF87E
:101408002C4481EA030621EA4C5123EA4C5350EA62
:10141800013518BF52EA033541F4801143F48013B3
:1014280038D0A0FB02CE4FF00005E1FB02E506F044
:101438000042E0FB03E54FF00006E1FB03569CF099
:10144800000F18BF4EF0010EA4F1FF04B6F5007F9F
:1014580064F5407404D25FEA4E0E6D4146EB060611
:1014680042EAC62141EA55514FEAC52040EA5E509A
:101478004FEACE2EB4F1FD0C88BFBCF5E06F1ED844
:10148800BEF1004F08BF5FEA500E50F1000041EB7B
:10149800045170BD06F0004646EA010140EA020028
:1014A80081EA0301B4EB5C04C2BFD4EB0C0541EA4A
:1014B800045170BD41F480114FF0000E013C00F35F
:1014C800AB8014F1360FDEBF002001F0004170BD83
:1014D800C4F10004203C35DA0C341BDC04F114049C
:1014E800C4F1200500FA05F320FA04F001FA05F228
:1014F80040EA020001F0004221F0004110EBD370F5
:1015080021FA04F642EB06015EEA430E08BF20EA20
:10151800D37070BDC4F10C04C4F1200500FA04F3C3
:1015280020FA05F001FA04F240EA020001F0004155
:1015380010EBD37041F100015EEA430E08BF20EAC8
:10154800D37070BDC4F1200500FA05F24EEA020E10
:1015580020FA04F301FA05F243EA020321FA04F03F
:1015680001F0004121FA04F220EA020000EBD370F6
:101578005EEA430E08BF20EAD37070BD94F0000FF6
:101588000FD101F00046400041EB010111F4801F2A
:1015980008BF013CF7D041EA060195F0000F18BFDB
:1015A800704703F00046520043EB030313F4801F17
:1015B80008BF013DF7D043EA0603704794EA0C0FD1
:1015C8000CEA135518BF95EA0C0F0CD050EA4106E7
:1015D80018BF52EA4306D1D181EA030101F0004164
:1015E8004FF0000070BD50EA410606BF104619468C
:1015F80052EA430619D094EA0C0F02D150EA013698
:1016080013D195EA0C0F05D152EA03361CBF1046D8
:1016180019460AD181EA030101F0004141F0FE4177
:1016280041F470014FF0000070BD41F0FE4141F4FB
:10163800780170BD70B54FF0FF0C4CF4E06C1CEAFB
:1016480011541DBF1CEA135594EA0C0F95EA0C0FB0
:1016580000F0A7F8A4EB050481EA030E52EA03356B
:101668004FEA013100F088804FEA03334FF080558C
:1016780045EA131343EA12634FEA022245EA1115B9
:1016880045EA10654FEA00260EF000419D4208BF6A
:10169800964244F1FD0404F5407402D25B084FEA17
:1016A8003202B61A65EB03055B084FEA32024FF4C3
:1016B80080104FF4002CB6EB020E75EB030E22BF20
:1016C800B61A754640EA0C005B084FEA3202B6EBE0
:1016D800020E75EB030E22BFB61A754640EA5C008F
:1016E8005B084FEA3202B6EB020E75EB030E22BF1F
:1016F800B61A754640EA9C005B084FEA3202B6EB20
:10170800020E75EB030E22BFB61A754640EADC00DE
:1017180055EA060E18D04FEA051545EA16754FEA40
:1017280006164FEAC30343EA52734FEAC2025FEA5E
:101738001C1CC0D111F4801F0BD141EA00014FF0ED
:1017480000004FF0004CB6E711F4801F04BF0143BE
:101758000020B4F1FD0C88BFBCF5E06F3FF6AFAEDA
:10176800B5EB030C04BFB6EB020C5FEA500C50F16A
:10177800000041EB045170BD0EF0004E4EEA1131ED
:1017880014EB5C04C2BFD4EB0C0541EA045170BDF4
:1017980041F480114FF0000E013C90E645EA060E38
:1017A8008DE60CEA135594EA0C0F08BF95EA0C0F66
:1017B8003FF43BAF94EA0C0F0AD150EA01347FF4AE
:1017C80034AF95EA0C0F7FF425AF104619462CE785
:1017D80095EA0C0F06D152EA03353FF4FDAE1046E8
:1017E800194622E750EA410618BF52EA43067FF439
:1017F800C5AE50EA41047FF40DAF52EA43057FF4C9
:10180800EBAE12E74FF0FF3C06E000BF4FF0010CD3
:1018180002E000BF4FF0010C4DF804CD4FEA410C37
:101828007FEA6C5C4FEA430C18BF7FEA6C5C1BD004
:1018380001B050EA410C0CBF52EA430C91EA030F85
:1018480002BF90EA020F0020704710F1000F91EAE2
:10185800030F58BF994208BF90422CBFD8176FEAB0
:10186800E37040F0010070474FEA410C7FEA6C5C7E
:1018780002D150EA013C07D14FEA430C7FEA6C5C85
:10188800D6D152EA033CD3D05DF8040B704700BFB1
:101898008446104662468C461946634600E000BFFF
:1018A80001B5FFF7B7FF002848BF10F1000F01BDD1
:1018B8004DF808EDFFF7F4FF0CBF012000205DF89C
:1018C80008FB00BF4DF808EDFFF7EAFF34BF012021
:1018D80000205DF808FB00BF4DF808EDFFF7E0FFBA
:1018E80094BF012000205DF808FB00BF4DF808ED0B
:1018F800FFF7CEFF94BF012000205DF808FB00BF72
:101908004DF808EDFFF7C4FF34BF012000205DF853
:1019180008FB00BF4FEA4102B2F1E04324BFB3F530
:10192800001CDCF1FE5C0DD901F0004C4FEAC0024E
:101938004CEA5070B2F1004F40EB830008BF20F032
:101948000100704711F0804F21D113F13872BCBFEC
:1019580001F00040704741F480114FEA5252C2F141
:101968001802C2F1200C10FA0CF320FA02F018BF8A
:1019780040F001004FEAC1234FEAD32303FA0CFCDD
:1019880040EA0C0023FA02F34FEA4303CCE77FEA6C
:10199800625307D150EA01331EBF4FF0FE4040F4B6
:1019A8004000704701F0004040F0FE4040F4000065
:1019B800704700BF80F0004002E000BF81F00041A6
:1019C80042001FBF5FEA410392EA030F7FEA226CDD
:1019D8007FEA236C6AD04FEA1262D2EB1363C1BF6D
:1019E800D218414048404140B8BF5B42192B88BFDC
:1019F800704710F0004F40F4000020F07F4018BFFF
:101A0800404211F0004F41F4000121F07F4118BF1E
:101A1800494292EA030F3FD0A2F1010241FA03FCC6
:101A280010EB0C00C3F1200301FA03F100F00043AE
:101A380002D5494260EB4000B0F5000F13D3B0F176
:101A4800807F06D340084FEA310102F10102FE2AE5
:101A580051D2B1F1004F40EBC25008BF20F0010055
:101A680040EA03007047490040EB000010F4000F03
:101A7800A2F10102EDD1B0FA80FCACF1080CB2EB96
:101A88000C0200FA0CF0AABF00EBC25052421843F5
:101A9800BCBFD0401843704792F0000F81F400019A
:101AA80006BF80F400000132013BB5E74FEA41036D
:101AB8007FEA226C18BF7FEA236C21D092EA030FD9
:101AC80004D092F0000F08BF0846704790EA010F53
:101AD8001CBF0020704712F07F4F04D1400028BF80
:101AE80040F00040704712F100723CBF00F5000062
:101AF800704700F0004343F0FE4040F40000704798
:101B08007FEA226216BF08467FEA23630146420243
:101B180006BF5FEA412390EA010F40F48000704756
:101B28004FF0000304E000BF10F0004348BF4042FC
:101B38005FEA000C08BF704743F0964301464FF038
:101B480000001CE050EA010208BF70474FF0000394
:101B58000AE000BF50EA010208BF704711F00043D5
:101B680002D5404261EB41015FEA010C02BF8446A5
:101B78000146002043F0B64308BFA3F18053A3F504
:101B88000003BCFA8CF2083AA3EBC25310DB01FA4B
:101B980002FC634400FA02FCC2F12002BCF1004FCF
:101BA80020FA02F243EB020008BF20F00100704760
:101BB80002F1200201FA02FCC2F1200250EA4C00B4
:101BC80021FA02F243EB020008BF20EADC707047FA
:101BD8004FF0FF0C1CEAD0521EBF1CEAD15392EA08
:101BE8000C0F93EA0C0F6FD01A4480EA010C4002E4
:101BF80018BF5FEA41211ED04FF0006343EA50103E
:101C080043EA5111A0FB01310CF00040B1F5000F7F
:101C18003EBF490041EAD3715B0040EA010062F12E
:101C28007F02FD2A1DD8B3F1004F40EBC25008BF18
:101C380020F00100704790F0000F0CF0004C08BF36
:101C480049024CEA502040EA51207F3AC2BFD2F103
:101C5800FF0340EAC250704740F400004FF0000311
:101C6800013A5DDC12F1190FDCBF00F0004070474B
:101C7800C2F10002410021FA02F1C2F1200200FA89
:101C880002FC5FEA310040F1000053EA4C0308BF50
:101C980020EADC70704792F0000F00F0004C02BFA1
:101CA800400010F4000F013AF9D040EA0C0093F01C
:101CB800000F01F0004C02BF490011F4000F013B76
:101CC800F9D041EA0C018FE70CEAD15392EA0C0FE4
:101CD80018BF93EA0C0F0AD030F0004C18BF31F04F
:101CE800004CD8D180EA010000F00040704790F025
:101CF800000F17BF90F0004F084691F0000F91F0C9
:101D0800004F14D092EA0C0F01D142020FD193EA8E
:101D18000C0F03D14B0218BF084608D180EA010016
:101D280000F0004040F0FE4040F40000704740F0F2
:101D3800FE4040F4400070474FF0FF0C1CEAD052C0
:101D48001EBF1CEAD15392EA0C0F93EA0C0F69D01C
:101D5800A2EB030280EA010C49024FEA402037D087
:101D68004FF0805343EA111143EA10130CF000407E
:101D78008B4238BF5B0042F17D024FF4000C8B426E
:101D880024BF5B1A40EA0C00B3EB510F24BFA3EB4E
:101D9800510340EA5C00B3EB910F24BFA3EB91031E
:101DA80040EA9C00B3EBD10F24BFA3EBD10340EA78
:101DB800DC001B0118BF5FEA1C1CE0D1FD2A3FF6BE
:101DC80050AF8B4240EBC25008BF20F00100704773
:101DD8000CF0004C4CEA50207F32C2BFD2F1FF0316
:101DE80040EAC250704740F400004FF00003013A47
:101DF80037E792F0000F00F0004C02BF400010F4EB
:101E0800000F013AF9D040EA0C0093F0000F01F0FE
:101E1800004C02BF490011F4000F013BF9D041EA20
:101E28000C0195E70CEAD15392EA0C0F08D1420253
:101E38007FF47DAF93EA0C0F7FF470AF084676E726
:101E480093EA0C0F04D14B023FF44CAF08466EE7FF
:101E580030F0004C18BF31F0004CCAD130F00042CD
:101E68007FF45CAF31F000437FF43CAF5FE700BF25
:101E78004FF0FF3C06E000BF4FF0010C02E000BF4E
:101E88004FF0010C4DF804CD4FEA40024FEA4103F0
:101E98007FEA226C18BF7FEA236C11D001B052EAA6
:101EA800530C18BF90EA010F58BFB2EB030088BF6C
:101EB800C81738BF6FEAE17018BF40F001007047DB
:101EC8007FEA226C02D15FEA402C05D17FEA236CBD
:101ED800E4D15FEA412CE1D05DF8040B704700BF04
:101EE800844608466146FFE70FB5FFF7C9FF00289B
:101EF80048BF10F1000F0FBD4DF808EDFFF7F4FFD4
:101F08000CBF012000205DF808FB00BF4DF808ED6C
:101F1800FFF7EAFF34BF012000205DF808FB00BF8F
:101F28004DF808EDFFF7E0FF94BF012000205DF8B1
:101F380008FB00BF4DF808EDFFF7D2FF94BF012062
:101F480000205DF808FB00BF4DF808EDFFF7C8FF5B
:101F580034BF012000205DF808FB00BF42000ED20C
:101F6800B2F1FE4F0BD34FF09E03B3EB126209D4CC
:101F78004FEA002343F0004323FA02F070474FF082
:101F88000000704712F1610F01D1420202D14FF0F7
:101F9800FF3070474FF00000704700BF00F026F890
:101FA8000C4880F30888002103E00B4B5B58435032
:101FB80004310A480A4B42189A42F6D3094A02E009
:101FC800002342F8043B084B9A42F9D318F098F9D9
:101FD8007047000000C00020485703080000002098
:101FE8006013002060130020985F00207047FEE710
:101FF80010B586B0002301244FF46022114801A9CE
:1020080001938DF80930039204938DF808408DF8F8
:10201800144023F033FA0B48214623F055FA0948B7
:1020280023F05CFA074823F05EFA0028FAD1054845
:1020380023F05DFA034823F05FFA0028FAD106B0CE
:1020480010BD00BF00240140014610B50D48012213
:10205800032323F05FFA0B48012123F051FA7F2074
:1020680024F08EF80748022123F09EFA0028F6D0C3
:102078000448022123F09EFA0248BDE8104023F0EC
:1020880090BA00BF002401400C4A0C2303FB012333
:1020980010B59C880CB9588010BD5B8803F11304F7
:1020A800844204DA142B07D9133B834204DC0C2343
:1020B80003FB012102238B8010BD00BFE02D00200F
:1020C8000A4B10B500241C7021464FF4E0720848F2
:1020D800FEF760F9074B43F604501C70064B1C7062
:1020E8000FF068FC054B187010BD00BF5C15002090
:1020F8002817002073190020F0180020F21800207B
:10210800074B1978013101F01F011970054B1A7836
:102118008A4203D1013202F01F021A70704700BFD1
:10212800F01800207319002010B50E4A0E2303FB87
:1021380000200D4A014614780C4A03FB042300F1E1
:102148000C0251F8044B914243F8044BF9D10A8828
:1021580000211A800E22FEF71DF9BDE81040FFF796
:10216800CFBF00BF60150020F018002028170020FE
:10217800084B1A5C002352FA03F111F0010FD8B290
:1021880002D00130C0B270470133042BF3D10120D3
:10219800704700BF2B1A002000F07F0000F5745034
:1021A8002DE9F84309300C46154698460FF002FC15
:1021B80000284FD043F63C37002638460FF0FAFB8C
:1021C800C0B25FFA86F988B120280FD04FEA5900CB
:1021D80000F5364037300FF0EDFBC0B208B10228E9
:1021E80004D10123B340227813432370113743F6F7
:1021F800C43301369F42E0D14BF2DE400FF0DAFBE8
:10220800C0B280B120280ED02B784BF2CD4043F0DD
:1022180001032B700FF0CEFBC0B220B1202802D0F2
:10222800012388F800304BF20F500FF0C3FBC0B207
:1022380080B120280ED02B784BF2CD4043F002031A
:102248002B700FF0B7FBC0B220B1202802D00123B9
:1022580088F80030BDE8F883034610465A1E10B5CA
:10226800032A1CD8DFE802F00E0E0207114A527842
:1022780002F0100203E00F4A527802F00802D2B2CC
:1022880072B10BE00C4A927802F04002D2B23AB135
:102298000A4A127802F003029A4200D140B10022A1
:1022A8000748105C984203D00132052AF8D1002172
:1022B800084610BDA85D0020DC390020773C0020CE
:1022C80020170020F8B5064643F63C35002428467A
:1022D8000FF070FBC0B2E7B268B120280BD07808C5
:1022E80000F5364037300FF065FB012803D1A040D8
:1022F80033781843307001341135082CE7D1F8BD14
:1023080003780E2202FB0313084AD3189978002396
:1023180051FA03F010F00100DAB202D0501CC0B23A
:1023280070470133082BF3D1704700BF28170020EE
:102338002DE9F04101248C40284A29490346E4B29A
:10234800107891F800C019E0264F0E2606FB00769B
:10235800F178A9B996F80680B8F1000F10D196F86F
:102368000580B8F1000F0BD196F80480B8F1000F82
:1023780006D1F67926B9013000F01F00054626E09F
:10238800FBB1012B05D0022B06D10E2101FB0077F2
:1023980039790C4218D014E0042B04D10E2101FB2A
:1023A8000077B9790CE0032B04D10E2101FB0077EB
:1023B800797905E0052B07D10E2101FB0077F97922
:1023C80011B11570BDE8F081013000F01F006045C3
:1023D800BAD11570FF20BDE8F08100BF7319002045
:1023E800F0180020281700202DE9F043444D454BF4
:1023F8002A780E2101FB0232917A85B0044698466C
:1024080039B101390523594301F56E51443189B277
:1024180001E043F6C431204604220FF0DCFA2B78A1
:102428000E2505FB038393F80B80364E344FB8F125
:10243800000F25D131232371073363713B7801A83D
:102448006B430422F15E06F087FA3B7802A805FB8D
:1024580003630222997A06F07FFA3B780DF10A00AD
:1024680005FB03650322697A06F076FAA01D01A927
:102478000922FEF765FA4FF00F0984F8108012E080
:10248800B8F1010F0FD132232371053363713B7803
:102498004FF0080905FB036393F90130E3713B78BA
:1024A8005D43735BA371002320461A4612E010F8BF
:1024B800011BA1F13005EDB2092D04D8EB18302924
:1024C800DBB203D004E037395B1800E00A33DBB233
:1024D8000132D2B24A45EAD10F21B3FBF1F108012A
:1024E800411A5B1AC3F10F03DBB2092BA35401D8BD
:1024F800303300E03733A35405B0BDE8F08300BFA4
:102508002617002028170020024B1A7842F00102F3
:102518001A707047911C002008B50C4B0C4A1B78A8
:102528000E2101FB0323D97A21B101290CBF09210E
:10253800002100E0102140221346064806F030F83A
:10254800054B1A7842F002021A7008BD26170020BF
:1025580028170020F3180020911C0020034B1A783C
:1025680002F0F8026FF3C3021A707047911C002042
:10257800024B1A7842F004021A707047911C00202E
:10258800024B1A7842F008021A707047911C00201A
:1025980038B5114B1C7814F0010502D1FFF7B4FFD0
:1025A80005E004F00405EDB21DB9FFF7E1FF284688
:1025B80038BD04F00805EDB215B9FFF7E1FFF6E7FD
:1025C80004F00204E4B21CB9FFF7A6FF204638BDA8
:1025D800FFF7C4FF012038BD911C0020014B18787B
:1025E800704700BF5C15002030B51E4B85B01B78C6
:1025F8000446002B34D11C4D2B78034113F0010FF6
:102608002ED01A4B1A4A1B780E2101FB0323DA78C5
:10261800024112F0010F1CD11B79034113F0010391
:1026280017D110F0010001F1F1014FEA540206D070
:1026380001320091019302926D20FE3905E00132CA
:102648000091019002923C20012103220B460FF0D9
:102658002FFA012313FA04F42B7823EA04042C70CC
:1026680005B030BDF2180020E918002073190020C9
:1026780028170020037830B513F0010F144A4FF0E3
:102688000E0419D104FB01210133012212FA03F3CC
:10269800CD7825EA0303CB7004780D79A41812FAD3
:1026A80004F425EA04040C7103789B189A408B788B
:1026B80023EA02028A7030BD04FB0121013B01229A
:1026C80012FA03F38A7822EA03038B7030BD00BF45
:1026D8002817002010B500230278590052FA01F497
:1026E80004F00304022C05D1013414FA01F122EAA2
:1026F800010202700133042BEED110BD2DE9F04F19
:1027080085B00192BDF838201C46744B0092DA78E7
:10271800054612F020028B4640F0D9808DF80E2035
:102728008DF80F208DF80D20DCB99B7803F040035D
:10273800DBB21BB101238DF80F3020E0684B5B78CA
:1027480003F00203DBB21BB101238DF80E3016E053
:102758000DF10F010DF10E020DF10D03FFF71CFD38
:102768000DE0012C0BD19B7803F04003DBB223B9B9
:102778000DF10F00FFF7A6FD01E08DF80F409DF861
:102788000F3023B99DF80E00002800F0A38044B94B
:1027980005F07F01490001F574510DF10A00663119
:1027A8000AE0012C0BD1E90101F51C4101F5B471D6
:1027B8000DF10A0001EB4B0102220FF00CF9BDF9F3
:1027C8000A3013B9002C00F08480009B33B9454BC4
:1027D800454F93F80080FFF793FC08E0434B444FC4
:1027E80093F8008008F1010202F01F021A700DF13F
:1027F8000F00FFF76FFF002C44D1BDF80A3069B213
:1028080040F6B83212EA210238BF4FF47A72D21871
:102818000E2303FB08F3ADF80A20FA529DF80F9037
:10282800224649460120FE18FFF716FD4946F0707A
:1028380022460220FFF710FD86F8029030719DF8BD
:102848000E90224649460420FFF706FD4946B0711E
:10285800824622460320FFF7FFFC05F07F057071D2
:102868003572BAF1000F00D128B1224B1B7813B989
:102878009DF80D3000E00023F37186F809B0019A45
:10288800B2721CE0012C1AD10E2303FB08F3BDF829
:102898000A202046FA529DF80F6000223146FD18A2
:1028A800FFF7DAFC3146E87000220220FFF7D4FC7B
:1028B80000232871AE70AB716B71EB71AB720E2394
:1028C80003FB0877FC72009B0120BB8102E000201B
:1028D80000E0204605B0BDE8F08F00BFDC390020DD
:1028E800A85D0020F0180020281700205B150020A4
:1028F80060150020761C002073B5154B04461B7824
:102908000E46D3B11348214621F05FFF0546A0B912
:10291800012E04F1010606D12046FFF729FC009597
:102928000246812005E02046FFF722FC009502467A
:10293800982031462B46FFF7E1FE2146054821F055
:102948002EFF0548214602B0BDE8704021F032BF95
:10295800F1180020961B00208E1900202DE9F7435E
:102968007B4B04461B7843B17A4B1B7803F0240356
:10297800042B02D1002900F0E880774B774F1B78B1
:10298800002B00F0C7807648214621F01EFF002862
:1029980040F0C08007F5C470214621F016FF80463C
:1029A800002840F0B7803B1993F880302D2B01D0D8
:1029B800532B3AD16B4E357845B30FF057FB04F1E2
:1029C8000108054650B12046FFF7D2FB337802468E
:1029D8001E33009393204146002307E02046FFF76B
:1029E800C7FB00950246414693202B46FFF786FE1B
:1029F8000FF03CFB014628B1337803201E330093C7
:102A0800002101E0009003200A4680E02046FFF7FD
:102A1800AFFB611C02462B4693200095FFF76EFE24
:102A28000095032029462A4671E0542B09D12046F7
:102A3800FFF79EFBCDF800800246611C94204346B8
:102A480066E0462B474D20D12E78BEB10FF00EFB25
:102A580004F10109064648B12046FFF789FB2B78A7
:102A680002461E3300939A20494622E02046FFF78B
:102A78007FFB0096024649469A2025E02046FFF74C
:102A880077FB009602469A2039E02E78002E2CD04B
:102A98000FF0ECFA04F11C09064660B12046FFF776
:102AA80067FB2B7802461E3369F07F000093C0B2A3
:102AB800611C434609E02046FFF75AFB024669F0CD
:102AC8007F000096C0B2611C3346FFF717FE0FF077
:102AD800CDFA21B2024628B12B7803201E33009389
:102AE800002214E00090032011E02046FFF740FB8D
:102AF800024604F11C0060F07F000096C0B2611C21
:102B08003346FFF7FBFD009603202146324601239A
:102B1800FFF7F4FD124821463F1921F040FE97F8CF
:102B280080302D2B0AD0532B08D0542B06D0462B9F
:102B380004D00D48214621F048FE30B10B4821460B
:102B480003B0BDE8F04321F035BE03B0BDE8F08323
:102B58005E150020841B0020F1180020202C002086
:102B6800961B0020EE1B0020A82D00208E1B0020A5
:102B7800002302780E2101FB0232044901338A182E
:102B88000021062B9170F4D1704700BF2817002050
:102B9800064B00201870064B1A78064B1B789A4291
:102BA80002D00146FFF7C4BBFF2070475C15002028
:102BB800F0180020731900200121814038B5114B0D
:102BC800C9431A78104BC9B202F0030203F5E07446
:102BD800012A04D1DD7801EA0505DD7005E0022A45
:102BE80003D11D7901EA05051D710E33A342EFD10A
:102BF800FFF7FAFC43F604500EF0DCFE034B1870A6
:102C080038BD00BF773C002028170020F2180020AC
:102C18002DE9F743A34D8DF807002B78A24C1BB183
:102C28002378C2B29A4204D043F604500EF0C2FE92
:102C380028709DF8073023709C4C2278072A00F2F0
:102C48002D81DFE812F008002400360054005D00F2
:102C580072008D00BA00964A3C211170954A1946B7
:102C6800107800F00300FFF763FB934BFF28187000
:102C780000F0368120F0AAFA904B002093F87420D7
:102C880042F0010283F874208D4B187064E0884B81
:102C98001B78002B00F0248120F060FC012840F014
:102CA8004D812378142201332370864B01381A7022
:102CB80047E17F4B1B78002B00F01281814E307862
:102CC80008B901234AE020F049FC022804D020F08A
:102CD80045FC032840F0328120F078FA237804225A
:102CE800013323701D233370774B1A7026E1704B24
:102CF8003C221A707548FFF777FB2378013323705D
:102D08006B4B1B78002B00F0EB806E4B1D78002D71
:102D180040F014811020FFF73BFC002800F01181DF
:102D280023782846013323700BE1614B1B78002B75
:102D380000F0D68005F09EFC002800F00281614B6F
:102D48007D221A705E4B002018705C4B93F874203B
:102D580042F0010283F87420237801332370F0E0F5
:102D6800534B1B78002B00F0BB8020F0F7FB0128A9
:102D7800544E03D020F0F2FB03280FD19DF8072012
:102D8800012111FA02F2524B197821EA02021A7053
:102D980064233370237801332370CFE03078002820
:102DA80040F0CC80484A032323701378013BDBB200
:102DB8001370002B00F09480C3E0404A414E92F813
:102DC8006A201AB13278002A40F0B88000223270A6
:102DD800013212FA03F3DFF8E0803E4F98F8001052
:102DE8004FF00E0909FB0172DB4392F803E0DBB2F6
:102DF80003EA0E0E907882F803E092F804E003EA02
:102E08000E0E0340937082F804E00DF10700FFF7FF
:102E180031FC98F8003009FB0372D278DFF89490FF
:102E28002AB999F8002002F00302012A0AD00E22DA
:102E380002FB03721279B2B999F8002002F003027A
:102E4800022A10D10E2202FB0377BA785AB9224F10
:102E58003A789A4207D11848FFF78AFE3B7801333F
:102E680003F01F033B7099F800009DF8071000F06D
:102E78000300FFF75DFA144B0422FF281A7088F844
:102E88000000164B42D0987800F04000C0B20028ED
:102E98003CD1032323701A33337052E00020207092
:102EA8004FE000BFF21800205F1500205C150020DD
:102EB800EA180020773C002026170020FC3B002061
:102EC8005D1500205A150020E8180020F31800208E
:102ED800E91800202817002073190020DC39002089
:102EE800FFF73CFB0023237020F070F92B78013B9F
:102EF800DBB22B702BB1144B9B7803F04003DBB291
:102F0800F3B19DF80700FFF757FE19E09B780E4ACA
:102F180003F04003DBB22BB1136843F400031360E2
:102F2800FFF7CEF8FFF71AFB20F050F900232370C3
:102F380043F604500EF03EFD287001E0002000E04A
:102F4800FF20BDE8FE8300BFDC390020044B1A785F
:102F58000AB1013A1A701B780BB9FFF72DBE7047FA
:102F6800F2180020044A054B10781B7803EA501029
:102F780000F00100704700BFDC3900205D1B002015
:102F8800044B054A1B781078C3F3400303EA10107A
:102F9800704700BF5D1B0020DC390020034B044A4A
:102FA8001B78D078C3F38003184070475D1B00205E
:102FB800DC390020044B054A1B78D078C3F3C003E2
:102FC80003EA5000704700BF5D1B0020DC39002079
:102FD800044B054A1B78D078C3F3001303EA90002A
:102FE800704700BF5D1B0020DC390020044B1878B7
:102FF800044BDB785B005BB2DB1103EAD01070474F
:103008005D1B0020DC39002008B50E2104481CF0A7
:1030180043FB044B5B7803EA000000F0010008BDA5
:103028007C1900205D1B002070B500241BE0304691
:10303800E9B21CF06FFB80B14FF43663634334226E
:1030480002FB05330A4AD3181B7A13F0010F04D088
:10305800084B1878C0F3001070BD0135382DE6D143
:103068000134022C02D0E6B20025E0E7002070BD52
:10307800503D00205D1B002008B51BF067FC034B8A
:103088001B7800EA931000F0010008BD5D1B0020CA
:10309800044B054A1B78D078C3F3401303EAD000E9
:1030A800704700BF5D1B0020DC3900202DE9F74F79
:1030B800FFF758FF8246FFF763FF8346FFF76EFF6F
:1030C8000190FFF777FF8146FFF782FF0446FFF77D
:1030D800ABFF0546FFF7DCFF8046FFF7CDFF07464D
:1030E800FFF784FF0646FFF78FFF019B45EA0404BC
:1030F8009B0043EA4B0343EA0A0343EAC90343EA52
:10310800481343EA871343EAC61343EA0023E0B2AD
:1031180043EA0010BDE8FE8F044B987800F00F00DA
:10312800A0F10203584240EB03007047CB1900207E
:10313800044B987800F00F00A0F10102504240EBD8
:1031480002007047CB190020044B987800F00F005C
:10315800A0F10301484240EB01007047CB19002061
:10316800054B987800F00F00A0F1060CDCF1000088
:1031780040EB0C00704700BFCB190020514AF0B556
:1031880013781446012B29D003D3022B40F09880E2
:103198005EE04D484D4B047819786FF3C304047012
:1031A80001F0F80158786FF3C301197000F080013D
:1031B800C9B2002900F08480012111709C78062290
:1031C80004F00F04544302464148005D60F30602D0
:1031D8005A701A7861F302021A70F0BD3B494D78B3
:1031E8000B4625F07F00002838D00A7802F0080244
:1031F800D2B222B9344A117841F0080111709A7894
:1032080002F00F02012A04D12F4A117841F001017E
:10321800117015F07F0F53D119789E7801F00700CF
:10322800062206F00F0602FB0606294F5D78BE5DF2
:10323800013066F3060500F007005D7090FBF2F5BB
:1032480002FB150262F30201197002232370F0BD1C
:103258001E494D780B4625F07F0028B98B7860F31E
:1032680003038B701070F0BD174A11786FF3C30118
:103278001170997801F00F01012903D111786FF3CA
:103288000001117015F07F0F1AD119789E7801F09E
:103298000700062206F00F0602FB06060C4F5D78B3
:1032A800BE5D013066F3060500F007005D7090FB17
:1032B800F2F502FB150262F3020119700123237073
:1032C800F0BD00BF1A1A00208D190020CB1900206C
:1032D800E861020810B51F4A1F4B92F9031009B1A3
:1032E800002231E008B1032119701978032930D878
:1032F800DFE801F00209192C1178002929D01548B6
:1033080081700121197092F90200124920B1134B02
:103318001A786FF3861217E0487808B9032213E089
:1033280088700221197092F902100A4889B90B4A6B
:10333800147861F386141470026861F30F22D1B215
:1033480061F31742026001221A7010BD002111605A
:10335800197010BDF01B00208B190020503B002075
:1033680070B543F6EF23044643F6F020012A08BF60
:1033780018460D460EF01EFB2678C0B20640164CC5
:103388000CD001201CF08CFB43F6EE200EF012FB53
:10339800236860F307036FF30F2314E02B781842B8
:1033A80012D030461CF07CFB0C4B43F6EE201A88FA
:1033B80066F34D321A800EF0FDFA2368C0B260F34E
:1033C800070360F30F23236094F9003013B1024B15
:1033D8000F22DA7070BD00BFF01B0020841B002094
:1033E80008B543F6FB200EF0E5FA014B187008BD4E
:1033F8008C190020014B1870704700BF671B002014
:10340800024B1A5C6FF303021A547047741A0020B7
:1034180070B50C46C10001F5CE411B48BF310822EA
:103428000EF0D9FA002518482946EEB221F0CDF958
:1034380008B9237823BB154B2278EB5C1A421FD1BD
:103448003046FFF7DDFFF6084BF2DF5030180EF07C
:10345800B1FA05F00703C0B2184110F0010F0FD1FF
:103468000B48294621F0B1F950B12946084821F006
:10347800A1F9074B06F5CC40CE30995D0EF090FAD5
:103488000135402DCFD170BD691B00202B1A0020BB
:10349800CE19002038B546F2167540242046FFF7AD
:1034A800AFFFA5F5CC43094AD63BD15C11F0100F0C
:1034B80006D06FF30411D154284600210EF070FA9B
:1034C8000134E4B20135E92CE8D138BD741A002082
:1034D8003F287FB5054607D800F5E24041300EF099
:1034E80069FAC3B22BB925E1964A1478002C00F08A
:1034F8002681954E725D02F00F014C1C04F00F04FA
:1035080064F303023F2D725533D8002C00F0178165
:1035180001339C4240F010818C4B5A1992F880205C
:10352800522A725D03D161F30302725504E16FF30D
:103538000302EC081B19725593F8902105F0070354
:1035480052FA03F313F0010F40F0F880294680483F
:1035580021F025F97E4B04F5CC40195DCE300124CD
:103568000EF01EFA2D1902230093019402951820DB
:10357800DAE0002C00F0E380724B1B7801339C42A8
:1035880040F0DA80735D05F5CC406FF30303D63065
:10359800012173550EF004FA735D43F0100373555F
:1035A800A5F14003DBB2032B07D8042200920133B4
:1035B800023201920293192031E0A5F14803DBB2EF
:1035C800032B0CD804220092013303320192029398
:1035D8001A200121043A0B460EF06AFAAEE0502D8B
:1035E80007D10423009301240333019302941B2081
:1035F8009AE0572D07D10423009301240333019344
:103608000294212090E0A5F15B03DBB2012B09D8DD
:1036180004220092013302320192029322200121F6
:10362800033AD8E75D2D06D1042300930193043BA8
:103638000293284662E05E2D07D1042300930133EC
:103648000193053B02935E2058E0A5F15F03DBB2CE
:103658006F2B09D804220092013392180192029329
:1036680033200121053AB6E705F13103DBB2032B1C
:1036780007D80422009201330332019202935F209B
:10368800A7E705F12903DBB2012B07D80422009232
:10369800013303320192029360209AE7DA2D07D1B1
:1036A800042300930124043B0194029361203BE02E
:1036B800D92D07D104230093023B0193023B0293C7
:1036C80062201BE0DD2D08D1042300930322043B74
:1036D80001920293632001217DE7DB2D06D10423AB
:1036E8000093043B01930293642007E0DC2D08D18A
:1036F80004230093043B01930293702001210322C9
:1037080069E7DE2D07D104230093012402330193D6
:103718000294682008E0E22D10D1042300930124CC
:103728000233019302946A202146032223460EF0B5
:10373800BFF904E01C4602E0002400E00124204612
:1037480004B070BD00000020741A0020202C002056
:10375800CE190020024B185CC0F30010704700BF60
:10376800741A0020F8B508220E4600210746FCF717
:1037780011FE46F2BF7500243378234113F0010F80
:1037880008D02946064808220EF025F9384604498B
:1037980020F0D3FF01340835042CEDD1F8BD00BF6B
:1037A800731B0020024846F2CE6108220EF013B9BE
:1037B800CE19002070B5044600F56A5044300EF06A
:1037C800F9F80B4D06462B7813F0010F02D1CC20E7
:1037D80021F0E8FD2B8843F001032B80054B1E5593
:1037E800054B13F8242042F0010203F8242070BD91
:1037F800841B0020AF1900209E190020024B185C82
:10380800084100F0010070472B1A002070B50546EA
:103818000024094BE0B2E618E35C4BB12946FFF7F8
:10382800EDFF28B1002333700448214620F0C2FF81
:103838000134402CEDD170BDA61B0020BB1900201F
:1038480038B5054600242846E1B2FFF7D7FF10B186
:10385800044BE35C23B90134042CF4D1002038BDB7
:10386800012038BDAF19002038B505460EF0FEFB23
:10387800A0B100242846E1B2FFF7C0FF40B1084BD1
:1038880013F8243013F0010F02D0064BE35C23B188
:103898000134042CEED1002038BD012038BD00BF12
:1038A8009E190020AF190020F8B5114800214022C8
:1038B800FCF770FD46F2BF75002401270D48294624
:1038C8000822A7400EF087F8FFB2002609483146C3
:1038D80020F07BFF20B1064BF25C47EA0202F2546B
:1038E8000136402EF2D101340835042CE5D1F8BD5B
:1038F8002B1A0020731B00202DE9FF4100263446B7
:10390800B0461A4B1B78234113F00102184B23D001
:10391800184F1D5D17F82430A84538BFA84613F086
:10392800010F1AD0CDB965F3000307F8243023B28C
:103938000122F71902935B2029462B460092019534
:103948000EF0B6F87B78B878F9781843621C2B46E5
:103958000095FEF7D3FE00E01A5501340436042C16
:10396800CFD1054B83F80080BDE8FF818C1900207A
:10397800AF1900209E1900208A19002010B50C4BA1
:103988001B78A3B10B4B1B788BB100240A48214646
:1039980020F01BFF40B10948214620F016FF18B956
:1039A80020460121FEF7DAFF0134402CEED110BD8C
:1039B800F11800205E1500208E1B00201E23002019
:1039C8002DE9F043324C334A238800266FF38613DF
:1039D8006FF3C4032380304B304F85B016701E70D0
:1039E8009146984617F8013B5BB32278D20052B251
:1039F80043EAA2122388402E62F3C40343F0400333
:103A080023801ED000253046E9B2FFF7F7FEA8B1A3
:103A180017F8013C13F0010F06D00122AA4099F8CB
:103A280000100A4389F8002013F0020F06D0012382
:103A3800AB4098F80020134388F800300135042D76
:103A4800E1D10136F6B2412ECCD1237803F04005FE
:103A5800EDB2D5B903F02403042B0BD1FFF78EFF89
:103A6800FF2300934020294601222B460195029509
:103A78000EF01EF8238800226FF345136FF38203BC
:103A88006FF3C4032380064B1A7005B0BDE8F083BA
:103A9800841B0020EC3A0020093B0020D9190020A3
:103AA800681B002010B500240548214620F08DFE33
:103AB80008B9044BE0540134402CF5D110BD00BFC7
:103AC8005F1B0020D919002010B5127804469DF814
:103AD8000810DAB1D3B111B10D4920F023FEACB111
:103AE800082246F2CE610B480DF075FF21460948C1
:103AF80020F023FE0749082246F2CE600DF065FF4C
:103B080005480449BDE8104020F02DBE10BD00BF97
:103B1800B82D002074190020CE19002030B5064BAE
:103B280004781D7824EA05040C7001781B7823EAD0
:103B38000103137030BD00BF8C19002038B50A4D41
:103B4800002415F8013F2D2B09D0532B07D0542BF7
:103B580005D0462B03D00548214620F02BFE013422
:103B6800402CEED138BD00BF9F2C00208E1B0020BA
:103B780010B50F4820F0CEFD00240E48214620F055
:103B880024FE80B10C4BE31893F88030482B06D004
:103B980003D82D2B03D0462B00E0542B03D1044827
:103BA800214620F0FCFD0134402CE6D110BD00BFB9
:103BB8001B1A00208E1B0020202C0020094A0A4BCB
:103BC800117831B1997801F00F01814201D00021BB
:103BD80011709A7860F303029A705A7842F0800262
:103BE8005A7070471A1A0020CB1900202DE9FF419E
:103BF8001E466D4BDDF82880154604461A780F4698
:103C080000236A4911F8231011F0010F05D0012192
:103C18009940C1F10F0101EA02020133042BF0D1EE
:103C2800634B1A70002C6FD014F0010F0AD0FF23D9
:103C380001210093FF3B0193029352200A460B4651
:103C48000DF036FF14F0020F0AD0FF230121009374
:103C5800FF3B0193029353200A460B460DF028FFC1
:103C680014F0040F0AD0FF2301210093FF3B0193B6
:103C7800029354200A460B460DF01AFF14F0080F61
:103C88000AD0FF2301210093FF3B019302935520A3
:103C98000A460B460DF00CFF14F0100F0AD0FF2354
:103CA80001210093FF3B0193029356200A460B46DD
:103CB8000DF0FEFE14F0200F0AD0FF23012100931F
:103CC800FF3B0193029357200A460B460DF0F0FE86
:103CD80014F0400F0AD0FF2301210093FF3B01930A
:103CE800029358200A460B460DF0E2FE14F0800FAE
:103CF8000AD0FF2301210093FF3B0193029359202F
:103D08000A460B460DF0D4FECFB1002430462146BA
:103D180020F05BFD60B1FF230093FF3B0193631C20
:103D28001BB2012102935A200A460B460DF0C0FE31
:103D380021463046013420F03DFD402CE6D1BDB18E
:103D480000244046214620F040FD70B1012D0CD1E1
:103D580004230093DB180193631C1BB202937420A5
:103D6800294603222B460DF0A3FE0134702CE8D11E
:103D78000F481049104AFFF7D1FE104B00221A7065
:103D880001320092063201920832029209490A4A27
:103D9800074809F073FE0A4B3C2251201A7004B000
:103DA800BDE8F0410EF04EBA8C1900209E19002093
:103DB800FC1C0020E51D0020D81D0020C11C00208F
:103DC800AE19002037B5FFF771F904460E4820F008
:103DD800CFFCD0F1010538BF00250C480E211BF09F
:103DE8005BFC10B114F4807F03D124B95DB1224685
:103DF80002E0012200E00022044B204600932946FD
:103E0800014BFFF7F3FE3EBD6C1A00207C19002021
:103E1800054B03EBD00393F8903100F0070053FAF9
:103E280000F000F001007047202C002010B50F4B67
:103E380004461B7813F0010315D0FFF701FD28B9DC
:103E48000B4B1B1993F88030462B0DD10EF00EF951
:103E580018B92046FFF7DCFF30B10648214620F0AC
:103E68009EFC012010BD184610BD00BF841B002019
:103E7800202C00206C1A0020024B1878003818BF3C
:103E880001207047AE19002010B5034C04EB8303E2
:103E980058709970DA7010BD9E19002010B5002472
:103EA8000948002100190E220E34FCF773FAB4F504
:103EB800E07FF5D1054A00231370054A0021995285
:103EC8000233AA2BF9D110BD601500205B15002024
:103ED8005A1E00207FB5474B04461B780E46AA2B76
:103EE80078D04548214620F070FC0546002871D15D
:103EF8002046FFF79BFF00286DD14048214620F05F
:103F080064FC50B93E48214620F05FFC054620B9C4
:103F18002046FFF7DDFA00285DD13A4B1B7823B91C
:103F2800394B1B7813F0010F09D1384BDB7803F0BC
:103F38002003DBB21BB9364B032283F84020012E45
:103F480005D82E48214620F040FC40B142E0022E20
:103F580007D12B48214620F038FC10B13AE0274819
:103F680000E02748214620F01AFC2A48214620F084
:103F780021FC022E15D10125294603222B46009645
:103F88004A206619019502960DF092FD2046FEF72B
:103F9800EFF800230246314618200093FEF7AEFBE7
:103FA80019E0012E09D102230093631C02930196A4
:103FB800122031460322334609E07EB9012102234B
:103FC8000093631802930191112003220B460DF010
:103FD8006FFD03E00025284604B070BD2046FEF7BB
:103FE800C7F8024601200023211800930125FEF797
:103FF80085FBF0E7671B0020CE1900208E190020F2
:10400800E61B00208C190020551E0020DC390020FA
:10401800D9190020961B00202DE9FF4704460D46BC
:104028007548214620F0D1FB8146002840F0DF800A
:104038002146714820F0B3FB7048214620F0BAFBB6
:104048006F4E0DBB01274FF00208E3190293424659
:10405800032039463B46CDF8008001970DF028FD36
:10406800327862B10EF002F8024630B13378404639
:104078001E33009321462A4604E0009000E0009297
:10408800404621463B4628E0012D2BD15D4B04F5E7
:10409800E24041301F5D0DF08DFC07F00F078742AD
:1040A80009DA631C022202930E2029462B4600924D
:1040B80001950DF0FDFC327892B10DF0D7FF024664
:1040C80038B14F4B0D201B7821461E330093002238
:1040D80002E000900D2021460123FEF70FFB5EE071
:1040E8000092F7E7022D0BD101230193E318029305
:1040F800142049462A464B4600950DF0D9FC4EE05F
:10410800032D4CD101272A464FF0020804EB070A79
:104118004D2039463B46CDF800800197CDF808A0E0
:104128000DF0C6FC35783DB30DF0A0FF024630B166
:10413800337840461E33009321464A4602E00090F9
:10414800214640463B46FEF7D9FA0DF08FFF671C23
:10415800054648B12046FEF70BF8337802461E3371
:1041680000931A2039462CE02046FEF701F8009506
:10417800024639461A202DE021462A463B4640464B
:104188000095FEF7BBFA2046FDF7F2FF51460246BE
:104198002B461A200095FEF7B1FA384628E0357804
:1041A800EDB10DF063FF04F11C06054658B1204639
:1041B800FDF7DEFF124B02461B7830461E33009394
:1041C800611C002307E02046FDF7D2FF0095024658
:1041D8003046611C2B46FEF791FA012008E0204684
:1041E800FDF7C6FF0095024604F11C00F1E7002028
:1041F80004B0BDE8F08700BF8E1B0020961B00208E
:10420800EE1B0020741A0020064B1B1893F840017F
:10421800492804D0452814BF0320022070470120F4
:10422800704700BF202C00202DE9F041244F0024C6
:104238003C702448214620F0C8FAE5B2224B0028F9
:1042480037D01E5D3B789E4200D303B93E70002EE6
:1042580030D131461C484022FCF79CF81B4B1C48C7
:1042680003EBD50393F8888104F0070348FA03F8B1
:10427800214608F0010820F0A8FA68B9B8F1000F43
:1042880002D02846022101E028463146FFF7C4FE45
:1042980028460DF0D7FF0DE0B8F1000F0AD12846E7
:1042A800FFF7B2FF0B4BDB7803F02003DBB20BB94F
:1042B800094B18550134402CBBD1BDE8F08100BF33
:1042C800EE1B0020BB190020A61B0020202C00207C
:1042D8008E1B0020DC390020D91900202DE9F04F71
:1042E800914B8BB01B7813F0010F06D08F4B1A78C7
:1042F8006FF386121A7001F05EBA8D498D4A0B78F9
:1043080010788D4D984218BF8C49137018BF0B70E8
:104318006B7803F00803DBB24BB143F6CF200DF006
:1043280049FB864B18702B886FF3CB232B80844B6B
:104338001B78AA2B08D18349AA3B0B702B8843F022
:1043480080032B8000F0BCBE6A787B4B02F0100221
:10435800D2B27D4CA2B11A886FF30C321A807B4B13
:104368001B7823B97A4B1B7813F0010F08D1E37837
:1043780003F02003DBB21BB9764B032283F84020FD
:104388002368754F6FF3186323603A7802F00202CE
:10439800D2B232B96B494A781AB16B4A43F080738A
:1043A8001360E67816F0010648D05D20FFF7D2F9D1
:1043B80000285AD16B78DFF8808103F00203DBB262
:1043C8002BBB5D30FFF784F8064600BBB8F8003019
:1043D800012143F40073A8F800300423032200935A
:1043E800019302900B460D200DF062FB45200DF065
:1043F80029FF3146012233460D200096FEF77EF94B
:1044080009203146324601230096FEF777F96B788A
:1044180003F00203DBB243B34C4B1B7823B94C4B7C
:104428001B7813F0010F20D1E37803F02003DBB2EF
:10443800DBB9484B032283F8402016E06B7803F081
:104448000203DBB26BB13146324601230A200096E3
:10445800FEF754F98D203146012233460096FEF7C7
:104468004DF92B886FF349232B802368354A6FF366
:104478005963236093787BB1D37823B93B7813F0E1
:104488000C0F05D108E03B7803F00C03042B03D094
:10449800236843F000732360E17801F00201C9B298
:1044A80000295BD05E20FFF755F9002865D16B78AD
:1044B800214F03F00403DBB2EBB95E30FFF708F8D5
:1044C8000646C0B93B88012143F480633B8004233E
:1044D800009301330322019302900B4617200DF03D
:1044E800E7FA45200DF0AEFE0D2031460122334695
:1044F8000096FEF703F96B7803F00403DBB2002B98
:104508003BD0124B1B7823B9114B1B7813F0010FCA
:1045180033D1E37803F02003DBB273BB0D4B0322E6
:1045280083F8402029E000BFFD1C0020503B0020FC
:10453800711B0020721B0020841B0020EF1B002031
:10454800671B002060130020DC3900208C19002034
:10455800551E0020D91900201E2C00206B7803F06E
:104568000403DBB22BB18D2001220B460091FEF72C
:10457800C5F82B886FF38A232B8023684FF05F0BD5
:104588006FF3DF732360002696E00698F9B21BF0FC
:10459800C1F8002875D04FF436637343342202FB08
:1045A8000733A749A8F15E0ACB1803F108021B7A62
:1045B8005FFA8AFA13F001034DD02368404643F0AE
:1045C800004323600592FFF7C5F8059A002864D1D7
:1045D800937813F0040F20D14046FEF779FF059A2F
:1045E8008146D0B99378012143F0040393700423E2
:1045F8000093DB180322019332200B46CDF808A064
:104608000DF056FA4A200DF01DFE0C2051460122ED
:104618004B46CDF80090FEF771F84FF436637343BC
:10462800342202FB0733864AD3189B7A13F0040F0F
:1046380033D0844B1B7823B9834B1B7813F0010FBD
:104648002BD1E37803F02003DBB233BB7F4B03228B
:1046580083F8402021E0927812F0040F05D08C20D6
:10466800514601220093FEF749F84FF4366373432D
:10467800342202FB07337249CB189A7A6FF382020D
:104688000AE04FF436637343342202FB07336C4A63
:10469800D3189A7A60F382029A72013708F10108F6
:1046A800382F5FFA88F87FF470AF01360BF1380BBA
:1046B800022E5FFA8BFB04D0F3B20693D84600278C
:1046C80063E72368624923F080636FF39E73236076
:1046D8000B79002B00F0B8835E4ADFF87CB10692B4
:1046E8004FF0CF0800261BF8011F37460136002976
:1046F80052D0236808F1710A43F080635FFA8AFA9E
:1047080023605046FFF726F800285CD118237B4326
:10471800DFF8489119F8032012F0100F23D1504602
:104728000593FEF7D5FE059B8246E0B919F80320EC
:10473800012142F0100209F80320042300930233F8
:10474800019333B2032202930F200B460DF0B0F908
:1047580045200DF077FD0D20514601225346CDF836
:1047680000A0FDF7CBFF18237B4319F8033013F0A3
:10477800100F28D0334B1B7823B9334B1B7813F019
:10478800010F20D1E37803F02003DBB2DBB92F4B14
:10479800032283F8402016E018237B43DFF8BC90FF
:1047A80019F8033013F0100F05D08D2001220B46A5
:1047B8000091FDF7A3FF18237B4319F803206FF33B
:1047C800041209F80320069B13F8011F0693002919
:1047D80046D02368404643F080432360FEF7BAFF83
:1047E800002854D14FF0180909FB07F9DFF86CA02D
:1047F8001AF8093013F0200F49D14046FEF768FE39
:104808000746002843D11AF80930012143F0200354
:104818000AF80930042300930333019333B20322C7
:1048280002934B200B460DF043F950200DF00AFD82
:104838001920394601223B460097FDF75FFF26E025
:10484800503D00208C190020551E0020D919002049
:10485800601300205E3A0020833A00208A3A002044
:1048680018237B43DFF8A89219F8033013F0200FC0
:1048780005D0992001220B460091FDF73FFF182330
:104888005F4319F807306FF3451309F8073008F14B
:104898000108042E5FFA88F87FF425AF934B197846
:1048A800002945D02368E22043F080632360FEF7A7
:1048B80051FF00284BD18E4B1A78984612F0400FC2
:1048C8001FD1E230FEF704FE0746D0B998F8003051
:1048D800032243F0400388F8003000960623033E85
:1048E800314601936920334602960DF0E1F84520E0
:1048F8000DF0A8FC0D20394632463B460097FDF7DF
:10490800FDFE98F8003013F0400F20D0794B1B784B
:1049180023B9794B1B7813F0010F18D1E37803F012
:104928002003DBB29BB9754B032283F840200EE0CD
:104938006F4E337813F0400F05D08D2001220B46BF
:104948000091FDF7DBFE33786FF3861333706C4B01
:10495800197800292DD02368502043F08043236024
:10496800FEF7F8FE002833D1614E337813F0200F9C
:104978002ED15030FEF7ACFD074648BB33780322F2
:1049880043F0200333700423012600930333314698
:1049980001931020334602960DF08AF850200DF04E
:1049A80051FC1920394632463B460097FDF7A6FED2
:1049B8000EE04F4E337813F0200F05D099200122D6
:1049C8000B460091FDF79AFE33786FF34513337069
:1049D8004C4B1978002946D02368DE2043F08063C9
:1049E8002360FEF7B7FE00284CD1474B1A7898464B
:1049F80012F0400F20D1DE30FEF76AFD0746D8B925
:104A080098F80030012643F0400388F8003004236A
:104A180000930233314603220193672033460296FE
:104A28000DF046F845200DF00DFC0D2039463246B4
:104A38003B460097FDF762FE98F8003013F0400FF0
:104A480020D02C4B1B7823B92B4B1B7813F0010F6C
:104A580018D1E37803F02003DBB29BB9274B03227C
:104A680083F840200EE0284E337813F0400F05D02D
:104A78008D2001220B460091FDF740FE33786FF33D
:104A880086133370214B1978002943D023685720A7
:104A980043F080432360FEF75DFE002849D11A4E9B
:104AA800337813F0200F44D15730FEF711FD074635
:104AB80000283ED13378032243F0200333700423C7
:104AC800012600930333314601931F203346029693
:104AD8000CF0EEFF50200DF0B5FB19203946324698
:104AE8003B460097FDF70AFE23E000BF503A00203E
:104AF8003F3A00208C190020551E0020D9190020AB
:104B0800E03900200C3A00201D3A0020113A00201C
:104B18008A3A0020864E337813F0200F05D099206A
:104B280001220B460091FDF7E9FD33786FF3451339
:104B380033704FF000084FF05B094FF0D70A464634
:104B48007C4B08F10108F15C7B4F002949D02368B0
:104B5800484643F080632360FEF7FCFD002852D1ED
:104B680013237343FA5C12F0200F22D148460593B1
:104B7800FEF7AEFC059B8346D8B9FA5C012142F0EA
:104B88002002FA5404230093023301930FFA88F3A6
:104B98000322029320200B460CF08AFF45200DF0DB
:104BA80051FB0D20594601225B46CDF800B0FDF7B8
:104BB800A5FD13237343FB5C13F0200F23D05F4B39
:104BC8001B7823B95E4B1B7813F0010F1BD1E378D8
:104BD80003F02003DBB2B3B95A4B032283F8402019
:104BE80011E013237343FB5C13F0200F05D08D20D5
:104BF80001220B460091FDF781FD13237343FA5CF4
:104C08006FF34512FA54504BF15C002933D02368F6
:104C1800504643F080432360FEF79CFD00283ED1B8
:104C2800132303FB06735A7812F0200F37D150462E
:104C38000593FEF74DFC059B834680BB5A780121FE
:104C480042F020025A7004230093033301930FFAB1
:104C580088F3032202934C200B460CF029FF5020C6
:104C68000DF0F0FA1920594601225B46CDF800B044
:104C7800FDF744FD13E0132303FB06735B7813F081
:104C8800200F05D0992001220B460091FDF736FD33
:104C9800132303FB06735A786FF345125A702B4B94
:104CA8001322F35C002B53D002FB06F317F803B072
:104CB800CBF3801BBBF1000F22D143F6DE20059316
:104CC8000CF078FE059BD8B1FA5C012142F0400255
:104CD800FA5404230093DB1801930FFA88F3032294
:104CE80002932F200B460CF0E3FE47200DF0AAFAA2
:104CF8000920414601225B46CDF800B0FDF7FEFCD5
:104D080013237343FB5C13F0400F32D00B4B1B781B
:104D180023B90B4B1B7813F0010F2AD1E37803F06A
:104D28002003DBB22BBB074B032283F8402020E093
:104D38001D3A00205C3A0020E63900208C1900203A
:104D4800551E0020D9190020513A0020133A00209E
:104D58007243BA5C12F0400F05D089204146012207
:104D68000093FDF7CBFC13237343FA5C6FF38612B1
:104D7800FA5401360AF1010A09F10109022E5FFA13
:104D88008AFA5FFA89F97FF4DBAEDFF848A2482790
:104D9800023E1AF8011FB0460136002937D02368B1
:104DA800384643F080432360FEF7D4FC002847D1FF
:104DB8004FF01E0909FB08F9DFF81CB21BF809308F
:104DC80013F0200F3CD13846FEF782FB80460028BE
:104DD80036D11BF80930012143F020030BF80930C4
:104DE800042300930333019333B203220293132065
:104DF8000B460CF05DFE50200DF024FA19204146B8
:104E080001224346CDF80080FDF778FC18E01E2308
:104E180003FB08F3DFF8C09119F8033013F0200FF3
:104E280005D0992001220B460091FDF767FC1E234F
:104E380003FB08F819F808306FF3451309F8083030
:104E48000137042EFFB2A4D1A67806F00806F6B200
:104E5800002E40F03581594906915FFA86F8B8F17D
:104E6800000F0CBF4022702247F61B43099207939C
:104E780049F61E59002447464FF4E07A0AFB06FA21
:104E88004E495FFA84F851440891084621461FF0BC
:104E98009CFC48B949480AF1700A504421461FF061
:104EA80094FC002800F0F980444A4FF4E07A0AFBA9
:104EB800062A0AF1E00A504621461FF086FC00281F
:104EC80040F0EB80504621461FF069FCDFF80CA14A
:104ED8000FB9484600E007980CF06CFD8AF800000E
:104EE8009AF80000DFF8F4B0002800F0D680013806
:104EF800C0B28BF800000BF067FE002840F0CD80B0
:104F08009BF8000000F56A507C300CF053FD2C4BE8
:104F1800C0B2187027B92B4B4B4413F85EAC03E0B2
:104F280006990B1993F850A100EA0A0ABAF1000F82
:104F380000F0B380089821461FF047FCDFF890B0D6
:104F480000B31E4A4FF4E07000FB06202146703083
:104F58001FF03BFCB0B91C49012F0B784AEA030A41
:104F68008BF800A056D13823B8FBF3F203FB128369
:104F78004FF436614A43DBB2342101FB0323134A61
:104F8800D31841E00D4B4FF4E07000FB063021468A
:104F980070301FF01AFC38B1089821461FF015FC34
:104FA80010B909490B7804E0074A13781AEA030F85
:104FB80016D023EA0A0A8BF800A02BE098280020D4
:104FC800961D00202090FF1F8C190020503D0020C6
:104FD800FC1C00203A3A00206B3B00206B1A002092
:104FE8004AEA030A012F8BF800A013D13823B8FB33
:104FF800F3F203FB12834FF436614A43DBB23421E8
:1050080001FB03238A49CB1893F8302042F0200291
:1050180083F8302087488849884AFEF77FFD864B09
:105028001B781BB1FEF742F8002836D18248844924
:1050380012F0EEFE68B10DF019F870BB804808F068
:1050480089FD50BB01237E487E497B4A0093FEF7C9
:105058003BFD002300937C4A013301931378754884
:1050680002937549754A774B08F008FD012F14D152
:105078003823B8FBF3F203FB12884FF436635A4324
:105088005FFA88F8342303FB08236949CB1893F89F
:10509800312042F0010283F831200134079A09993E
:1050A800E3B205328B4209F101090792FFF4E4AE3D
:1050B800069A013602F5E072022E06927FF4CDAE12
:1050C800624E73786FF3C71373702B7803F0800206
:1050D800D2B2002A00F0DE805D490C78002C40F046
:1050E800D98003F02403042B0BD1FEF747FCFF23E0
:1050F80000934020214601222346019402940CF09B
:10510800D7FC2B8800246FF3C7136FF3820364F373
:10511800451364F3410364F300034E4A64F34923DF
:1051280064F38A2314702B804B4B1A7842F0C00228
:105138001A705A7864F3C3025A70FEF7FFFC4748A6
:105148001FF0E8FA46481FF0E5FA46481FF0E2FA71
:10515800412245482146FBF71DF9444B1A7802F0D5
:10516800DF0264F304121A701A7E02F0DF0264F39D
:1051780004121A7693F8302002F0DF0264F3041266
:1051880083F8302093F8482002F0DF0264F3041219
:1051980083F84820364B1A7802F0DF0264F386124F
:1051A8001A70344B1A7864F345121A709A7F64F3B4
:1051B80045129A7793F83C2064F3451283F83C2013
:1051C80093F85A2064F3451283F85A202A4B1A7828
:1051D80002F0DF0264F386121A70284B5A7864F3DF
:1051E80045125A701A7802F0BF0264F345121A7019
:1051F8001A7D64F345121A75DA7C02F0BF0264F373
:105208004512DA7411E04FF436626243342101FB2F
:1052180003221B49013352189178382B6FF382010E
:105228009170F0D10134022C2CD00023EBE700BFA1
:10523800503D0020FC1C0020E51D0020D81D00204A
:1052480096190020C11C0020961D0020CB190020B3
:1052580060130020681B0020503B0020E61B002044
:105268008E190020BB190020D91900208A3A002085
:105278003F3A00206B3B00201D3A0020E639002011
:10528800583D0020042272480021FBF783F8714B37
:1052980000221A70704C2378002B48D129786F4A65
:1052A80001F00201C9B2D9B16D481188477863F39A
:1052B8004D3163F3C30741F0800147701180CA2064
:1052C80020F070F8C62020F06DF820F0B9F8654A93
:1052D80013780BB90DF042F8FEF7DCF8FEF7DEFDA7
:1052E800614A2B8811786FF341036FF300016FF364
:1052F800000311705D48002140222B80FBF74AF81B
:105308005B481FF007FA5B481FF004FA5A481FF081
:1053180001FA5A481FF002FA04224D480021FBF70F
:1053280039F84C4A00231370554A13706AE02F78F5
:1053380007F00203DBB293B917F001070FD14C480D
:105348001FF0E8F92378F8B23B4113F0010F03D0BE
:10535800FEF730FA0CF080FE0137042FF2D12B78DB
:105368003E4F13F0010F25D0FEF72CFD3B8843F08C
:1053780002033B80FEF7C0FA364B93F80080B8F181
:10538800000F14D1CA2020F00DF8CD2020F00AF823
:105398003B883C4868F300033B80334B1A7842F063
:1053A80001021A701FF0B6F9FEF774F802E0012046
:1053B800FEF704FC2B7803F00202D2B212B3304A93
:1053C80012782AB113F0010F02D10220FEF7F6FB82
:1053D800FEF72AFF2C4927481FF0BAF92549264825
:1053E8001FF0A0F9FEF7C4FB224928481FF09AF9DC
:1053F800274926481FF0A1F9FEF754FB1F481D490D
:105408001FF0B1F9204923481FF08CF915490B7892
:105418000BB9FEF7D5FA737803F08003DBB2002BE3
:1054280040D12B7803F02403042B06D143F6EC205B
:105438000CF0C0FA08B1062032E0FEF71DFD08B1F5
:1054480005202DE00DF074F830B3032028E000BFEC
:10545800AF1900208A1900208C190020841B002015
:10546800503B0020601300208D190020A61B00204F
:10547800493100205F1B0020BB1900209E1B002023
:10548800EE1B00206C1A0020CE1900208E1B002075
:105498001B1A0020B319002001F05AF810B104209B
:1054A800FEF78CFB694B1B781BB173786FF3C7133E
:1054B8007370674A137813B1664B1B78CBB12B789E
:1054C800654E03F04403402B13D10021BF330093F2
:1054D8003F200B460222019102910CF0E9FA338831
:1054E80043F6CE2043F0040333800CF063FA5B4BA1
:1054F800187057495A4E0B789BB1564B197881B999
:105508002A78554B02F04002D2B252B11A8861F3A0
:1055180082021A80337823B943F6CE200CF04AFA77
:1055280030702A78DFF8308102F00400C0B24D4BA9
:1055380000287AD002F02000C0B2484F90B11A7803
:10554800002042F0C0021A70FDF7C4FE3B78002B21
:1055580071D1B8F8002063F3820263F34512A8F80A
:10556800002068E0D20052B219789211D2B241F00C
:10557800C00112F0010F197003D0C9B260F3C7114E
:10558800197012F0020F03D01A786FF386121A708E
:105598001B78344A03F04003DBB24BB9537843F02D
:1055A8000803537023781BB12B8843F400532B80D6
:1055B8000120FDF78FFE43F6CD200CF0FBF9C0B2B9
:1055C8000128307002D1264B02221A703C78002C38
:1055D80031D1FEF7D3F9FF23012200934020214661
:1055E8002346019402940CF063FA2B8843F6CD20ED
:1055F80043F020032B800CF0DDF9184B1A4A187081
:10560800144B14701A780AB1013A1A70197891B9C2
:105618000F4A13787BB1FF230093412002220B46E7
:10562800019102910CF044FA05E01A7842F0C002A8
:105638001A70FDF74FFE0CF02BFF0C481FF098F87E
:105648000B4BB8B91A7860F3820216E08E57002027
:10565800711B0020EF1B0020841B0020681B00200A
:10566800D8190020503B002060130020231A002086
:105678008D1900201A7842F004021A706A784F488F
:1056880012F001011A780CBF61F3410242F00202E4
:105698001A704B491FF067F84A4948481FF04DF8FF
:1056A800464849491FF049F83378012B40F0838078
:1056B8002B8800246FF349236FF38A232B80434BF5
:1056C80041221C7021464248FAF764FE41481FF007
:1056D80021F8FEF733FA3B481FF01CF83A481FF050
:1056E80019F83D4B1A7802F0DF0264F304121A70BD
:1056F8001A7E02F0DF0264F304121A7693F830205F
:1057080002F0DF0264F3041283F8302093F8482093
:1057180002F0DF0264F3041283F848202F4B1A7852
:1057280002F0DF0264F386121A702D4B1A7864F3C4
:1057380045121A709A7F64F345129A7793F83C20C1
:1057480064F3451283F83C2093F85A2064F3451219
:1057580083F85A20234B1A7802F0DF0264F386128A
:105768001A70214B5A7864F345125A701A7802F06D
:10577800BF0264F345121A701A7D64F345121A7554
:10578800DA7C02F0BF0264F34512DA7411E04FF4D8
:1057980036626243342101FB032214490133521853
:1057A8009178382B6FF382019170F0D10134022C7B
:1057B80001D00023EBE70BB0BDE8F08FCE35002019
:1057C8008E1B00208E190020E61B0020D81900200F
:1057D800D9190020BB1900208A3A00203F3A00203E
:1057E8006B3B00201D3A0020E6390020583D002080
:1057F8002DE9FF4104460D460CF074FEA04B1A1922
:1058080092F880709F4A98461278AA2A0AD1A7F17E
:105818004F03DAB20B2A00F2AD819B4A5BB29A4081
:1058280040F1A881994B0C2202FB04335A7A0833C1
:10583800AA42C0F09F81FF2A00F09C81FF229A7043
:10584800934808EBD403214693F888511EF0BDFF16
:105858000646002840F08E8104F007031D41502FB2
:1058680005F0010500F0268114D8462F00F0F280DB
:1058780009D8412F00F09E80452F00F01B812D2F65
:1058880040F0768134E0482F00F0C5804F2F40F07B
:105898006F810EE0542F67D006D8522F00F08A800F
:1058A800532F40F065811CE0A7F15903012B00F24A
:1058B8005F81784821461EF088FF0646002840F0A0
:1058C80059815A2F01D1744802E0592F04D17348E5
:1058D80021461EF064FF54E121466F481EF05FFF29
:1058E800F5E76F4821461EF070FF002800F042815E
:1058F8006C4821461EF069FF8046002840F03A8136
:10590800214668481EF04BFF674821461EF052FFAB
:105918000227012655B1A419142041463A464346A8
:105928000097019602940CF0C3F82AE129463A46FA
:10593800334604F101080A2000970196CDF8088043
:105948000CF0B6F82046FCF713FC414602462B46FD
:1059580013200095FCF7D2FE384629462A463346DE
:105968000095FCF7CBFE0CE14E4821461EF02DFFBA
:105978000746002840F005810126022231463346B9
:10598800A5193E200092019602950CF091F8204648
:10599800FCF7EEFB294602463B4614200097FCF72D
:1059A800ADFE21463F481EF0FAFE21463E481EF055
:1059B80001FFE6E03A4821461EF007FF06460028A8
:1059C80000F0DF80374821461EF0FFFE064628B962
:1059D8002046FDF77DFD002840F0D380002D40F0E3
:1059E8008E802046FEF722FA002840F0C580204627
:1059F800FEF70AFC2D4BDB7803F02003DBB20BB972
:105A08002B4B1855412F00F08880522F40F0B08062
:105A18002046012183E0234821461EF0D6FE28B9FE
:105A28002046FDF755FD002840F0A480002D66D1E2
:105A38002046FEF7FBF9002840F09E801B4BDB78E0
:105A480003F02003DBB2002B67D1194B032283F844
:105A5800402062E0134821461EF0B7FE064628B9EA
:105A68002046FDF735FD002840F08B802046FEF7E4
:105A7800DDF900287ED1002D41D1204603214EE0DA
:105A8800202C0020671B002000003080E02D002023
:105A9800CE19002078290020982800200829002005
:105AA8005F1B00208E1B0020961B0020DC39002085
:105AB800D9190020354821461EF087FE06460028E1
:105AC8005FD02046FDF7D0FE20B1214630481EF0B9
:105AD80066FE4FE0502F28D12E4B1B782BBB20465B
:105AE800FDF7AEFE08BB2C4821461EF06EFE0646AA
:105AF80020B92046FDF7ECFC002842D115B120461C
:105B080002210CE02046FEF77FFB244BDB7803F0F4
:105B18002003DBB20BB9224B185520460021FEF7B3
:105B28007BFA061E18BF01262BE02046FDF788FEEB
:105B38000546F8B91B4821461EF047FE0646D8B967
:105B48002046FDF7C5FC0746D8B9164821461EF081
:105B580026FE154A135D8BB910494E7806F02006CB
:105B6800F6B26EB908EB040393F80031135508E058
:105B7800012606E0002604E02E4602E03E4600E04C
:105B88001E46304604B0BDE8F08100BF5F1B002010
:105B98006C1A0020EE1B00208E1B0020DC39002030
:105BA800D9190020BB190020A61B0020032210B51C
:105BB80005490648FAF7C4FE054806490222BDE829
:105BC8001040FAF7BDBE00BFF625002004020020F1
:105BD80009020020F425002070B5844C237813F0C6
:105BE800010F0AD00CF04AFA38B10020804902F0BF
:105BF8008DFE804B8048197849E0804D2B78002B2A
:105C08004AD00CF041FA002846D07D4B1B7873B976
:105C18007C4B5B7813F0010F09D00CF027FA30B9F0
:105C2800237803F02403042B01D10330BEE0764C23
:105C3800207870B10020754902F068FE21780122B1
:105C4800734802F089FE00201021621C07F0C8FA90
:105C580002E0704902F05AFE6F4C684807F014FBE6
:105C68002378002B00F018810CF008FA002800F0C7
:105C780013816A496A481022FAF762FE68485B2174
:105C8800FAF706FC002800F007812178013083220A
:105C9800BDE8704002F060BE624C237803F0050353
:105CA800012B5DD10020604902F030FE2021102236
:105CB8005E48FAF76FFB601D5D490322FAF7EAFDBB
:105CC80040BBE01C5B490222FAF7E4FD30B95A48B0
:105CD800FAF7B0FD5849024654480BE0E01C574912
:105CE8000222FAF7D7FD40B95548FAF7A3FD5449FF
:105CF80002464E48FAF724FE0EE0E01C5149022203
:105D0800FAF7C8FD30B95048FAF794FD4E490246F3
:105D18004648EFE7FFF74AFF6278303AD3B2092BDB
:105D280000F2BA803F4B9B78303BDBB2092B00F284
:105D3800B3800A2101FB0231C9B2002900F0AC800E
:105D4800374BFF220C291A7740F2A68010295A7780
:105D580040F2A28013299A7740F29E80DA7770BDCC
:105D68003A4C237803F00203DBB213B10020384920
:105D78008EE0234E3378EBB9224B5B7813F0010F9A
:105D880018D00CF073F9A8B932481EF0F1FC60B1D4
:105D98002268314B02EA03033BB918F0D7FD20B95A
:105DA800E37803F04003DBB223B10020BDE8704084
:105DB8000AF0E2B9337863B90CF058F948B1274BC7
:105DC8001B7803F00603042B03D02B780BB90120B2
:105DD800ECE7FEF751F810B10020214958E0214BBB
:105DE8001D78002D42D0204952E000BF841B0020BE
:105DF800E9F702088A190020000200208C19002007
:105E0800941D0020551E0020DE1C0020FCCC02083A
:105E180005020020BACC0208EE1B0020DBCC0208E9
:105E2800F4010020F125002003D20208040200201A
:105E3800545403085854030866D202085B540308F4
:105E480045D202085E54030824D20208DC39002037
:105E58005AE10208231A00203000000F8D19002093
:105E68008CDF0208651300201DCD02080B4802F0E4
:105E7800FCFC0A4802F0F0FC094802F0EDFC1DF0B9
:105E880023F9E37803F02003DBB22BB10549284658
:105E9800BDE8704002F03ABD70BD00BFE81D0020AB
:105EA800081D002015CC0208054B1B78D8019B0162
:105EB8005BB2DB1140B243EAE070C0B2704700BF8A
:105EC800841B002070B50E4686B0410001220546AD
:105ED80001F5E97105A80BF07EFD0021012E8DF872
:105EE80015104FF0FF0205F1010305D10092019151
:105EF80002930920FB3A04E00092019102931E20CC
:105F080004220B460BF0D4FD05A83D49FAF746FBE1
:105F180050B105A83B49FAF741FB28B105A83A4911
:105F2800FAF73CFB002867D105A83749FAF736FB92
:105F3800364B0446F8B95A78214642F010025A7096
:105F4800FF23022200930190FE3B02903D200BF0BC
:105F5800AFFD4D200CF076F9691C01222346122072
:105F68000094FCF7CBFB1220214622460123009423
:105F7800FCF7C4FB03E05A786FF304125A7000244C
:105F8800E0B2552115F0BAFE38B12846214616F080
:105F980056F810B1204616F041F80134082CEFD11C
:105FA8003EBB1B481B491C4AFDF7B8FD19481B4955
:105FB80011F02EFF68B10CF059F850B9174807F0E6
:105FC800C9FD30B9012315481549124A0093FDF758
:105FD8007BFD144B0F491D7000230093053301937B
:105FE800114B0D4A1B780A4802930D4B07F046FDEA
:105FF80002E00E4B00221A7005A806B070BD00BF63
:10600800E554030861540308F1560308503B002087
:10601800FC1C0020E51D0020D81D0020961900203A
:10602800C11C0020E33B0020961D0020AE19002073
:1060380007B54100012201A801F5E9710BF0CBFC7D
:10604800002301A804498DF80530FAF7A7FAD0F122
:10605800010038BF00200EBDE554030807B5410014
:10606800012201A801F5E9710BF0B5FC002301A894
:1060780004498DF80530FAF791FAD0F1010038BFDC
:1060880000200EBDAE56030870B5154B04461B180C
:1060980093F88050B1B1134821461EF096FB88B999
:1060A800114821461EF07BFBA5F15903DBB2012BF9
:1060B8000CD94F2D0AD0542D08D021460B481EF07C
:1060C8006EFB07E0084821461EF074FB074821468E
:1060D8001EF070FB04480649BDE870401EF022BB64
:1060E800202C0020CE190020231A0020C3190020DC
:1060F8009E1B0020024B1878C0F38000704700BF39
:106108008D190020024B1A8860F308221A80704704
:10611800841B0020034B5878C00140B2C011C0B2A4
:10612800704700BF841B0020014B1878704700BFE0
:106138008C19002030B5457800230021C2189170D1
:1061480055FA03F111F0010F08D0064959188C7C53
:10615800017804EA0101A14208BF91700133042BC0
:10616800EBD130BDDE1C002046F6A93104220BF02D
:1061780032BC000070B5104C0546112220460021A3
:10618800FAF708F9002004F8010C2A78103414F8FA
:10619800011FC3B291420BD152B10849013301F832
:1061A800013B112246F6F953BDE8704002F0FABAF5
:1061B80001300428EBD170BDDF1C0020DE1C00205C
:1061C8001FB520B1134B1A8842F480521A80124B23
:1061D80000245A78214642F010025A70FF23022206
:1061E80000933D20FE3B019402940BF061FC4D208E
:1061F8000CF028F820210122234612200094FCF7F5
:106208007DFA12202146224601230094FCF776FAF3
:106218001FBD00BF841B0020503B00202DE9F34127
:106228002D4C0722E37849F6B44702FB003349F6C0
:10623800D540DBB218180BF0BDFB257964795FFAFD
:1062480080F8002648FA06F313F0010F3AD03946D1
:10625800042201A80BF0BFFB9DF804009DF805304F
:106268009DF806109DF8072000282BD0002929D07A
:10627800002B27D0002A25D0934204D19C4221D15B
:1062880085421FD30FE09A4210D99C421AD39442F8
:1062980018D89C4201D994421AD39C4201D1854214
:1062A80016D294420ED18D420CD811E09C4201D1F5
:1062B80085420DD2944201D18D4209D99C4207D81A
:1062C800944205D301360437082EBBD1002000E0E4
:1062D8000120BDE8FC8100BFFC54002010B5044635
:1062E80049F60D5000EBD4000BF064FB04F00704F2
:1062F800C0B2204100F0010010BD70B5C30849F6D6
:106308000D555D19044628460E460BF053FB04F064
:106318000704C0B2012126B9A14040EA0101C9B26F
:1063280002E0A14020EA01012846BDE870400BF0D8
:1063380037BB0000F0B57E4B8DB0DD78042200EB52
:10634800C505EDB2E90001F5084104A801F59E7103
:106358000BF041FB774B784E1A78002304A9C95CEF
:10636800312905D13039994041EA0202D2B205E01B
:10637800302903D12F39994022EA01020133042B35
:10638800ECD132706C486D496D4AFDF7C7FB6B4B19
:106398001B7813B96A4B1B78F3B16848694911F047
:1063A80037FD68B10BF062FE50B9664807F0D2FBC2
:1063B80030B9012363486449604A0093FDF784FBC0
:1063C8000023009302330193FD3302935A485B493B
:1063D8005B4A5D4B07F052FB05EB0511002401F504
:1063E8000A41347004A8FC3108220BF0F4FA26465E
:1063F800E0B2542115F082FC002838D004AB1B5DB4
:10640800312B03D1204615F00FFD38B104AB1B5DCD
:10641800302B2CD1204615F007FD40B34EB9FF2391
:1064280000933420314604223346019602960BF03D
:106438003FFB04AE305D2146303815F003FD335D77
:106448000126312B4FF0030306D10093A3191BB289
:1064580001960293352005E00093631C1BB2019658
:1064680002933620002104220B460BF021FB013455
:10647800082CBDD1A90101F50E4104A8B431202290
:106488000BF0A9FA083C04AD274615F8013BE6B223
:106498000134302B03D13046FFF720FF38B115F80F
:1064A800013C312B2CD13046FFF718FF40B34FB9D0
:1064B800FF2300933420394604223B460197029774
:1064C8000BF0F6FA15F8011C30463039C9B2FFF75F
:1064D80014FF15F8013C0021302B4FF0FF0305D1C4
:1064E800009323B201910293372004E0009323B272
:1064F80001910293382004220B460BF0D9FA0127A8
:10650800202CC2D1114D6B7803F00403DBB263B1C8
:10651800203C2046FFF7E2FE38B90134E4B2202CD3
:10652800F7D16B7860F382036B700DB0F0BD00BFDC
:10653800FC5400208C190020FC1C0020E51D0020C4
:10654800D81D002096190020C11C0020503B0020B7
:10655800014B1878704700BF651300202DE9F04FF4
:106568004E4B00221A704E4A85B01678002E40F025
:1065780091804C4B4FF4B468DA78997808FB02F2B2
:106588004FF03C0808FB01285A78474F90441FFAFF
:1065980088F8BA466CE03AF815303C24DAB254432D
:1065A80004EB13244C44A4B2042CEEB207D842F2F4
:1065B8005A73984503D904F51C546034A4B2444571
:1065C80011D949F6D4400BF0F5F9C8EB040383421E
:1065D80009DC364B1A787B1993F83830934302D08C
:1065E8002E4901230B702F4AD378B34232D142F29D
:1065F8006073B4FBF3F203FB12439BB2434523D110
:106608002B4B9B7813F0090F44D12A4B5B7803F08E
:106618008003DBB2002B3DD1274B5B7803F00203EC
:10662800DBB2002B36D1254B1A781BEA020F11D1A9
:106638000199009841EA02021A70FFF7EFFD48B984
:106648000098FFF777FE05E01C4B02991A7801EADB
:1066580002021A70013509F5B469072D1FFA89F984
:1066680099D1039E07370136042E0AF10E0A11D07C
:106678004FF0010B0BFA06FB5FFA8BF301936FEAFD
:106688000B03F2B2DBB24FF00009009202934D46C1
:10669800039680E705B0BDE8F08F00BF65130020C2
:1066A800F51B0020FC540020F61B00208C1900204C
:1066B800DC3900205F3B0020C6330020F41B00209B
:1066C80073B50C4601EBC001C9B2C90001F5084118
:1066D8000546042201A801F59E710BF07CF9104BC8
:1066E800002003EBC402121B521982F8380001AAD9
:1066F800125C312A0AD10121814003EBC402121B2A
:10670800521992F83860314382F838100130042861
:10671800EDD101A9312230231EF05FF8C0B27CBD53
:10672800F61B002000B501EBC001C9B2890189B090
:1067380001F50E41B431202268460BF04CF92020B7
:106748006946312230231EF048F8C0B209B000BDB6
:1067580007B501EBC001C9B201EB011101F50A410E
:10676800FC31082268460BF036F9082069463122C8
:1067780030231EF032F8C0B20EBD00002DE9F843F8
:10678800002634462BE021462846FFF799FF21468C
:1067980081462846FFF7C6FF214640EA09092846F0
:1067A800FFF7D6FF5FFA89F949EA000010F0FF0FFA
:1067B80005D04046394602220BF00DF903E04FF0B0
:1067C800FF33A8F800300135EDB20237072D08F184
:1067D8000208D8D10134E4B20E3E042C07D0054B90
:1067E800C6F50847C6EB0308CC370025CBE7BDE85C
:1067F800F88300BFF61B002010B51FF055F84FF4C2
:1068080080301FF071F81FF089F90128044628D15B
:1068180010201EF06BFF02201EF05CFF00201FF00E
:10682800A3F800201FF0B4F84FF480601FF0A6F81A
:106838004FF440401FF0B6F84FF480304FF4E011A9
:106848001FF06EF820461FF077F839201FF052F934
:106858000028FAD002201FF075F81FF07DF80828EC
:10686800FBD17C2001211FF00FF946F60120012100
:106878001FF00AF90C4801211FF012F90B480121F9
:106888001FF00EF9042001211FF00AF97E201FF0E5
:1068980031F938B11FF058F9054B04211A7861F322
:1068A80044021A7010BD00BF0340060020080818F3
:1068B8007157002010B50C46014620B110220C4833
:1068C800FAF73EF804E00A4820211022F9F762FDA1
:1068D80034B1084821461022BDE81040FAF730B814
:1068E800044820211022BDE81040F9F753BD00BF2D
:1068F800F40100200402002010B5FF2B1446029A70
:1069080003D0421802F8013C08E06FF07F439A4236
:1069180004D01314437013128370C2701BF0C6FAAC
:1069280002E07F201FF02CFC1BF0ACFA0028F8D105
:10693800ACB10B4890F82010163001F00F011BF095
:10694800B5FA02E07F201FF01BFC1BF09BFA002821
:10695800F8D1044B93F8693013F0010FE9D110BD59
:10696800900C00208C56002010B50A4B002203EB37
:106978008003013B1046084951184C7813F8011F51
:106988008C4205D10130C0B20C320428F3D1FB305F
:1069980010BD00BF12620208E02D002070B50D4C3A
:1069A80005460E464FF4007200212046F9F7F2FC26
:1069B8002A46314604F50070F9F744FC642024F8AF
:1069C800035C1CF053FE0023A4F82D33024B642211
:1069D8001A6070BDF5570020FC25002010B5054C45
:1069E800002120464FF40072F9F7D4FC0023A4F8E4
:1069F8002D3310BDF5570020164B2DE9F0415D8968
:106A080007462846FBF78CF81349FBF795F9134B13
:106A1800134E1860D723B5FBF3F5EDB28222294651
:106A28000446F01901F098FF2846FBF77DF8014667
:106A38002046FAF7C3FF0B49FBF7CAF8FBF78EFAB3
:106A48000337BE19C1B281223046BDE8F04101F0DA
:106A580083BF00BF1C310020000057434C1C00209E
:106A6800F40100200000204170B54B4D2868FAF76A
:106A780063FC45A3D3E90023FAF7FEFAFAF74AFFC5
:106A8800FAF75AFC42A3D3E90023FAF7A9FC3EA37C
:106A9800D3E90023FAF7CEFDFAF73CFFFAF74CFCEE
:106AA800FAF756FAFAF736FF3C4906462860FBF72C
:106AB80037FA20B13046FBF751FAC4B25EE03046EF
:106AC8003649FBF741FA50B130463549FBF728FA09
:106AD80028B13046FBF742FAC0B2441C4EE03046BB
:106AE8002F49FBF731FA50B130462E49FBF718FA17
:106AF80028B13046FBF732FAC0B2841C3EE030467B
:106B08002849FBF721FA50B130462749FBF708FA24
:106B180028B13046FBF722FAC0B2C41C2EE030463A
:106B28002149FBF711FA50B130462049FBF7F8F933
:106B380028B13046FBF712FAC0B2041D1EE03046F9
:106B48001A49FBF701FA50B130461949FBF7E8F941
:106B580028B13046FBF702FAC0B2441D0EE03046B9
:106B68001349FBF7F1F948B130461249FBF7D8F958
:106B780020B13046FBF7F2F9C0B2841D0A20214645
:106B8800BDE870400AF00CBF736891ED7CFF7F4050
:106B98000000000080842E41501C0020000010419D
:106BA8000000F0410000484200008E420000B84258
:106BB8000000E0420000F2422DE9F04F9DB01BF0CA
:106BC8000BF909201CF0EEFE1CF0D4FC4FF46140D8
:106BD8001CF024FF09201CF0A1FF0022A1484FF45B
:106BE80080411EF0E8FDA04800211FF0B1F99F493F
:106BF80004224B78DFF898E26FF300034B709C4B4C
:106C08009C4C1A705A709A70DA709B4B033A1A703F
:106C18009A4B00201F328EF8000020705A710590A0
:106C28000546069006467F201FF0AAFA23780E2B09
:106C380001F2B681DFE813F00F004F009500E00085
:106C48007902DE0330048504EA06DC07EF075808FA
:106C5800B108D00882098A4E8A48317801F00F01BC
:106C6800013149014118FFF725FE337813F00F036E
:106C780008D1854A92F80123012A41F09181834A7B
:106C8800138024E0012B03D17F4B93F819330BE0D9
:106C9800022B04D17C4B93F80D33032B05E0032B17
:106CA80006D1794B93F80D33012B41F079810EE031
:106CB800774901220A7077484FF400711EF07BFD76
:106CC800754BC8221A6033786FF30303BFE3337838
:106CD8005A1C01F05FB8704B1A6822B96D484FF41E
:106CE80000711EF068FDDFF898816C4898F8001074
:106CF80001F00F01013149014118FFF7DBFD36B101
:106D080098F800305A1C62F3030388F800305F4B90
:106D180000221A8098F8001001F00F02022A03D10D
:106D28001A7842F010020AE0042A03D11A7842F0D5
:106D3800040204E0052A05D11A7842F040021A70CC
:106D480001F02EB9062A04D14D4B6FF303011970D7
:106D58007EE301F00F01012212FA01F1198001F01E
:106D68001FB9474E4E48317801F00F0101314901F2
:106D78004118FFF79FFD96F8008008F00F08B8F15A
:106D8800070F27DC18F0010F464B02D0002058806F
:106D980002E04FF0FF3159804FEA6809062209F1F5
:106DA800010902FB09394FF0FF32A9F802204046D9
:106DB800FFF7DAFDFF2806D03B4B03EB40005823D2
:106DC800437401F0EDB80023A9F8023008F1010876
:106DD80001F08AB80021102213A8F9F7DBFA0FA8EE
:106DE80000211022F9F7D6FA23780133237033787B
:106DF8006FF3030301F07BB8DFF884A09AF80080F2
:106E080018F00F0840F03F81284E337803F0400314
:106E1800DBB2F3B926486FF07F43817A01220093F1
:106E280001F00F01FF23FFF767FD224B93F869205C
:106E380012F0400F08D093F86C3013F0040F03D011
:106E4800337843F0400333707378142262F3C70336
:106E58007370737813F0F80F30D0174800F12001E1
:106E6800A7E300BF00180140002C01403631002084
:106E7800202C0020561C0020631300208A3A002092
:106E8800551C002032620208E02D0020503B0020F3
:106E98002C260020000C0140FC250020D2620208AC
:106EA800B26302080A3B0020F4010020C739002021
:106EB800900C00208C560020D2640208BC4B1B7832
:106EC80003F04003DBB2002B00F0D980DFF8048325
:106ED800DFF8049398F8003013F00C0B30D1B54E5E
:106EE8006FF07F4396F82B1006F12100009301F014
:106EF8000F0101220523FFF7FFFC96F84C104FF411
:106F0800860A06F1420001F00F010122FF23CDF8A5
:106F180000A0FFF7F1FC96F84110FF2306F13700B7
:106F280001F00F015A46CDF800A0FFF7E5FC042355
:106F380089F8003098F8003043F0080301F02EB8C3
:106F480003F00803DBB2002B39D099F800A0BAF19E
:106F5800000F03D0984800F1400138E0954E6FF0DB
:106F68007F4B717D06F10B0001F00F010122FF2319
:106F7800CDF800B0FFF7C0FC96F82B1006F1210001
:106F880001F00F0101220723CDF800B0FFF7B4FC90
:106F980096F836104FF48603009306F12C00FF2371
:106FA80001F00F015246FFF7A7FC98F800306AF38A
:106FB800C303DBB243F0040388F800305AE099F8C1
:106FC80000C0BCF1000F08D07B4800F16001FFF75A
:106FD80071FC99F80020303208E2764E6FF07F405D
:106FE800717DFF23009001F00F0106F10B000122D3
:106FF800CDF80CC0FFF780FC9AF80030DFF8C4B178
:1070080003F0100A5FFA8AFADDF80CC0BAF1000F33
:107018000CD098F800206CF3820288F800205A1CE3
:1070280062F303038BF8003000F0BABF96F82B1018
:107038006FF07F42009206F1210001F00F0101225A
:107048000C23FFF759FC96F836104FF4860300938B
:107058005246FF2306F12C0001F00F01FFF74CFC0C
:107068009BF8003083F01002C2F3001262F304139D
:107078008BF80030042389F8003000F091BF4E48A7
:1070880000F1800195E2B8F1010F3CD14A4800F1C6
:10709800A001FFF70FFC002E00F082879AF800305D
:1070A800444E5A1C62F303038AF8003096F82B10FA
:1070B8006FF07F4906F1210042460F2301F00F01CE
:1070C800CDF80090FFF718FC96F82B1006F1210078
:1070D80042460E2301F00F01CDF80090FFF70CFC9B
:1070E80096F82B1006F12100424601F00F010F23FC
:1070F800CDF80090FFF700FC3048802142461EF092
:107108005AFB00F04DBF2C4800F1C001FFF7D2FB3D
:10711800002E00F045872A4B96221A609AF8003014
:107128006FF303038AF8003092E1264E317811F0AC
:107138000F0A16D1244800F12001FFF7BBFB204BB2
:107148001B68002B40F02C8713A8F9F773FB40222B
:107158001346014613A801F023FA3378012200F000
:1071680019BEBAF1010F39D112486FF07F4390F878
:10717800201000220093163001F00F01FF23FFF7C3
:10718800BBFB01F077FA002800F00A873378022267
:1071980062F3030333700D4B1A7842F080021A70C1
:1071A8000B4B5A7842F002025A7000F0F9BE00BF49
:1071B800C7390020900C0020D2640208001001405A
:1071C800FC250020551C0020B2650208CC3900209F
:1071D800723C0020105E0020975F002001F00F0134
:1071E80001F10E0303F00F03012B44D89B4849011A
:1071F8004118FFF75FFB9A486FF07F4390F8201023
:1072080000221630009301F00F01FF23FFF774FBF3
:107218001BF0F8FF337803F00F03022B13D117F09C
:1072280061FB002800F0BC868E4B1A7842F04002C1
:107238006FF304121A705A786FF345125A70337844
:10724800032200F0A7BD17F037FB78B117F0D6FB83
:1072580017F08EFA844B00201A7858816FF3C71202
:107268001A703378042262F3030333707F4B1A7861
:107278006FF3000263E5BAF1040F4DD1DFF8DC913A
:107288004901DFF8108249444846FFF713FB98F894
:107298000010774B01F00402D2B27AB941F0040130
:1072A8006F4883F800A088F8001090F836104FF463
:1072B800860300932C3001F00F01EEE293F800A052
:1072C800BAF1000F40F06C8665486FF07F45417D4C
:1072D80001220B3001F00F01FF230095FFF70CFB93
:1072E80064480122817AFF2301F00F010095FFF71E
:1072F80003FB98F8003005226AF3820388F800300F
:107308003378484662F30303337009F1A001FFF7AD
:10731800D1FA554600F044BEDFF84481FF2398F8BF
:10732800201000226FF07F4908F1160001F00F01CC
:10733800CDF80090FFF7E0FA2BB2072B18D133787D
:1073480008F121006FF3030333702378012201331E
:10735800237098F82B100E2301F00F01CDF8009040
:10736800FFF7CAFA4448802100221EF024FA0025BB
:10737800424E96F86B3013F0040F00F0118698F81F
:1073880057106FF07F43002200933D48FF2301F020
:107398000F01FFF7B1FA96F86B303A4A03F00F0382
:1073A800012B137003D1002D08BF01250CE0022B1F
:1073B80004D12BB2012B08BF032505E0032B03D111
:1073C8002BB2032B08BF0725ABB213F0010F02D075
:1073D8002D4A3121517713F0020F02D02A4A322167
:1073E800917713F0040F00F0DB853322264BDA7710
:1073F80000F0D6BD1948254E00F1C001FFF75AFA32
:1074080096F80090DFF85C8019F00F090CD117F09E
:10741800C9F898F8003069F3000388F80030337829
:107428005A1C62F30303337017F04EF998F80030D2
:1074380013F0010F00F0B4850022154880211EF0DA
:10744800BAF90A4B00225A70337862F30303337097
:1074580023780133237000F0A3BD00BFB265020892
:10746800900C0020723C0020CC390020EA3B002020
:10747800975F002001000020001001408C5600207A
:10748800DD0C0020C6390020F4010020551C002026
:1074980000180140105E00208648874E00F1E00188
:1074A800FFF708FA0FA8F9F7C5F90FA902468348AC
:1074B800F9F746FA00218248B18090F8C5106FF0BC
:1074C8007F4300220093BB30FF2301F00F01FFF739
:1074D80013FA7C4A92F86B1092F86C30327843EACF
:1074E800012312F0010FB38010D0A3F1EB0292B286
:1074F8000A2A04D9A3F5E6739BB2282B02D8F3888D
:107508000133F38033786FF3000333707378002B03
:1075180040F04685684AD2887AB16B4A1BA8117830
:1075280063F30301117022788DF86F3001322270F5
:1075380028228DF86C201EF05DF90022F28000F000
:107548002FBD624EDFF8ACA1337803F004085FFA70
:1075580088F8B8F1000F15D109A841461522F8F7A7
:1075680019FF5B4BCAF800801B684546CDF82730E9
:107578003368474643F004033360564BA3F8368319
:1075880000F00EBD03F08003DBB2002B67D1DAF800
:107598000010002940F004854F48FFF78BF94F4849
:1075A8004FF480511EF0FDF8012806D04A4800F13A
:1075B800A001FFF77FF900F0F3BC4649B1F8362384
:1075C800002A43D009314648013AF9F7B9F9444B42
:1075D80003F1100113F8012B0D2A01D00A2A02D158
:1075E800202203F8012C8B42F4D13E4B4FF03C088B
:1075F80008FB073808F11E084046F9F71BF9414611
:1076080002463948F9F746F9D8B9022F03D1336849
:1076180043F0100304E0032F03D1336843F0400321
:107628003360327853005BB203EAC263DB17326817
:10763800DBB263F3C71232601BB1FFF7CFF900F07A
:10764800AFBC0137FFB2042F08BF0227254B3C26E9
:1076580006FB07363046F9F7EDF8314626E0DAF84A
:107668000080B8F1000F40F09B84737803F020028B
:10767800D2B2002A40D11D4B09A81A889B781C4910
:107688008DF82630ADF82420F8F7DEFE114B5B7A32
:10769800302B07D1FFF7A2F9336843F40053336066
:1076A80000F07EBC09A8F9F7C5F809A9FFF776F933
:1076B80000F076BCB2650208EA3B00200802002010
:1076C800900C00208C560020551C0020002600201D
:1076D80063540308EC570020B26602080008014012
:1076E800040200200C000020F5570020685403080D
:1076F8006C540308FC25002003F04003DBB2002B88
:1077080040F08980B14800F16001FFF7D3F8B04834
:10771800F9F790F88046AE49AE484246F9F7BAF80C
:10772800002873D1AC4B43445B7A302B6ED1FFF702
:1077380055F93368DFF8D09243F48043336099F801
:107748002B106FF07F43009309F12100082301F00B
:107758000F010122FFF7D0F86423CAF800307F2018
:107768001EF00EFDDAF80030002BF8D1984699F893
:107778008E10D633994E89F886304B3B6FF07F4A8E
:1077880089F88730964801F00F0142467433CDF8E6
:1077980000A0FFF7B1F896F8B91106F5D6700330D6
:1077A80001F00F014246FF23CDF800A0FFF7A4F82F
:1077B80096F8C41106F5DD7001F00F014246FF236B
:1077C800CDF800A0FFF798F896F8CF1106F5E2700B
:1077D800013001F00F014246FF23CDF800A0FFF76A
:1077E8008BF896F8DA1106F5E87001F00F014246B9
:1077F800FF23CDF800A0FFF77FF899F89910794892
:10780800CDF800A001F00F01424646E07648F9F7AE
:1078180011F875494AE796F802B0DFF8EC910BF0D9
:10782800020B5FFA8BFBBBF1000F3AD199F82010DD
:10783800FF236FF07F4809F1160001F00F015A4647
:10784800CDF80080FFF758F8684B93F86B3003F0D9
:107858000803DBB2002B00F0A38399F82B10012258
:1078680009F1210001F00F010323CDF80080FFF793
:1078780043F83368554843F4003300F1800133601E
:10788800FFF718F855485A4690F8E51100F5EC70DE
:10789800CDF80080033001F00F01FF23FFF72CF82B
:1078A8007EE3CAF8008099F820106FF07F430093B8
:1078B8004246FF2309F1160001F00F01FFF71CF8FB
:1078C8002AB241F211139A421DD1434B5B7A302BF5
:1078D80013D1FFF783F83368454668F3514368F3DB
:1078E8008E3368F34D333360414B1A7868F30302E3
:1078F8001A7023780133237052E33E48F8F79AFF51
:107908003C49FFF74BF8394E96F86B3013F0040FEB
:1079180000F0468325B9384820211022F8F73AFDAF
:107928007F201EF02DFC99F857106FF07F4300223E
:1079380000933248FF2301F00F01FEF7DDFF96F8B0
:107948006B202F4B02F00F020D2A1A7005D125B9B2
:107958002C4A412191754FF480551A78062A08D18E
:107968002AB2B2F5805F04D1264A3621D1754FF488
:1079780088551A78082A08D12AB2B2F5885F04D146
:10798800204A3821117641F210151B780B2B09D1AA
:107998002AB241F210139A4204D11A4B2A225A767B
:1079A80041F211150D486FF07F4390F8F011002255
:1079B800009300F5F370FF2301F00F01FEF79CFF21
:1079C80096F86B3013F0010FAAD0E9E2B26602080C
:1079D8001A010020F5570020EC5700200100002074
:1079E800140D00201F0D0020FC0000208C560020E4
:1079F800551C00203801002004020020DD0C002066
:107A0800C6390020F4010020900C0020A34B1A78FE
:107A180042B300221A700F20FAF716FB06460A2016
:107A2800FAF712FB9E4B9F4958814A7812F0010FD2
:107A380018D06436301A58829B4B1A78642A01D1C0
:107A48009B321A701B78984EFF2B0BD00A21B3FB80
:107A5800F1F1964B1931198095481EF079FA33786F
:107A680001333370DFF8648298F8003013F00F06A2
:107A780012D18E4B19228B481A804378192143F072
:107A8800010343708A481EF063FA8A4800F1200116
:107A9800FEF710FF04967CE2012E68D1804B5A8ACB
:107AA800A2F1690189B2112908D8049911F0010FCE
:107AB80004D141F00101C9B204910592049A12F06F
:107AC800020F0DD15B897C4A1380A3F5C263023B88
:107AD8009BB2D72B04D8049840F00203DBB204937E
:107AE8001B20FEF789FF0599744B0AB2632A05DD4E
:107AF800642192FBF1F230321A7401E0092A0CDD9C
:107B0800059A11B2642291FBF2F002FB10120A20CE
:107B180012B292FBF0F230325A74059802B2642025
:107B280092FBF0F100FB11210A2209B291FBF2F05D
:107B380002FB101230329A745B4B1B78FF2B08D172
:107B480058495B484B786FF300034B7000211EF0D7
:107B5800FFF9049A032A40F023825248002143780F
:107B68006FF30003437052481EF0F2F911E2022E3F
:107B780003D1534BC8221A600BE2032E16D1504B87
:107B88001B68002B40F00C824A4800F14001FEF7C8
:107B980091FE1B20FEF730FF414B5B89A3F51E6366
:107BA8000F3B9BB2542B00F2FB81F2E1042E0CD167
:107BB8003B4B98890FF0DEFC002840F0F1813D48EE
:107BC80000F16001FEF776FEE3E1052E07D1344BA4
:107BD80098890FF0CFFC032840F0E281D9E1062E06
:107BE80040F0D78122786FF3030301322270D5E188
:107BF800344800F12001FEF75DFE334B1B78002B63
:107C080000F0CE81237801332370304B1A786FF35C
:107C18000302FFF794B82D4EDFF8A480337813F0F1
:107C28000F021AD12A4800F12001FEF743FE294825
:107C3800F8F700FE274902462748F8F703FB2548CE
:107C4800F8F7F8FD254BA3F8160233785A1C62F3AF
:107C5800030333701BF08CFF91E0012A16D1D8F88A
:107C68000030002B40F09C811BF0AEFF012840F053
:107C780097811B48F8F7DEFD194902461948F8F7BD
:107C880009FE002840F08C8111486FE0D8F80020E8
:107C9800002A40F085810B217BE000BF661300209D
:107CA8001C31002036310020641C00208C0C002080
:107CB800002C014072670208581C0020F4010020C3
:107CC800FC250020F2670208541C0020551C0020E7
:107CD8003268020874010020B4370020905B00204D
:107CE80092010020915B0020874E337813F00F0833
:107CF8000CD186484146FEF7DDFD33785A1C62F305
:107D080003033370824BA3F8028049E1B8F1010FF5
:107D180018D1804804211DF044FD002800F040815E
:107D28007A4800F12001FEF7C5FD33784FF0FF31A6
:107D38005A1C62F303033370774B64221A60744B46
:107D480059802DE1B8F1020FDFF8CC811BD1D8F8AA
:107D58000030002B40F024816E4804211DF021FDE5
:107D6800002840F01D816A4B5880684800F14001A6
:107D7800FEF7A0FD33785A1C62F3030333706423C3
:107D8800C8F800300CE1D8F80020002A40F008813B
:107D98000C21217062F30303A9E0604910234FF41A
:107DA8000052CB700D3B8B700A805D481DF0AAFC19
:107DB8000A2200215B48F8F7EDFA80201DF006FC46
:107DC800237801332370504B1A786FF303021A702B
:107DD800514BC8221A60E3E05348DFF848A100F18C
:107DE8002001FEF767FD9AF80030002B00F0D880DC
:107DF8004E48DAF80020444E0260BAF80420828027
:107E08009AF806208271317811F00F0159D1DFF804
:107E18000881D8F80010002940F0C2809AF80410B0
:107E2800A2F5A6524FF0640B103A0BFB01229AF808
:107E380005004FF00A0909FB00200393F9F770FECB
:107E48003B49F9F779FF02469AF80200039BA0F52F
:107E5800A65010380BFB030B9AF80100354B09FBB1
:107E680000B018600392F9F75BFE039A01461046CA
:107E7800F9F7A6FD304B1860F9F75EFA1EA3D3E9AF
:107E8800002382468B46F9F731FD002800F08880F0
:107E9800504659461AA3D3E90023F9F71DFD0028D7
:107EA8007ED0FEF7E1FD337848465A1C62F303039F
:107EB8003370C823C8F8003009F07CFDC0B20790C1
:107EC8006EE001296CD10D300799832200F044FD42
:107ED800114BD3F80080B8F1000F61D140461DF076
:107EE80075FB237801332370337868F30303337009
:107EF80056E000BFAFF30080736891ED7CFF7F40D0
:107F08000AD7A3703D008040551C002092680208E3
:107F18000A3B0020000C0140FC25002032310020E3
:107F2800001001406C1C0020F268020804020020C6
:107F380000007A44681C0020501C00208448854EAC
:107F480000F12001FEF7B6FCF37913F0010F27D0FA
:107F5800DFF8488298F8009019F00F0920D17E4B7D
:107F68000A2259781878103902FB0011B170197972
:107F7800D878103902FB00117170D9799B791039C2
:107F880002FB0312327018F039FFF37969F300032A
:107F9800F37198F800305A1C62F3030388F8003034
:107FA800DFF8FC9199F8006016F001063EF43BAE4C
:107FB8006A4B01221A701AF071FD2378092B01D03F
:107FC8000D2B28D10120664912F0FCFA654B664A50
:107FD8005B7803F01F03D35C644A522B137002D101
:107FE800634B01221A70634B634A03F1200153F873
:107FF800040B8B4242F8040BF9D1002117A812F0A8
:108008000BFB17A80D211BF04FFD5C4B1A780132B2
:1080180002F003021A7099F8006006F00206F6B240
:10802800002E00F08B800FF053FD13F095FE06989C
:108038000322431C93FBF2F202EB42029B1ADBB2CF
:108048000693002B79D1DFF8488198F84960C24639
:10805800002E4DD0022E03D198F80130312B49D093
:1080680023780E2B13D1464846490522F8F712FC0F
:108078008246002840D1B21F37484349F8F760FCD0
:10808800344B5646DA7942F00102DA7135E00D2BAD
:1080980003D13E483A49072227E0032B22D13C4B23
:1080A800002713F8012F2C2A03D00137FFB2B7425B
:1080B800F7D113A832493A46F8F742FC7B1C07E08F
:1080C8000AEB03025278303AD2B2092A03D80133B4
:1080D800DBB2B342F4D30AEB0701FA430FA802312B
:1080E800D21802E0264909A8721EF8F729FC03E015
:1080F800069E02E0012600E000261E4B204A03F1FE
:10810800100153F8040B8B4242F8040BF9D1214BB0
:10811800214A03F1100153F8040B8B4242F8040B77
:10812800F9D1402388F811301C3B88F82230023BF3
:1081380088F84B301BF040FA00E0002699F8003030
:1081480003F0F5036FF3000389F80030FEF76BBD09
:1081580032690208FC5400205A1C002066130020D3
:108168002D5B00202C5B00203C9F0208303A002049
:10817800541C0020F4010020643A0020E13900205A
:108188009B5700206F540308A05700206C1C002048
:108198009A57002004020020AC570020551C0020EC
:1081A80074570020AFF3008010B5044640181146FC
:1081B800F8F7E2FA2046F8F73DFBC0B210BD42548A
:1081C8000131C8B27047000010B50D4B0D4A1B783D
:1081D8000C460E2101FB0323997A39B10139052395
:1081E800594301F56E51443189B201E043F6C43177
:1081F8000019042209F0EFFB201DC0B210BD00BF1A
:10820800B15D00202817002010B5054B0C461978E1
:1082180000190131042200F09FFB201DC0B210BDDF
:10822800B15D002000F5344008B5CB3009F0C2FB41
:1082380010F0FF0F14BF0020012008BD10B50A463A
:1082480000210446FFF7B0FF01462046FFF7DCFF98
:10825800114A01462046FFF7A7FF23220146204680
:10826800FFF7ADFF01462046FFF7AEFF5B22014650
:108278002046FFF7A4FF232201462046FFF79FFF71
:1082880001462046FFF7A0FF7C2201462046BDE8B4
:108298001040FFF794BF00BF7554030810B55D2266
:1082A8000446FFF78CFF0D2201462046FFF787FFA3
:1082B8000023235410BD38B51D460C4640182C1910
:1082C80011461A4600F048FBE0B238BD2DE9F041EE
:1082D80018490446FFF7B2FF174F0E263B78174D93
:1082E80073430146EA5A20460423FFF7E4FF20229D
:1082F80001462046FFF763FF3B78014606FB035320
:1083080020469A7A0223FFF7D6FF2022014620460C
:10831800FFF755FF3B78014606FB035520466A7A6E
:108328000323FFF7C8FF01462046BDE8F041FFF7E9
:10833800B5BF00BF78540308B15D0020281700209E
:108348002DE9F047264E0E223378264F534337F94E
:108358000380FA1824494FF47A73044698FBF3F81B
:10836800157AFFF76BFF4E2201462046FFF727FFDD
:108378001E4B1C2202FB05355FFA88F8B8F1030F83
:1083880001460CBF05F1120205F108022046FFF76D
:108398000BFFA1468046002519E019F8013BA32BE5
:1083A80007D133780E2202FB0373204629465A7AF6
:1083B80008E0242B09D133780E2202FB03739A7A42
:1083C800204629460223FFF776FF0135EDB24545E1
:1083D800E3D120462946BDE8F047FFF75FBF00BF5D
:1083E800B15D002028170020825403085C9F020812
:1083F800074B187800F00400C0B240B11A686FF358
:1084080082021A60034B00221A70034B18787047D7
:10841800DC390020901C0020781C0020054B00212E
:108428001970054B05481A6861F382021A60122216
:10843800F7F7B0BF901C0020DC390020781C002022
:1084480038B5084C084922780546F7F7FBFE23782B
:108458000021E954054B1A6861F382021A602078FA
:1084680038BD00BF901C0020781C0020DC3900209B
:10847800064A07491378112BC85401D801331370E1
:10848800044A136843F0040313607047901C0020EB
:10849800781C0020DC390020054B1B7813F0010FF5
:1084A80005D1044B181810F8010CFFF7E1BF70470D
:1084B800911C0020726902082DE9F041334C002319
:1084C80014F8101094F82A2001F00F0161F3030248
:1084D80084F82A2004EB400084F8293084F82830F6
:1084E8004378DFF8B88063F30712638C4FF4D277D0
:1084F800E38498F800302A267B4306FB0133244D99
:108508002448E95A84F82A201DF020FD98F8003004
:1085180094F82A207B4302F00F0206FB0233EB1883
:1085280059881C48013989B21DF014FD01210A46F9
:1085380018481DF0DBFC012116481DF0C8FC98F80E
:10854800003094F82A207B43120906FB02331248B4
:10855800E95A1DF0FBFC98F8002094F82A3057439C
:108568001B0906FB0376AD1969880B48013989B2E6
:108578001DF0EEFC01210A4607481DF0B7FC06482D
:108588000121BDE8F0411DF0A2BC00BF921C0020F3
:108598007E6902080008004000340140BE1C00202B
:1085A80030B5164C94F82B50A38445F001050023F0
:1085B80084F82B50628484F8211084F8203019E064
:1085C800C55CA5F13002D2B2092A08D9A5F1410249
:1085D800D2B2052A9ABFA5F13702D2B22A46084D6F
:1085E800013305EB420292F8495392F8482325706B
:1085F80062700234DAB28A42E2D330BD921C0020A3
:108608007E690208124B10B59A8C0024DA8483F82C
:10861800294083F82840224601210E481DF066FCB7
:1086280064210C481DF092FC32210A481DF092FC8E
:108638000121224608481DF059FC642106481DF016
:1086480085FC05483221BDE810401DF081BC00BF03
:10865800921C0020000800400034014010B50021A1
:108668002C220348F7F796FEBDE81040FFF7CABF73
:10867800921C002070B5214C2378042B39D8DFE8F0
:1086880003F0030D152A30001D4B012093F82B3001
:1086980013F0010F30D02070013870BD184B93F8DB
:1086A8002000FFF709FF0223237022E0144DEE8C0F
:1086B800FEB9FFF7A7FF95F8203095F82120013380
:1086C800DBB29A4285F8203001D8042300E0032366
:1086D8002370304670BD0A4BD88C50B901232370E3
:1086E80070BD074BDD8C35B9FFF7B8FF2570012049
:1086F80070BD002070BD002070BD00BFBF1C0020F1
:10870800921C0020044B00225A701A709A7842F08A
:1087180001029A70704700BFE81D0020202102481E
:108728000A46F7F737BE00BFF401002038B5044603
:1087380008460D46F8F77EF898B10319202B094B27
:10874800C8BFC4F120001C19002308E014F8012B4D
:10875800E02A14BFEA5C202204F8012C013383428A
:10876800F4DB38BDF40100200D4B46F669321B6876
:108778009B6893420FD043F6FC2293420BD0122BF6
:1087880009D0B3F5E97F08D046F60D401B1A5842C8
:1087980040EB03007047012070470120704700BF7D
:1087A800F81C0020F0B51F4687B006460C46084660
:1087B80000211546F7F7EEFD244B07B19F80B3F96A
:1087C800041005A801EB8601042209F004F900262B
:1087D80005AB9B5D013BDBB2B92B35D81D2B4FEAAE
:1087E800031209D8D31803F52641684601F5BF716D
:1087F800112209F0F0F80BE01549D3185B186A4606
:1088080003F11007186859680833BB4203C2F9D14D
:108818002046F8F70FF8C7B26846F8F70BF838188B
:10882800A84203D8E0196946F7F7A6FF6846F8F7A3
:1088380001F87B1C1B18AB4203D2E0190549F7F776
:1088480003FE0136042EC3D107B0F0BDE81D002099
:10885800803603089A54030810B500216C22044698
:10886800F7F798FD0123A37010BD00234370037030
:10887800837843F001038370704700002DE9F041CD
:108888009378804613F0010F0D4614463AD06FF3E3
:10889800000393701AF068FE6378002B32D12378B6
:1088A8000BB90A336370A378174F6FF30003A370F3
:1088B8001AF05AFE217807EB08066118073130468E
:1088C8002A46F8F73DF83046F7F7B4FFC6B2AE428D
:1088D8000DD80AD20023237006EB08000A33637010
:1088E80038182021AA1BF7F755FDAE420AD1227885
:1088F800A3181B7A1BB101322270BDE8F0812370E6
:108908000A236370BDE8F081F4010020054B1A7852
:108918000AB100221A701B7846F68A4202FB03113C
:10892800FFF704BFDB1C0020F8B505460C46081805
:10893800002109F035F8013CE4B26719384609F01E
:1089480039F8C6B2202E03D83846002109F028F895
:108958000CB1202EEFD9F8BD02F00F03032B22F043
:108968007F0230B5D2B20CD94FF47A7491FBF4F48B
:108978002025E4B2057002B114B13034047000222D
:108988000130B1F57A7F05DB4FF47A7491FBF4F589
:1089980004FB1511022B0BD9642491FBF4F4202558
:1089A800E4B2057002B114B1303404700022013011
:1089B800632904DD642491FBF4F504FB1511012BF4
:1089C8000AD90A2391FBF3F32024DBB2047002B125
:1089D8000BB1303303700130092904DD0A2391FB00
:1089E800F3F203FB12113031017030BD13B5104B97
:1089F80001461B689A899C7B12F0100214BF022062
:108A0800012034B10B4C9B7C2478634303FB001199
:108A180009B23AB10DF10600022208F0DCFFBDF8F8
:108A2800060002E0084608F0C5FF00B21CBD00BF02
:108A3800F81C0020871D002010B50F4B1B689A8971
:108A48009C7B12F0100214BF0221012134B10B4C9F
:108A58009B7C2478634303FB010000B22AB10849D8
:108A68000222BDE8104008F0B0BF054B1968BDE808
:108A7800104008F095BF00BFF81C0020871D00209B
:108A8800A01D00203038C0B2092894BFFF20002064
:108A980070470000024B1A786FF300021A70704793
:108AA800D71D002070B5FFF7F5FF884B1A781E2AEE
:108AB80001D91E221A70864C2678254606F0F00643
:108AC800202E72D109F0D2FA00286ED1814B1B7882
:108AD80033B92378C3F30312013262F307135EE05C
:108AE8007D4B1B7803F08003DBB2002B59D07B4809
:108AF800F7F7A0FEC5B27A4CBDB120467949324697
:108B0800F7F71EFF0A2D0BD82A4620467349F7F7B8
:108B180017FF60193146C5F10A02F7F73BFC04E07C
:108B280020466E490A22F7F70BFF6F4B1B7813F0AC
:108B3800010F01D0472300E02023E372684C042290
:108B480004F10C00A521F7F725FC684B1A7852B1FF
:108B5800FF23012A237306D9022A637303D0032A49
:108B6800A37318BFE373624C257815F0600502D132
:108B780094F8A33013B95F485F4902E05D4804F1F7
:108B8800A3010622F7F7DCFE5C4B1B78452B40F06F
:108B98009A81002D40F09781237843F08003237059
:108BA80070BD4F485649324682E12C7804F0F004F3
:108BB800102C3FD109F05AFA00283BD12022514904
:108BC8004748F7F7BDFE46484E492246F7F7B8FE34
:108BD8004D4B1B7813F0010F06D04C48F7F72AFECF
:108BE8004A4902464A4805E04A48F7F723FE4949F8
:108BF80002464748F7F7A4FE364B1B781BB9464890
:108C08004649102254E1444845491022F7F798FE96
:108C1800314B1B7803F08003DBB22BB13B48F7F7ED
:108C280009FE02463F484FE03A48F7F703FE02467E
:108C38003C4842E02B7803F0F003302B7ED109F05A
:108C480015FA00287AD1264C202237492046F7F712
:108C580077FEA521052204F10B00F7F79BFB334BA8
:108C68001B78042B02D9FF23E37300E002D1FF2312
:108C7800A37301E0032B02D1FF23637301E0022BEE
:108C880002D1FF23237300E00BB1FF23E372284BCB
:108C98005B7813F0600F05D03F23E372237363738F
:108CA800A373E373234B1B7803F02003DBB233B1C8
:108CB8001848F7F7BFFD02461F481649F8E0134861
:108CC800F7F7B8FD02461C481049F1E0E31D002003
:108CD800D71D00202C260020002600200426002076
:108CE800F40100206CFC0208A85D0020F926002091
:108CF800342600200E02002087D20208C01C002063
:108D08002AFC02086F320308723C0020B9330308BA
:108D180001020020DA330308040200203C3803086B
:108D280090320308110200202CD302081F2C0020C7
:108D38003C310020DC3900200F0200202B7813F092
:108D4800F0030CD1202260496048F7F7F9FD604B29
:108D58005E4819888322BDE87040FFF7FDBD602B8F
:108D68001ED109F083F9D8B95A4920225748F7F794
:108D7800E7FD5948F7F75EFD574902465748F7F7A8
:108D8800DFFD5748F7F756FD554902465548F7F7AE
:108D9800D7FD5548F7F74EFD53490246534887E03B
:108DA8002B7803F0F003102B06D109F05FF918B106
:108DB80046484F4920227BE02B7803F0F004402CF2
:108DC80002D0502C78D108E040484A492022F7F7D1
:108DD800B7FD494B1B784BB94CE03C48474920222A
:108DE800F7F7AEFD464B1B783BB943E0454B5A7845
:108DF80082B11B78022B14D105E0434B1B7813F08A
:108E0800010F07D00DE04148F7F714FD3F4902462E
:108E18003F4835E03F48F7F70DFD3E4902463C48DC
:108E28002EE03D48F7F706FD3B4902463848F7F77C
:108E380087FD402C0BBF334B384B5B78DB78022B1C
:108E48000AD0042B0FD0012B1CD13548F7F7F2FCC0
:108E58003349024633481BE03348F7F7EBFC324905
:108E68000246304814E03148F7F7E4FC2F4902463F
:108E78002C480DE02E48F7F7DDFC2D490246244822
:108E8800F7F75EFD2B48F7F7D5FC2A490246254837
:108E9800F7F756FD284B1B78ABB92021072221484C
:108EA800F7F778FA2248F7F7C5FC214902461D482A
:108EB800BDE87040F7F744BD204A6FF307131370FD
:108EC8001F4B00221A6070BDC9D20208F4010020AD
:108ED800D61C0020A8D20208A8CB0208F80100205E
:108EE800B2CB020808020020ADCB02080F02002016
:108EF8000BD30208B1320308C4390020D232030868
:108F08002C260020D6350020A85D002077330308E2
:108F1800FD0100201C340308B9330308D4250020C0
:108F2800F33203080D020020143303083533030815
:108F3800FB33030856330308BB330020D71D00203A
:108F4800F81C0020204B70B5F022204D1A702B78A9
:108F580013F0010F0BD01E4C207810F0010006D141
:108F68001C49FFF7D3FC237843F0010323701A4E02
:108F78003378532B0ED1164C237813F0010F07D0FA
:108F880000201649FFF7C2FC23786FF30003237013
:108F9800FFF780FD3378232B14D10D4B1B7813F08A
:108FA800010F0FD1FFF776FD2B780D4A43F006032A
:108FB8002B701378013BDBB213700A4A52F8232056
:108FC800094B1A6070BD00BFE31D0020D71D0020AB
:108FD800FD1C002040280308C01C00201F2803088F
:108FE800B71D0020C41D0020F81C00202DE9F04109
:108FF8005C4BF0225C4D1A702A7802F01003DBB249
:10900800002B2DD1594963F347120B601C462A7077
:10901800574A9A5C2D2A01D00134E4B20133082B57
:10902800F6D1544E3A213046F7F732FA38B1801B60
:10903800C0B20130301821460222FFF78DFC4E4B9A
:109048001B78452B40F08B8000242046013412F019
:10905800DBFE082CF9D12B7843F010032B7038E095
:10906800464C237813F0010F17D1404E4448FFF7C0
:10907800F3FB404F3168384601310222FFF76CFCA0
:109088002D23BB70307846F695533E496522FFF78D
:1090980089FB237843F00103237003200D21384A0C
:1090A800FFF7ECFB2D78304E15F0E00541D110208C
:1090B8003549FFF72BFC304B1B78442B0DD12B4A3D
:1090C800136801332A4903F00703C95C2D29F8D036
:1090D8001360BDE8F041FFF7DDBC532B0DD13278AA
:1090E8004E3B63F347123270204A28491268062023
:1090F80000FB02125380BDE8F081232B2FD11B4BBC
:109108001D60337803F0EF0365F347133370FFF7FF
:10911800C1FC23781E4A43F0060323701378013BF1
:10912800DBB213701B4A52F823201B4B1A60BDE8B0
:10913800F081104C10201949FFF7E8FB04F11000EA
:109148002821F7F7A5F950B1001B3178C0B20130DA
:10915800201849098022BDE8F041FFF7FDBBBDE8B2
:10916800F08100BFE31D0020FD1C0020A01D002091
:10917800ED3A0020F4010020C01C0020D71D00207B
:10918800E81D0020EF1D0020BC2703080A3B002033
:10919800B71D0020C41D0020F81C0020DD2703088F
:1091A800454B2DE9F041F022444E1A703378444D76
:1091B80043F0010333702B68424C9B7C022B06D191
:1091C800414B1B7803F04003DBB23BB10FE0012BAE
:1091D8000DD13E4B1B7813F0010F08D109F0BEF8F2
:1091E800236800206FF355532360394944E0A3787E
:1091F800344F03F02003DBB2C3B909F0AFF8F878B5
:1092080000F02000C0B288B92968324B897C1A78EE
:1092180061F301021A703B682D4943F400133B6067
:10922800FFF774FB2C4B802283F843200DF052FD8E
:10923800804678B12B689B7C012B08D1234B5B7847
:1092480003F01003DBB213B10020244914E000201E
:10925800234911E00DF06EFD074610B14046214943
:109268000AE00DF0AFFD10B138461F4904E01A4B73
:1092780093F8433013B91D49FFF748FB1C4B1B7883
:10928800232B16D1FFF706FC337843F0060333701F
:1092980009F064F823686FF3555323600CF00EFC53
:1092A800144A1378013BDBB21370134A52F8233087
:1092B8002B60BDE8F08100BFE31D0020D71D002012
:1092C800F81C0020DC39002000260020723C002019
:1092D80061280308773C002081210020A328030887
:1092E80082280308E5280308C42803080629030878
:1092F800C01C0020B71D0020C41D00202DE9F3412B
:109308006E4B6F4DF0221A702B686E4C9B7C1BB90C
:10931800637843F0100302E0637843F008036A4E71
:109328006370337843F001033370238823F47E633A
:1093380023F01E03DB04DB0CB3F5805F08D0634B1E
:109348001B7883B15F4B5B7803F00803DBB253B142
:10935800637800206FF341035D496370FFF7D6FA25
:10936800F8F7AEFE84E06378564F03F00203DBB2F1
:10937800FBB9BB78EBB9574B93F8008018F001089C
:1093880017D1F8F79DFE7B7843F002037B702B68BA
:10939800B3F91030022B7B780CBF43F0040368F359
:1093A800820300217B70082001220B460091F9F707
:1093B800A5F9A378434A032B28D003D8012B0BD057
:1093C8000DD806E0052B2DD0517825D3FF2B32D1AF
:1093D8002BE000203E4949E000203F4946E03F4855
:1093E800F7F728FADFF82C81C7B23C4908F11000DA
:1093F8003A46F7F7A5FA0F2F3AD807F1100040447C
:109408002021C7F11002F6F7C5FF31E0344B187878
:1094180000282DD1334929E06FF341015170002014
:10942800314923E00020314920E06FF341015170B8
:1094380000202F491AE0053BDBB26FF34101022BF4
:10944800517002D100202B4910E0012B02D10020DD
:1094580029490BE0032B02D10020284906E0052BFF
:1094680002D10020264901E026490020FFF74EFAE4
:10947800637803F00203DBB20BB9F8F721FE224B45
:109488001B78232B18D1FFF705FB3378002243F014
:10949800060333706378A27003F0E50362F3820376
:1094A8006370F8F70DFE194A1378013BDBB21370AD
:1094B800174A52F823302B60BDE8FC81E31D0020D9
:1094C800F81C0020A85D0020D71D0020D6350020FC
:1094D80061280308AE5D0020A4240308B75D0020BE
:1094E800AC5D0020C5240308692903084925030841
:1094F800AC250308E62403080725030828250308E4
:109508006A2503088B250308C01C0020B71D00200E
:10951800C41D0020F40100207B4B2DE9F341F0220B
:109528007A4E1A7033787A4D43F0010333702B6802
:10953800784C9B7C022B11D1774B1B7803F04003AE
:10954800DBB293B1754B1B7803F02003DBB2BBB1E0
:10955800A37803F04003DBB23BB111E0012B0FD13C
:109568006F4B1B7813F0010F0AD1F8F7A9FD236898
:10957800002023F480036FF3D753236069498FE0F9
:10958800A778DFF8908107F04003DFB2002F34D1CD
:10959800F8F796FD2968644B897C1A78384661F398
:1095A80001021A70D8F800305E4943F4800367F36B
:1095B800D753C8F80030FFF7A9F92B68198A21B9E1
:1095C8000091082001220B4615E00BB2022B0CD1AA
:1095D80001223B46082039460097F9F78FF8534B8C
:1095E8001A7842F008021A7007E0012B05D100979B
:1095F8000E2039463A46F9F781F80DF06BFB07461D
:1096080078B12B689B7C012B08D1454B5B7803F024
:109618001003DBB213B10020454941E00020454961
:109628003EE0414B3946187800F00300F8F780FE19
:10963800FF280FD13D4B1B7803F01803182B31D0AE
:10964800A07800F08000C0B210B138463A4927E04F
:109658003A4925E00DF06EFB8046E0B1334B1878AF
:1096680000F008085FFA88F8B8F1000F0AD1F8F797
:10967800B5FFC0B2022801D840460AE0062811D832
:10968800404604E000F01000C0B210B138462C4942
:1096980006E02C4904E00DF095FB18B12A49404634
:1096A800FFF734F9294B1B78232B29D1FFF7F2F95F
:1096B800337843F006033370F8F702FD236823F488
:1096C80080036FF3D7532360184B1A786FF3C302E4
:1096D8001A701F4A1378013BDBB213701D4A52F807
:1096E80023302B60104B1B7803F00303022B02D1AD
:1096F8000DF0C6FA20B102B0BDE8F0410CF0DEB9B9
:1097080002B0BDE8F08100BFE31D0020D71D002096
:10971800F81C0020DC390020002600203426002018
:10972800723C002061280308773C0020101F0020AD
:10973800A328030882280308692903088A2903083B
:109748004829030827290308C4280308C01C002047
:10975800B71D0020C41D002010B5FFF79BF90A486B
:109768002523C377094B0A4A1B6813219B7C1C30AD
:1097780001FB03235B78093903F00F035943832264
:10978800BDE81040FFF7E8B8F4010020F81C0020FD
:10979800E63900202DE9F047514D524F2B78F02241
:1097A80043F001032B70504BDFF878911A703B6837
:1097B8009C6847F2F373E21A544244EB0204132103
:1097C80061434A4A565C5318C6F300065FFA86F8A6
:1097D8009246B8F1000F23D140464549FFF796F865
:1097E80099F80030232B79D1FFF754F92B78414AA7
:1097F80043F006032B701378013BDBB213703E4A2B
:1098080052F823303B603D4B1E703D4B1E703D4B64
:109818001E703D4BC3F800803C4B1E70BDE8F087BE
:1098280099F80020232A21D19A786FF300029A70C0
:109838000EF0FAF9FFF72EF92B782E4A43F00603BB
:109848002B701378013BDBB213702B4A52F823308C
:109858002A4A3B6000231370294A1370294A13705F
:10986800294A1360294A1370BDE8F087532A13D197
:109878009A7812F001010FD172206043244D42F012
:1098880001022E5C61F300062E549A701E4B0122D1
:109898001A60204616F0FAFC132303FB04A39B78F6
:1098A80013F0010F02D000201A4913E0164B1B6871
:1098B80073B9382102221848FFF74EF8204615F0F0
:1098C8007FFF014615480222BDE8F047FFF744B87C
:1098D80013490020BDE8F047FFF718B8BDE8F08746
:1098E800D71D0020F81C0020E31D0020E6390020C9
:1098F800F7E00208B71D0020C41D0020DD1C002071
:10990800061D0020871D0020A01D0020921D00209C
:10991800105400209A2B0308120200200D02002088
:10992800792B0308C01C00202DE9F0412D4E2E4F45
:10993800307800F5E240F13008F03CF83B78C4B2EA
:1099480013F0010F26D0294D2B78552B0AD1EC2C7A
:1099580001D0013CE4B23078214600F5E240F13014
:1099680008F01EF82B78442B0DD1A4F11403DBB2B8
:10997800D72B01D90134E4B23078214600F5E24012
:10998800F13008F00DF82B78532B03D1FFF782F84C
:109998000EF04AF9164B1B7803F08003DBB253B183
:1099A8003B7813F0010F06D0124820210422BDE8AD
:1099B800F041F6F7EFBC14F0800F0F4805D12B23C8
:1099C8000A2103746143113006E02D230374373BE9
:1099D8005C43113004F520610322BDE8F041FEF735
:1099E800BBBF00BF871D0020D71D0020C01C002062
:1099F800DC39002004020020F40100201FB5204BB0
:109A080020491A781AB1087840F0010008700978DE
:109A18001C4C11F0010F31D01B490978532901D092
:109A28000AB103E082B901221A700DE023290BD193
:109A3800002018701549FEF769FFFFF72BF8237807
:109A480043F00603237019E01B78012B16D120215F
:109A58000A460F48F6F79EFC0E4B68461B68102214
:109A6800996807F0B8FF002409491DF8040001EBC4
:109A7800440101341AF0C4FE102CF5D11FBD00BFFB
:109A8800871D0020D71D0020C01C0020B22E03080F
:109A9800F4010020F81C0020034B1B78532B01D144
:109AA800FEF7F8BF704700BFC01C0020084BFF2816
:109AB8001A68936807D1917B41B10649927C09786D
:109AC80001FB023302E0927C02FB00331846704728
:109AD800F81C0020871D00204328F8B504460D46D1
:109AE800174608D1114B0A261A7891FBF6F66FF340
:109AF800C3021A7000E00E462046FEF7C3FF90B17D
:109B08000A4B303C1A780A2602F00801C9B200292B
:109B180018BF002506FB05466FF3C30236B21A705C
:109B2800BE42A8BF3E4630B2F8BD00BFD71D0020D8
:109B3800624B2DE9F3411A689846157C977C604C76
:109B48002DB1604821780222FEF706FF00E025705B
:109B5800FF01237807F51C4707F5B47707EB4307A0
:109B6800594E0BB90DB10FE015B901A8394601E0FE
:109B780001A8B91E022207F02EFF9DF80430F375E4
:109B88009DF80530337605E006F117003F210222E3
:109B9800F6F700FC5B23B375023373764B4B1B78E7
:109BA80013F0010F5DD04A4B1B78A3F13002D2B2FB
:109BB800092A31D822780AB9002D3CD1454A1178B2
:109BC80096469942444A01D00021117043481178C1
:109BD800A3F1300490F800C004EB840404EB0108FE
:109BE80002A801318444C9B23D48641810F80880BD
:109BF800005D0CF8048C117008B1032901D900210B
:109C080011708EF800300DB9384600E0B81E01A971
:109C1800022207F0DAFE17E0232B04D12F4B1A7823
:109C280092B9013205E02A2B05D12C4B1A785AB18A
:109C3800013A1A7008E0532B06D12A4A533B137095
:109C4800264A1370FFF728FF274B1B7803F0800381
:109C5800DBB2002B2FD0214B1B78F6182023F3758D
:109C680029E045B31A4B1878A0F13003DBB2092B71
:109C780010D81C4A137803B92370013303F0010389
:109C88001370D8F800302178B3F91020FFF724FFBB
:109C9800207005E0432803D1124B1B7803B92370C9
:109CA800114B1B7803F08003DBB223B10548202158
:109CB8000222F6F76FFBBDE8FC8100BFF81C00200C
:109CC800071D002002020020F4010020D71D0020FB
:109CD800C01C0020DA1C0020061D0020D81C002013
:109CE800EC6C0208921D0020DC390020F7B5384ED4
:109CF800384D3378384C6FF34103337019F026FA36
:109D0800FFF7CAFE02238DF807302B7883B1334A58
:109D1800D17941F00101D171314A207802EBC303B6
:109D28005F6B93F839203978FFF7D6FE38700DE06D
:109D3800337813F0010F06D02378303BDBB2062BC3
:109D48009CBF264AD37003238DF80730337813F06D
:109D5800010F12D0234B1B7803F08003DBB263B1F1
:109D680029781F4B204803EBC10393F838309DF83E
:109D78000720C0182021F6F70DFB2378232B09D1E3
:109D88001A4A2B781268927C013A934202DA114AF5
:109D98000133137023782A2B04D12B7813B10D4A81
:109DA800013B13702378532B0FD117F027F80B4B77
:109DB80000212970DA7961F30002DA71FFF76CFE8D
:109DC8000B4B9A7942F004029A7100232370FEBD6E
:109DD800D71D0020921D0020C01C0020FC5400202C
:109DE800EC6C0208DC390020F4010020F81C00208B
:109DF800041F00202DE9F74F924E934C3378934D72
:109E0800232B934F25D12368986843F6F123984272
:109E180017D1DFF86082296898F8000000F56A50C9
:109E2800713007F0BDFD98F80000013000F0010026
:109E380088F8000000F56A50713007F0BBFD286013
:109E480007E000B2FEF7D2FD28603B7843F0080334
:109E58003B703378532B40F06781236849F61552DD
:109E68009B68934202D12A687A4B15E04BF2B642BE
:109E7800934202D12A68784B0EE04BF23342934268
:109E880002D12A68754B07E049F66652934204D11D
:109E98002A68734B02B101221A7023689A6843F644
:109EA800DD239A420AD16F4B29681A7861F30002C0
:109EB8001A7008F0DBF808B108F0F6F8236843F6E2
:109EC800E0229B68934206D1664B29681A7861F3B1
:109ED800C7121A7019E043F6EA22934206D1614B81
:109EE80029685A7861F300025A700EE043F6E722B7
:109EF80093420AD129685C4B19B11A6842F00052A2
:109F080002E01A6861F35D721A6023689A684BF27E
:109F18004C539A420AD12968544B19B11A7842F025
:109F2800200202E01A7861F345121A7023689A68D1
:109F38004BF2D9539A4202D1287819F06FFE236860
:109F480043F6DA229B68934203D12A68484B1A7079
:109F580008E049F61E52934204D12B6813B93B4BD3
:109F680001221A6023689A684BF2DA539A420BD19D
:109F7800404A2B6812784049032B8B5404D13F4B3D
:109F88005A7942F010025A71236849F65E529B686A
:109F9800934202D129683A4A05E049F66152934250
:109FA80003D12968374A117016E049F66252934284
:109FB80003D12968344A117015E049F66452934276
:109FC80003D12968314A11701CE049F66552934261
:109FD80002D12A682E4B13E043F60852934202D16D
:109FE8002A682C4B0CE04AF26C72934202D12A6820
:109FF800294B05E04BF2CA42934203D12A68274B0A
:10A008001A700AE049F61652934206D12A68244B80
:10A0180001201A7001460EF00FFC2368986843F679
:10A02800F12398423ED1DFF84C80296898F8000067
:10A0380000F56A50713007F0B3FC002388F800304F
:10A0480033E000BFC01C0020F81C0020A01D002029
:10A05800D71D00202C260020C4390020BB33002047
:10A06800BE1C0020551E0020DC390020A85D002001
:10A078008A570020871D002020170020D4250020A3
:10A08800443D0020423D0020753C0020E93B002073
:10A09800841F00205E150020F51B0020761C002080
:10A0A8005E3B002000B2FEF7C7FC23689A6843F6BF
:10A0B80098139A4236D12968DFF8A8B2DFF8D0A2FF
:10A0C8000BEBC1031B79DFF8A082C3F34113012B0B
:10A0D800DFF8C09221DD98F8000000F566501C30CA
:10A0E80007F05EFC98F80030DAF8001009EB03027C
:10A0F80011710BEBC1021279C2F34112032A0CD180
:10A10800974A126890680830C01807F049FC98F818
:10A118000030DAF800204B441A7298F800302A68A8
:10A1280009F80320FFF7B8FC3B78DFF86C8213F0DE
:10A13800010F00F0DC80216843F698128B68934287
:10A148007FD1884A2B68914602EBC3010979C1F394
:10A158004111012906DD844A1278032A02D9FEF743
:10A1680099FCD0E03278442A36D15FFA83F82DE0A2
:10A1780008F101087B4B5FFA88F803EBC8031B79E9
:10A18800C3F34113012B06DD784B1B7823BB764BB9
:10A198001B78032B20D8DFF8D0A19AF800300F2BBA
:10A1A80008D807F063FF70B109EBC8031B7913F0F7
:10A1B800100F08D19AF800300F2B07D909EBC80304
:10A1C8001B79DB0902D0C5F8008005E009EBC8035C
:10A1D8001B7913F0080FCBD03378552B40F09380C0
:10A1E8002E782BE0013EF6B209EBC6031B79C3F3C8
:10A1F8004113012B08DD5D4B1B78002B40F0838059
:10A20800594B1B78042B7ED8DFF85C8198F8003016
:10A218000F2B08D807F02AFF70B109EBC6031B798A
:10A2280013F0100F08D198F800300F2B06D909EB5E
:10A23800C6031B79DB0901D02E6064E0002ED1D162
:10A2480061E04BF2DA5293420AD005DCA3F53442BE
:10A25800CA3A012A0ED803E04BF23762934209D179
:10A2680033782F2B4FD9B1F91020303293424ADC82
:10A27800303B30E043F6F122934207D13A4B1B784A
:10A2880023B13078B5F900103B222CE007F0EEFE40
:10A2980018B3236843F6C4219A688A4203D047F268
:10A2A80001118A4204D13078B5F900102D221AE044
:10A2B800A2F56A516139052903D943F6E9218A4291
:10A2C80001D1012307E043F6E0218A4202D00A3196
:10A2D8008A4203D100232B6015E023683078B5F952
:10A2E8000010B3F91020FFF7F7FB28600BE0236894
:10A2F800B3F90800FEF77AFB286098F8003043F0BD
:10A30800080388F80030FFF7C7FB236843F6D2221A
:10A31800986890420BD12B6813B91548154901E08C
:10A32800134815490222F6F70BFB0226C6E14BF249
:10A33800376290420AD12B6813B91048104931E0AE
:10A34800012B0E480CBF0F490F492BE04BF2DA5294
:10A35800904236D12B68012B20D108480B4921E0C7
:10A36800F81C002014040020871D0020820D002006
:10A3780012020020506D0208526D020804020020EB
:10A38800961A0308D81A0308B71A03086D190308A0
:10A39800A01D0020202C0020D71D0020022B05D155
:10A3A800A448A5491022F6F7CBFA86E1032B02D17F
:10A3B800A048A249F6E7042B9E480CBFA049A14932
:10A3C800F0E74BF2CA4290420AD12B6813B9994878
:10A3D8009D49E7E7022B97480CBF9C499C49E1E758
:10A3E8004BF2CB4290420AD12B6813B99148994954
:10A3F800D8E7012B40F061818E489749D2E749F6AA
:10A408006352904203D043F6EE2290420ED1286860
:10A418000A21B0FBF1F201FB1201904B3031D977E0
:10A4280030322E2199775A77032647E143F6F122F5
:10A4380090423ED18A4B1B78E3B9022229688948A9
:10A44800FEF78AFA43F6F220FEF7D0FA0222014616
:10A458008548FEF781FA3B7813F0010F00F07E8102
:10A46800824B1B7803F08003DBB2002B00F076816F
:10A478007C4819E0FEF7BAFA022201467948FEF74D
:10A488006BFA022278482968FEF766FA3B7813F0DF
:10A49800010F00F06381754B1B7803F08003DBB27A
:10A4A800002B00F05B81704820210222F5F772FF33
:10A4B80054E143F69812904240F0B2802B686C4EFB
:10A4C800DFF89C8156F8331010225A48F6F738FA0C
:10A4D8000DF1060298F800000DF1070110F0F6F9E9
:10A4E8004246334620B316786249895D03291FD056
:10A4F800296803EBC1010979C1F34111012917D179
:10A50800032E15D95C490B225C48F6F719FA5C480A
:10A51800711C0222FEF720FA9DF8071059480131F4
:10A528000222FEF719FA9DF806105748013118E083
:10A538002E68157803EBC601097903EBC606367950
:10A54800C1F34111012906F00706C8BF05F003054C
:10A55800012E0ADC4D4949480B22F6F7F1F9484823
:10A56800691C0222FEF7F8F9A7E0022E0BD1484930
:10A578000B224248F6F7E4F932464148691CFEF7D7
:10A58800EBF90E369AE0032E0BD142490B223B48D9
:10A59800F6F7D6F93A48691C0222FEF7DDF90D36BE
:10A5A8008CE0042E10D13C490B223448F6F7C8F948
:10A5B8003348691C0222FEF7CFF93248691D02228E
:10A5C800FEF7CAF90C3679E0052E10D133490B2273
:10A5D8002A48F6F7B5F92A48691C0222FEF7BCF9A1
:10A5E8002848691D0222FEF7B7F90B3666E0062EE9
:10A5F80063D12B490B222148F6F7A2F92048691CA0
:10A608000222FEF7A9F91F48691D0222FEF7A4F9E4
:10A61800244805F109010222FEF79EF90A364DE0A9
:10A62800B3F91060092E3FDD632ECCBF0326022646
:10A638003BE000BF040200208E190308AF1903088D
:10A64800D01903084C1903083B1B03087D1B03089A
:10A658005C1B0308BF1B0308E01B0308F401002070
:10A66800871D00200F02002012020020DC39002084
:10A6780014040020202C002024350308F9010020B0
:10A68800FA010020FE01002001020020E234030844
:10A698003D340308C13403087F3403085E340308DB
:10A6A800A03403080202002001262D482968801BD7
:10A6B80046F08002FEF750F900E010263B7813F0D0
:10A6C800010F0BD0274B1B7803F08003DBB22BB1B3
:10A6D80023482021801B3246F5F75CFE224EB378D2
:10A6E80003F00203DBB2002B38D0FEF73DF81F4D14
:10A6F800034628B92878F11D6522FEF753F808E0CB
:10A70800B2792978B388F01D01FB023109B207F04C
:10A7180062F9236847F201129B68934213D006DC62
:10A7280043F6C42293420ED043F69E5209E047F204
:10A738008112934207D049F61E52934203D047F242
:10A74800411293420AD105200B21074AFEF796F8D9
:10A758002978074801310222FEF7FEF8BDE8FE8F8E
:10A7680014020020DC390020E81D0020871D00208D
:10A77800F5010020F0B5114B1F78114B303F1E68D2
:10A788000DE0D6F814C01CF803C00133644501D1AC
:10A7980012E00023DAB28242F3D301350D70094B7F
:10A7A8000622094902FB07330D785B1993F86840C4
:10A7B800002CEED10C70F9321046F0BDC01C002000
:10A7C800F81C0020EC6C0208061D00202DE9F74F4C
:10A7D800974C984E23689A6843F609539A4203D1D6
:10A7E80033780BB9013333702368934F9968B3F901
:10A7F80010303A78B3F1010848BF03F106084FEA70
:10A80800E808337808F1010812F0010F03FB081873
:10A818008A4D00F0AD808A4B1A789946432A4DD16B
:10A8280028780FFA88FA0AEBD00007F0C3F82268F4
:10A83800844B916846F2C8629142186001D12A7827
:10A848003AB12A78012102F0070211FA02F25040C7
:10A858001860287819780AEBD00007F0A1F8236867
:10A8680047F2E1129B68934209D1744B1A78764BF0
:10A8780003EBD203734A126883F8A0211EE046F660
:10A88800A932934205D13178002001310EF030FB16
:10A8980014E046F2BF7A4FF0000B23689B685345DB
:10A8A80004D101200BEB00010EF022FB0AF1080A8B
:10A8B80046F2DF739A450BF1010BEED199F800309F
:10A8C800232B10D122682B78927C013A93420ADA22
:10A8D8005A4A013313705D4B9B7803F00203DBB2D5
:10A8E8000BB1FDF70FFF99F800302A2B0CD12B780C
:10A8F80053B1524A013B1370544B9B7803F0020347
:10A90800DBB20BB1FDF7FEFE99F80030552B14D1E0
:10A918002368997C0F2910D92A7808398A42474B2D
:10A9280001DA083200E000221A70484B9B7803F0E5
:10A938000203DBB20BB1FDF7E5FE99F80030442BBA
:10A9480042D123689A7C0F2A3ED929783B4B0729A4
:10A9580002D90839197001E0083A1A703B4B9B7804
:10A9680003F00203DBB2002B2ED0FDF7CBFE2BE069
:10A9780049F6D54399420ED1314B1B78A3F13101E9
:10A98800C9B2032907D842F006023A700722534396
:10A99800284A573B137023689A6843F609539A422A
:10A9A80012D133781B2B08D9284B46F695429A804A
:10A9B8009A7842F002029A7006E05901C918244BAD
:10A9C8000020C918FDF7A2FFFFF766F8214A2B7887
:10A9D80011789346994288BF137012780F329342C8
:10A9E80002DD1C4A0F3B137023684FF0000A93F8EE
:10A9F8001290B9F10F0F9ABFC9F120095FFA89F9CE
:10AA08004FF010099BF800004FFA8AF318180FFA54
:10AA180088F202EBE000019306F0CCFF9BF80020DF
:10AA2800019B5FFA80FC9B1803F007032BE000BF33
:10AA3800F81C0020871D0020D71D0020921D002033
:10AA4800C01C0020A01D0020202C0020E81D002094
:10AA5800F01D0308891D00204CFA03F065490133F5
:10AA680000F0010000280CBFA520DB20DBB201F8B4
:10AA780009000AF1010A09F10109082B5FFA8AFAAB
:10AA88005FFA89F903D0B9F1200FE5D109E0B9F1EE
:10AA9800200F06D023684FFA8AF19B7C89189942C7
:10AAA800B0DB3B7813F0010F15D0236852499B7C2B
:10AAB80009780F2B01F0800198BFC3F11003C9B2C8
:10AAC80094BFDBB2002331B1297810318A1A494981
:10AAD800CB185F219954494FBB7803F00203DBB2CE
:10AAE800002B61D0FDF740FE0346F8B9226846F610
:10AAF800A93192688A4206D024318A4203D043F6AB
:10AB0800E5118A4204D130783D496522002308E0E6
:10AB180043F609518A4207D130781C38C0B2F91D72
:10AB28006522FDF73FFE18E02878F8E7236846F627
:10AB380069329B68934203D043F6FC22934202D1C8
:10AB4800BA79317801E0BA792978BB882C4801FBB9
:10AB58000231BA7909B206F03EFF23689A7C102ABE
:10AB68001DD89B6846F6693293420ED006DC43F640
:10AB7800E512934209D043F6FC2204E046F6A932D6
:10AB8800934202D02432934202D11020072108E0D8
:10AB980043F60952934202D10020102101E005201A
:10ABA8000B21164AFDF76AFE226846F60D419368A6
:10ABB8008B421BD046F6C7218B4217D043F6ED21B6
:10ABC8008B4202D10B4BDB219977937C0B2B0DD950
:10ABD800BB7803F00203DBB243B12978094801319D
:10ABE800022203B0BDE8F04FFDF7B6BE03B0BDE8E2
:10ABF800F08F00BFF4010020DC390020E81D0020A0
:10AC0800EF1D0020F5010020114B002270B50D4604
:10AC18001A7118B11B7803B920234370BDB10D48D0
:10AC2800F5F708FE0446681C5CB10A492246F5F7A8
:10AC380009FB022C0BDC601C28182021C4F103023C
:10AC480001E020210322BDE87040F5F7A3BB70BDE9
:10AC5800741D0020751D002038B50546002408E045
:10AC6800601906F0A7FE3038C0B2092808D80134A8
:10AC7800E4B2044B1B78303B9C42F1DB012038BD29
:10AC8800002038BDDC1C002008B506F093FE002328
:10AC9800C0B2064AD25C824201D1202804D10133D5
:10ACA800082BF6D1002008BD012008BD906D0208D0
:10ACB80070B506460D4600240DB12D232B55A0195D
:10ACC8000021013406F06CFE062CF5D170BD0000A1
:10ACD8002DE9F04F974C984F206839788368068A99
:10ACE8009AB201FB06260D4648F63C118B4287B006
:10ACF800B6B20BD1914B1A785B7802F00702C3F316
:10AD0800420303EBC20306EBC3062BE048F6FC2123
:10AD18008B4212D1894B8A481A78597802F0070277
:10AD280088235A43C1F34201773B03FB01232021C7
:10AD38000822F618F5F72EFB14E048F6B4618B42AA
:10AD48000BD17E4B1A785B7802F00702C3F34203FB
:10AD580003EBC2039B01F61804E0B3F5E97F08BFD3
:10AD680002EB4506774B784D1A78984612F0010F9A
:10AD780053D123689A6847F209039A4204D046F6E9
:10AD880009639A4240F04481704B1B782A2B3BD1CF
:10AD98006F4B93F8009009F1010909F0010983F854
:10ADA8000090B9F1000F1AD046F609639A4208D10B
:10ADB800684B46F695429A809A7842F002029A7059
:10ADC80026E1202110226448F5F7E4FA3B780020B8
:10ADD8005901C918614BC918FDF798FD18E15D487C
:10ADE800FDF73AFD236848469A6846F609639A4291
:10ADF8000CBF5B495B49FDF789FD39785A48013139
:10AE08000222FDF7A9FD03E1552B02D0442B40F0A7
:10AE1800FF804F4B00221A70FAE023685869F5F753
:10AE280009FD4A4B834693F800A09946BAF1450FAD
:10AE380002D14E4B00221A705046FDF723FE00281F
:10AE48004DD04B4B5FFA8BFB1A7852450ED15846C2
:10AE5800FFF790FCFF2804D15846FFF78BFCFF282A
:10AE68003DD0444B1A7801321A7015E0DFF804A17E
:10AE780000228AF8002058460593FFF77BFCFF283C
:10AE8800059B04D09AF8002001328AF8002099F82E
:10AE98000020FF281A7022D02168374A4B691060B9
:10AEA8001B5C886847F209018842136092460FD1FB
:10AEB800562B01D0542B0BD13B78123BDBB2022B23
:10AEC80006D82B7830B2C01806F074FDCAF8000016
:10AED8002B7830B2C018DAF8001006F061FD99F846
:10AEE8000030552B17D12368997C0F2913D92A785C
:10AEF80008398A42144B01DA083200E000221A703D
:10AF0800144B9B7803F00203DBB20BB1FDF7FAFB9D
:10AF1800184B00221A7099F80030442B3BD1236853
:10AF28009A7C0F2A37D92978074B072926D9083957
:10AF3800197025E0F81C0020871D00208D1D0020B9
:10AF480004020020D71D0020921D0020C01C0020F4
:10AF5800E21D0020E81D0020F4010020131603085C
:10AF68002414030866140308F5010020D81C0020E7
:10AF7800DA1C0020061D0020A01D0020083A1A70C7
:10AF8800964B9B7803F00203DBB20BB1FDF7BAFBDB
:10AF9800934B00221A7099F80030432B0CD1236888
:10AFA80030B25B6919788F4B19602B78C01806F09E
:10AFB800F7FC8B4B00221A7099F80030232B13D121
:10AFC80022682B78927C013A93420DDA864A013343
:10AFD8001370834B00221A70804B9B7803F0020396
:10AFE800DBB20BB1FDF78EFB99F800302A2B0FD19D
:10AFF8002B786BB17C4A013B1370794B00221A7095
:10B00800764B9B7803F00203DBB20BB1FDF77AFBBA
:10B01800FEF742FD754A2B7811789246994288BF0F
:10B02800137012780F32934202DD704A0F3B13708F
:10B0380023684FF0000B93F81290B9F10F0F9ABFE5
:10B04800C9F120095FFA89F94FF010099AF8000050
:10B0580033B218185844059306F0ACFC644A02F859
:10B06800090009F101095FFA89F9B9F11F0F059B78
:10B0780005D821680BF1010B897C8B45E6DB98F834
:10B08800001011F0010F16D021685A48897C007809
:10B098000F2900F0800098BFC1F11001C0B294BF21
:10B0A800C9B2002138B128789AF8006010305218D7
:10B0B800801B5F211154226890684AF26A7290429C
:10B0C8000AD14D4B1B78532B2FD106F073FC4B4BF9
:10B0D800187006F069FD28E0B0F5E97F25D1464AE9
:10B0E8001278532A21D11846FFF7CEFD0646E0B95B
:10B0F8003B78DA00D31A03F11200FFF7ADFD60B117
:10B10800FF2300933E4B01961B787920013302936D
:10B1180031460422334606F0CBFC3B780021DA00A6
:10B12800D31A03F11200FFF7C3FD2C4EB37803F0D6
:10B138000203DBB2002B6ED0FDF716FB034680B985
:10B14800226848F6B46192688A420AD046F60961D4
:10B158008A4214BF28783878F11D6522FDF722FB52
:10B168000FE02368B2799B682648B3F5E97F0CBFE6
:10B1780039782978B38801FB0231B27909B206F02F
:10B188002AFC23689A7C032A08D99A6848F63C1155
:10B198008A4203D046F609618A4214D19B6848F670
:10B1A8003C1293420CD198F8003013F0010F01D0F3
:10B1B80010202CE0202107221348F5F7EBF82AE0AD
:10B1C800B3F5E97F02D105200B2121E046F609629B
:10B1D80093421BD1002010211AE000BFE81D002077
:10B1E800061D0020A01D0020921D0020891D0020A2
:10B1F800F4010020DC390020C01C0020DC1C0020E9
:10B20800871D0020EF1D00200402002000200721D8
:10B21800104AFDF733FB23689A7C032A16D9B278C3
:10B2280002F00202D2B28AB19B6848F63C129342FD
:10B238000CD046F60962934208D0297806480131B5
:10B24800022207B0BDE8F04FFDF786BB07B0BDE8A6
:10B25800F08F00BFE81D0020F50100202DE9F04F18
:10B26800794E8BB033689D6893F81290122D01D0F7
:10B278000B2D09D1754A122D92F80090A9F13009C9
:10B288005FFA89F915D01DE04BF2E7539D4203D0D0
:10B2980028339D4240F053836D482821F5F7F8F88C
:10B2A8008046002800F04E8301302821F5F7F0F899
:10B2B80048E39F7B37B9674BB846D879FEF7F6FB6A
:10B2C800044615E00027B846FF20FEF7EFFB4BF2D7
:10B2D800D8339D4204460BD14BF2B74006F06AFBC7
:10B2E800C0B2099020B15B4B9B790BB1FDF7D2FB43
:10B2F8003368594D9A68122A1AD19B7BC3B12B78AF
:10B3080013F0010F08D12046FFF7A6FC534B10B1EC
:10B3180001221A7000E018704E4B9B7943B1204609
:10B32800FFF79AFC20B14D4B1B780BB1FDF7B2FB30
:10B338002978DFF844A111F0010100F087819AF81B
:10B348000030DFF838B118460793FDF79BFB079BE1
:10B35800002800F0B5804249002008704148424A60
:10B3680090F800C013609C45404940F089803368DC
:10B378009B8903F00F03032B1ED13D4BACF1300C1E
:10B3880018784FF00A0E05903A480EFB0C00DDF8CD
:10B3980014E000EB0E0C0EF1010E5FFA8EFE704405
:10B3A8009CF8ADC090F8AD00C2F800C083F800E08A
:10B3B800002872D1187070E0082B2CD12C4BACF1FE
:10B3C80030001B7800EB800C0CEB030E294BDFF8E8
:10B3D800A0C013F80E3008930BB98CF800309CF815
:10B3E80000E000EB8000059070440EF1010E5FFA5A
:10B3F8008EFE8CF800E01F4BDDF814C01B5C089033
:10B408000CEB0E00DFF86CE013601EF80030002B28
:10B4180043D1174811E0072B11D1BCF1300F10D1DF
:10B428001348037823B14FF02B0EC2F800E001E077
:10B43800C2F800C0013303F0010303702DE0062BAE
:10B448002BD10B78013327E0F81C0020DC1C0020EE
:10B4580004020020961D0020D71D0020671300203D
:10B468008F570020DA1C0020A01D0020921D00200C
:10B47800061D0020EC6C0208C01C0020DD1C00200A
:10B48800DFF898E203709BF800304FF0010C8EF85B
:10B4980000C013B10B7863440B7040238BF8003065
:10B4A8000B784B4503D39B4B09F1FF301870087894
:10B4B8001168201806F074FA2B7843F004032B70F7
:10B4C8009AF80030232B2FD1924B09F1FF311A78CB
:10B4D8008A4229DA72B932684BF2E75192688A4295
:10B4E80008D028318A4205D02046079306F062FA30
:10B4F800079BC8B118780130C0B21870201806F040
:10B5080059FA28B9834B20211878201806F048FAF0
:10B51800814B40221A702B78804A43F004032B7029
:10B5280000238BF8003013709AF800302A2B10D1C2
:10B53800784B1A786AB1013A1A70774B40221A7020
:10B548002B78764A43F004032B7000238BF80030E5
:10B5580013709AF80030432B1FD16E4B187848456A
:10B5680005D220182021079306F01AFA079B9BF8AA
:10B5780000203AB91B7809F1FF32934202DA654A92
:10B58800013313702B78644A43F004032B700023B3
:10B598001370624A8BF8003013709BF8003013B1B7
:10B5A8005F4A013B13709BF80030012B0ED1594BB9
:10B5B8001A784A4501D201321A70584A002313708A
:10B5C8002A7842F004022A708BF800302B7803F0B6
:10B5D8000402D2B2002A71D0524A6FF38203137068
:10B5E800002111225048F4F7D5FE504A494B1178F2
:10B5F8001B78994288BF137011780F318B4202DD96
:10B608004A490F3B0B70117847481022611806F021
:10B61800E2F94548F5F70EF933684BF2E7519B68B4
:10B62800C2B28B4202D028318B4205D122B94048A0
:10B63800F5F700F9421CD2B20F2A3FD83A48202128
:10B648008018C2F11002F4F7A5FE37E0DFF8D8B091
:10B6580011225846F4F79EFE33684BF2E7529B6876
:10B66800934202D02832934209D1214604222E481F
:10B6780006F0B1F940463946FFF7C6FA1EE0214602
:10B688001022584606F0A7F95846F5F7D3F80246AF
:10B698002021C2F110025844F4F77CFE21464A46A4
:10B6A800244806F098F9244A1020937882F80690E6
:10B6B80043F0020393700146FDF7E0F89AF8003072
:10B6C800532B75D133689A684BF2D8339A4208D114
:10B6D800204606F06FF920B14BF2B740012106F081
:10B6E8005FF93368DFF838A09B68122B40D12046F9
:10B6F800FFF7B2FA8346002830D0104BFF221978A2
:10B708000F4BF9B9009201911B787820013302930D
:10B71800FB3A1FE0921D00208F570020061D0020D5
:10B72800DD1C0020D71D0020741D0020891D00206D
:10B73800751D00200F1D0020081D00206713002024
:10B74800871D00200021009201911B787A20013387
:10B75800029304220B4606F0ABF909E08AF80000D0
:10B768007D492046FFF7A4FA7C4B83F800B0EFE050
:10B7780020464946FDF7D8F8794B00201870336801
:10B788008AF800009B684AF27E72934202D10090C8
:10B79800013005E04BF2FA32934206D101230093BF
:10B7A8000146024603460DF0CFFB6E48FDF754F8FC
:10B7B800FEF772F92B7813F0010F17D033684BF2AC
:10B7C800E7529B68934202D02832934204D1404604
:10B7D8003946FFF719FA09E05F4B634A03F1100194
:10B7E80053F8040B8B4242F8040BF9D133689A687A
:10B7F800122A1ED19B7BE3B12046FFF72DFAC0B178
:10B808002B7813F0010F14D1584B9A7922B9DA79B1
:10B81800574B1B789A420CD0564B1A780023303A73
:10B8280005E055492A20C91801330874DBB2934250
:10B83800F7DB326893680B2B01D0122B0AD14A4BE5
:10B84800991D13F8010B202802D10D3003F8010CC3
:10B858008B42F6D192684BF2D8339A4214D1434BBB
:10B868009B798BB1099878B14FF0000909EB040076
:10B8780006F0A0F818B1404B2A224B441A7409F17B
:10B888000109B9F1100FF1D12B7813F0010F25D070
:10B898003A4B1B7803F08003DBB2FBB133689A683C
:10B8A8004BF2E7539A422D4B03D04BF20F618A4279
:10B8B8000CD11B7833B9B8F1000F0FD05F3388F87B
:10B8C80001300BE057B15F22FA5407E0244A1B7895
:10B8D800127810339B1A284A5F21D154284CA37838
:10B8E80003F00203DBB2002B32D0FCF73DFF204906
:10B8F800034628B908786522E11DFCF753FF12E0DA
:10B908003068B4F90430A27984680978122C01FBF4
:10B91800023105D1807B18B91449C97902FB01317C
:10B92800184806F058F833689B68122B10D1082085
:10B93800134A01460BB0BDE8F04FFCF79FBF002744
:10B94800B84600E0074609F1FF395FFA89F9BBE418
:10B958000BB0BDE8F08F00BF741D0020921D0020C1
:10B96800891D0020081D002004020020961D0020CB
:10B97800871D0020DC1C0020F4010020DC39002099
:10B98800E81D0020EF1D002024282DE9F041144671
:10B9980026D16B4B43F63C321B686A4D9B686A4E56
:10B9A800934206D12B7813F0010F0ED02438674943
:10B9B80009E04BF20F6293420AD12B7813F0010F82
:10B9C80003D063490020FCF7A1FF2978490800E06B
:10B9D8002978301901310222FCF7BEFF0234AAE0AF
:10B9E800E72809D1574B58481978801801310322A4
:10B9F800FCF7B2FF03349EE0A3282AD1514D2B78DF
:10BA08003F2B15D810465349FCF780FF5148F4F7EF
:10BA180011FF2A2124184C48E4B2F4F739FD002814
:10BA280000F08A80297802220131FCF795FF83E033
:10BA38005901494DC918691801F582411046DF318D
:10BA4800FCF764FF05F59240FE30F4F7F3FE241886
:10BA580071E0F22821D13B4F3B4D3978072605EBA1
:10BA68000208B1FBF6F1404601310222FCF774FFEF
:10BA780039782D23B1FBF6F688F80230F3009E1BC7
:10BA88008B1B364FDBB207EB83031988E21CA952E4
:10BA98009B78A818837006344DE025280BD1304BCD
:10BAA80046F695429A8045229A719A78053842F06E
:10BAB80002029A703CE05E280BD1294B46F695525B
:10BAC8009A8045229A719A783E3842F002029A701A
:10BAD8002EE07C280BD1224B46F248129A80112284
:10BAE8009A719A785C3842F002029A7020E0EC2849
:10BAF8000BD11B4B46F6D9529A8045229A719A78F7
:10BB0800CC3842F002029A7012E0A7280BD1144BED
:10BB180046F6F9529A8045229A719A78873842F007
:10BB280002029A7004E0E02801D1541C03E018B125
:10BB3800054B18550134E4B22046BDE8F08100BF3A
:10BB4800F81C0020871D0020F4010020780E03084F
:10BB5800360E0308F2150308F4CB02086DF8020844
:10BB6800E81D002038B50A4B46F68A451B780024A4
:10BB780005FB030507E0074B22461978FFF704FF8A
:10BB8800041B2D190446287808B11F2CF3D938BD99
:10BB9800DB1C0020871D002070B5002543F62064BB
:10BBA800204605F007FF064604F1080005F002FFED
:10BBB80016F0FF0F06D020F07F0010F0FF0F01D025
:10BBC8000135ADB246F23F139C4201D00934E7E794
:10BBD800284670BD38B5B0F900500B4C05EBC505CB
:10BBE80005F578552835284605F0E4FEC1B211F070
:10BBF800800F07D023882846013B01F07F0123806E
:10BC080005F0CEFE208838BDD61C0020454B2DE916
:10BC1800F74F1B88444A044689461788DFF80C8189
:10BC280023B14FF0000A0AE09A4608E00529FBD143
:10BC380098F8003043F0040388F8003070E098F872
:10BC4800003013F0030F0BD013F0010F02D0B4F142
:10BC5800FF3F05D103F00203DBB21BB1012C01D079
:10BC68003F19BFB23BB2B3F1FF3F04D0B3F57A7FBF
:10BC780008BF002701E040F2E7370FFA87FB0BEB1C
:10BC8800CB0303F5785303F12000019305F092FEEE
:10BC980010F0FF0F019B16D0B9F1050F09D103F180
:10BCA800280005F087FE20F07F0010F0FF0FC6D0B7
:10BCB80022E0B9F1000F1FD003F1280005F07AFE49
:10BCC80000F07F0618E00AF1010AB4F1FF3F1FFAFD
:10BCD8008AFA04D198F8003043F0010305E0012CFA
:10BCE80005D198F8003043F0020388F80030BAF51F
:10BCF8007A7F0DD03D46A2E74E4505D0B9F1000F39
:10BD080002D0B9F1050F9AD1BAF1000F05D000E0C1
:10BD18003D46054A2DB2156002E0034BC3F800B05A
:10BD2800BDE8FE8FD61C0020A01D0020A41D002009
:10BD3800F0B503789BB05A1ED2B2792A0F4600F2AA
:10BD4800C8805E01644AF3189B18644A46F68A461E
:10BD58001278457806FB0236E7213046F4F798FB5F
:10BD68000446F0B930467C21F4F792FB0446C0B98A
:10BD780030462521F4F78CFB044690B9304624213F
:10BD8800F4F786FB044660B930464021F4F780FB9F
:10BD9800044630B93046F921F4F77AFB0446002806
:10BDA80076D0A41B0FB14E4800E04E4831462246DB
:10BDB800A619F4F7C5FD3046E721F4F769FB30B161
:10BDC80028466946652246F6D953FCF7EBFC30460F
:10BDD8007C21F4F75DFB50B1691EC9B201EB01117A
:10BDE80001F5C24168464831112205F0F4FD30469C
:10BDF8002521F4F74DFB38B1681EC0B269466522AB
:10BE080046F69543FCF7CEFC3046F921F4F740FBA3
:10BE180038B1681EC0B26946652246F69553FCF7EC
:10BE2800C1FC30464021F4F733FB50B1691EC9B25A
:10BE380001EB011101F5E84168463B31112205F09B
:10BE4800CAFD30462421F4F723FB50B10FB1244832
:10BE580000E02448001929460222FCF77DFD02343F
:10BE68000BE00FB11E4800E01E4800196946F4F7C0
:10BE780083FC6846F4F7DEFC0419002F29D01A4A1F
:10BE88009378141943F0020393700023E37116E0CA
:10BE98003046F4F7CFFC05461FB9124831462A460A
:10BEA80015E0102810DD2A460D483146F4F748FD04
:10BEB8000D4A9378551943F002039370EC711020E2
:10BEC8000146FCF7DBFC04E0084831461022F4F791
:10BED80037FD1BB0F0BD00BFD7FD0208DB1C0020FA
:10BEE800EF1D002052320020E81D0020040200202F
:10BEF8000C4B1B7813F0010202D000200A4905E020
:10BF080003F00200C0B218B108491046FCF7FEBCA5
:10BF180003F00403DBB20BB10549F7E7054801213B
:10BF2800FFF706BFA41D0020B0D302088FD3020874
:10BF3800D1D30208D91D002070B5124D124C002033
:10BF48001249FCF7F3FB2846A1780222FCF704FD0E
:10BF5800E81CE1780222FCF7FFFC05F108002179D2
:10BF68000222FCF7F9FC05F10B0061790222FCF7CB
:10BF7800F3FCA17905F10E000222BDE87040FCF740
:10BF8800EBBC00BFF4010020D91D0020FD6D0208A4
:10BF98002DE9F341504F514C3B689D7C237813F0B9
:10BFA800010F2FD1022243F61E610DF1060005F0A4
:10BFB80012FD4B4EBDF806304FF0FF303360294676
:10BFC800FFF724FE237843F001032370454B1B78C9
:10BFD80013F0030F14D1B6F90010434801EBC10167
:10BFE80001F578512031092205F0F5FC3F4B1B88FB
:10BFF8001BB13046FFF7EEFD10B90020FAF782F8C2
:10C00800FFF79AFF3A4E3378552B0DD1DFF8D480DD
:10C018003848FCF721FC98F800304FF0FF306FF3F8
:10C02800410388F800300DE0442B2BD1DFF8B480B1
:10C038003048FCF711FC98F8003001206FF300033A
:10C0480088F800302946FFF7E1FD98F8003013F032
:10C05800030F15D1224D2448B5F90010092201EB30
:10C06800C10101F57851203105F0B5FC1F4B1B8843
:10C078001BB12846FFF7AEFD10B90020FAF742F8C9
:10C08800FFF75AFFFFF734FF3378232B22D1154BE4
:10C09800184E1A7802F0FC026FF382021A70FCF74D
:10C0A800F9FCB3786FF34103B370134B1D7835B9BE
:10C0B800FCF728FB3046FCF7CFFB3D600AE022780E
:10C0C800013DEDB242F0060222701D700B4B53F891
:10C0D80025303B60BDE8FC81F81C0020D71D0020FE
:10C0E800A01D0020A41D0020D91D0020D61C002062
:10C0F800C01C0020E81D0020B71D0020C41D002022
:10C108002DE9F0411646104A0F4653780E21C3F325
:10C1180042034B43117803F50843CC330B4D01F030
:10C128000701044603EB4101022205F054FCE8191B
:10C1380021780222FCF710FC6178A8190222BDE8D8
:10C14800F041FCF709BC00BF8D1D0020F401002060
:10C15800044B02225978044BC1F3420118180131EB
:10C16800FCF7FABB8D1D0020F401002010B5074B29
:10C17800074C1B78074A03F0070304EB83031C886A
:10C18800111814529B788B7010BD00BF8D1D0020B4
:10C198006DF80208F4010020084B1B789B0902D0B7
:10C1A800012B06D102E01020054904E010200549C2
:10C1B80001E005491020FCF7A9BB00BF8D1D002038
:10C1C80052E0020873E0020894E002082DE9F04109
:10C1D800DFF868800F4698F80010174DC1F3820108
:10C1E8000446164605F1080001310222FCF7B4FBAB
:10C1F80098F80010042201F01C0101F51C41B4312B
:10C20800204605F0E8FBE81921780222FCF7A4FB98
:10C21800F81C281861780222FCF79EFBA819A1785F
:10C228000222FCF799FBF01CE17828180222BDE8ED
:10C23800F041FCF791BB00BFF4010020D91C00209D
:10C24800064B1B7803F08003DBB233B1435C044830
:10C258002021C0180222F4F79DB87047DC3900206D
:10C26800F40100202DE9F743654D664C2B682178D1
:10C278009B68022203EB41010DF1060005F0ABFBC0
:10C288002B68A9469A6843F6F4239A4208D10020FD
:10C298005D49FCF73BFBBDF806804FF4B46303E04F
:10C2A800BDF806804FF46163B8FBF3F103FB118816
:10C2B8003C221FFA88F8B8FBF2F302FB1388CFB2CE
:10C2C800DEB2022251483946FCF746FB5FFA88F88D
:10C2D80002224F483146FCF73FFB02224D484146B7
:10C2E800FCF73AFB4C4B1B7813F0010F6ED04B4B0D
:10C2F8004B4D1878232804D12B78012B62D80133B1
:10C3080005E02A2805D12B78002B5BD0013B2B7048
:10C3180058E0A0F13003DBB2092B01D943284BD1F7
:10C328002B7873B9D9F8003039B29A6843F6F423F8
:10C338009A4201D10A2200E01122FDF7CDFBC7B2D3
:10C3480016E0012B0ED1D9F8003031B29A6843F6C5
:10C35800F4239A4201D1172200E03B22FDF7BCFBEF
:10C36800C6B205E041463B22FDF7B6FB5FFA80F80E
:10C37800D9F800309A6843F6F4239A4209D13C234D
:10C388005E434FF4B46303FB0767B844ADF8068017
:10C3980006E03846314642460FF08DFEADF80600FD
:10C3A800D9F8003020789B680DF1060103EB4000B6
:10C3B800022205F00AFB05E0532803D100232B7065
:10C3C800FDF76AFB17482978FFF73AFFD9F80030DC
:10C3D8009A6843F6F4239A4210D0207812496522CD
:10C3E8000023FCF7DFF905200B21104AFCF746FA79
:10C3F80021780F4801310222FCF7AEFABDE8FE832E
:10C40800F81C0020871D0020771203080402002072
:10C418000A02002012020020D71D0020C01C0020A4
:10C42800921D00200E6E0208EF1D0020E81D00205E
:10C43800F501002073B59A4B9A4D1A7812F0010F46
:10C4480005D12A7812F0380204BF2A706A701A7867
:10C45800934E42F001021A702B78924C13F0380276
:10C468003ED191490978552904D113F0070F2FD0EF
:10C47800DA1D0AE044290CD103F0070201323D39E4
:10C4880092FBF1F1C800411A521A62F302032370B9
:10C498001EE053290AD1C3F3C201013161F3C50378
:10C4A8002370637862F34303637011E023290FD18B
:10C4B800FCF7F0FA33787D4A43F0060333701378BB
:10C4C800013BDBB213707A4A52F82320794B1A6089
:10C4D80000207949FCF71AFA1C20FFF747FEDDE037
:10C4E800082A2ED175490020FCF710FA0620FFF71C
:10C4F8002FFE0C20FFF73AFE1521182201A8FFF79E
:10C50800FFFD694B1B78552B06D1637803F0FE03BA
:10C51800C3F34202013A07E0442B0BD1637803F0DE
:10C52800FE03C3F34202013202F0030262F3430343
:10C538006370B3E0532B28D0232B40F0AF802378CF
:10C54800A6E0102A51D15D490020FCF7DFF906204A
:10C55800FFF7FEFD0C20FFF709FE1521182201A8A0
:10C56800FFF7CEFD6178564801F00101FFF768FE3C
:10C578004D4B1878232801D02A2804D16378DA4350
:10C5880062F30003D4E7532804D12378C3F3C2022B
:10C59800013280E0A0F13003DBB2092B01D9432836
:10C5A8007CD16B7802AA03F001033B21D41883F0F5
:10C5B80001024B43172606FB023214F8041CFDF750
:10C5C8008BFA04F8040C6B780E22C3F3420353432E
:10C5D800287803F50843CC3300F0070003EB40004C
:10C5E80001A90C3A05F0F1F958E0182A4DD1334960
:10C5F8000020FCF78BF90620FFF7AAFD0C20FFF7B7
:10C60800B5FDFFF7C9FD284B1B78552B07D12378BB
:10C6180013F0C00F42D0C3F38112013A06E0442B55
:10C6280007D123789A09012A38DC013262F387138B
:10C6380033E0232B04D12378C3F3C202023A2AE061
:10C64800532B2BD1FCF726FA33781E4A43F0060306
:10C658003370164B1648197840F8212001311970AB
:10C668002378C3F3C201013161F3C503C3F3811118
:10C678002370104B11B1012904D101E01C3202E0F2
:10C68800114A00E0114A1A6008E0114A00211170AD
:10C69800C3F3C202013A62F3C50323707CBD00BF35
:10C6A800D71D00208D1D0020C01C0020B71D0020B4
:10C6B800C41D0020F81C002010E0020831E0020828
:10C6C800116E0208146E02084C6E0208686E0208A9
:10C6D800921D002073B5494B494D1A7812F0010F8D
:10C6E80004D12A7812F0030208BF2A701A78434E40
:10C6F80042F001021A702B78414C13F003022ED13C
:10C70800404A1278552A03D1C3F38202013A04E061
:10C71800442A06D1C3F38202013262F384032370F0
:10C7280017E0532A03D15A1C62F30103F7E7232ABF
:10C738000FD1FCF7AFF93378334A43F0060333706F
:10C748001378013BDBB21370304A52F82320304B88
:10C758001A6001A810211B22FFF738FD4CE0012ABE
:10C768004AD101A810211A32FFF730FD254B18785D
:10C77800232804D12378C3F34112013205E02A2883
:10C7880007D12378C3F34112013A62F346132370A9
:10C798002CE0532804D12378DA1C62F30103F6E76E
:10C7A800A0F13003DBB2092B01D943281ED12B7825
:10C7B80002AAC3F34113D4180C215A1C03F0010335
:10C7C8004B4302F001021F2614F8041C06FB023238
:10C7D800FDF782F904F8040C287801A900F01C0080
:10C7E80000F51C40B430042205F0EFF82978094818
:10C7F800C1F34111FFF724FD7CBD00BFD71D002008
:10C80800D91C0020C01C0020B71D0020C41D00201A
:10C81800F81C0020846E0208064B1B7803F0800386
:10C82800DBB233B1435C04482021C0180322F3F77C
:10C83800B1BD7047DC390020F40100204328F8B569
:10C8480004460D46174606D1104B00261A786FF39A
:10C85800C3021A7000E00E462046FCF713F990B1A7
:10C868000A4B303C1A780A2602F00801C9B200299E
:10C8780018BF002506FB05466FF3C30236B21A70CF
:10C88800BE42A8BF3E4630B2F8BD00BFD71D00204B
:10C898002DE9F3416E4F6F4E3B7843F001033B7037
:10C8A800347844B94BF22F4005F084F86A4B6B4951
:10C8B8001860204617E0012C02D10020684912E0D8
:10C8C800022C02D1002067490DE0032C02D1002080
:10C8D800654908E0042C02D10020644903E0052CD6
:10C8E80003D163490020FCF711F83178D9B9614BBD
:10C8F8001B78312B01D1013101E0302B05D1564B8A
:10C908004BF22F40196005F04BF85B4B1A785B4BE4
:10C9180002F08002D2B20AB1202202E04E4A126826
:10C928003032DA776EE001290BD002290CD00329C6
:10C938000DD004290ED04BF22B45052918BF002530
:10C948000AE04BF21B4507E04BF21F4504E04BF2AF
:10C95800234501E04BF227452946042201A805F0AA
:10C968003AF8474B474A03F1100153F8040B8B423E
:10C9780042F8040BF9D1032243489DF80410FBF751
:10C98800EBFF032241489DF80510FBF7E5FF032262
:10C998003F489DF80610FBF7DFFF3E4803229DF84D
:10C9A8000710FBF7D9FF334B3B4C1878232804D1E9
:10C9B8002378022B22D8013304E02A2804D12378D3
:10C9C800E3B1013B237019E0A0F13003DBB2092B7E
:10C9D80001D9432812D194F8008002AA904418F88B
:10C9E800041CFF22FFF72AFF08F8040C207802AA8B
:10C9F800131813F8041C281804F0D2FF27482178CC
:10CA0800FFF70AFF1B4B1B78532B1FD1224B002229
:10CA18001A7033780133DBB2062B337004D0012B44
:10CA280014D10D4B1B688BB1FDF736F8002333701A
:10CA38003B781B4A43F006033B701378013BDBB29B
:10CA48001370184A52F82320174B1A60BDE8FC816E
:10CA5800D71D0020871D0020A01D0020FD2B0308E6
:10CA6800262D0308472D0308682D0308892D030880
:10CA7800AA2D0308C01C0020DC390020F401002086
:10CA88008C5403080402002005020020090200203B
:10CA98000D02002011020020921D0020886E02085D
:10CAA800B71D0020C41D0020F81C002070B5174CCD
:10CAB8000D460646002120464FF4C172F3F76AFC82
:10CAC800FF2D0AD1B10001F5D84120469531042245
:10CAD80004F081FF23789BB970BDFE2D01D1173E6C
:10CAE80002E0FD2D02D10136267009E0B60006F5F8
:10CAF800D8409530401904F05DFFC0B2207020B1D5
:10CB08000248BDE8704018F0D7BB70BDFC1F00207C
:10CB18002DE9F04118F002FC60B110208F49FBF7B5
:10CB2800F5FE8F4B1B78432B40F0EF81BDE8F041B9
:10CB380018F016BC18F004FC002826D0894C23787D
:10CB48006BB110208849FBF7E1FE88482D21103091
:10CB5800F3F79EFC002800F0D881217810E010201F
:10CB68008349FBF7D3FE81482D211030F3F790FC61
:10CB78000446002800F0C98118F0FAFB0146204657
:10CB88008222BDE8F041FBF7E7BE7A4C43F6CC229F
:10CB980023689B68934250D0774E744D307803EBEE
:10CBA800800004F007FF032201467448FBF7D4FE17
:10CBB8002368986846F6F95398422BD0203B984250
:10CBC80028D03378013000EB830004F0F3FE032211
:10CBD800014605F11500FBF7BFFE236830789B6816
:10CBE800023303EB800004F0E5FE0322014605F161
:10CBF8001900FBF7B1FE236830789B68033303EB19
:10CC0800800004F0D7FE0322014605F11D00FBF762
:10CC1800A3FE0EE02D2103225948F3F7BBFB2D217B
:10CC280003225848F3F7B6FB57482D210322F3F7A0
:10CC3800B1FB20232B772B762B75544B1B7813F0E5
:10CC4800010F00F0BD80236843F6CC229B68444D59
:10CC5800934261D04E4E484F32783878D31803EB60
:10CC6800800004F0A7FE4B4B0146186028789846D0
:10CC7800A0F13002D2B2092A01D943280FD109B252
:10CC8800BA22FCF729FF236832789B680146C8F866
:10CC980000003878D31803EB800004F081FE2B786D
:10CCA8002A2B04D1337813B1394A013B13702B78FE
:10CCB800232B0ED13378022B0BD8226846F6D95194
:10CCC80092688A4205D020318A4202D0304A013324
:10CCD80013702B78552B01D0442B0FD12368317852
:10CCE8009B68A3F5D843B3F1950248BFA3F192021C
:10CCF8003B7803EBA202D0B2FFF7D8FE264B1B7895
:10CD080003F08003DBB23BB13278184B03EB8203AC
:10CD180020225A749A74DA742B78532B06D023681D
:10CD28009A6843F6CC239A4240F0EF80FBF7B2FEB4
:10CD3800236846F695429B68934203D10E4B022026
:10CD4800197806E046F6F952934227D10A4B00209B
:10CD580019780131BDE8F0410CF0CAB82C15030868
:10CD6800C01C00205815002003140308F4010020FB
:10CD78004D150308F81C0020871D0020050200201F
:10CD8800090200200D02002011020020D71D0020FA
:10CD9800921D0020A01D0020DC39002046F6D95243
:10CDA800934204D15A4B012019780918D2E746F664
:10CDB8009552934240F0A980554B03201978C8E753
:10CDC80023684AF27E729B6893423FD1504E1020EE
:10CDD8005049FBF79BFD31784F4D01EB011101F5EF
:10CDE800264101F5BF711022284604F0F4FD2B46B8
:10CDF80005F110012A461078474F78B94749FBF7E3
:10CE080085FD3846E721F3F743FB78B13178401BBD
:10CE1800381801310322FBF79FFD07E013F8010BD7
:10CE280010B9203003F8010C8B42E4D13C4D2B782B
:10CE38002A2B03D13078FD21FFF738FE2B78432BBE
:10CE480063D1307823680130C0B259E043F6CC2270
:10CE58009342334E1AD010203249FBF757FD3378EE
:10CE68002A2B52D1304B1B689B68A3F5D843B3F1EA
:10CE7800950248BFA3F19202254BFF211B7803EBD3
:10CE8800A202D0B2BDE8F041FFF710BE3378204DC2
:10CE9800552B04D12B78142B01D1033B2B703378FD
:10CEA800442B05D12B78122B02D1194B15221A705D
:10CEB8002B78DFF878805901C918414401F594416D
:10CEC80000201F31FBF722FD08F592411020173191
:10CED8002F78FBF71BFD3378112F8CBF0327002712
:10CEE8002A2B05D12878FE21C01BC0B2FFF7DEFD32
:10CEF8003378432B09D12B78173BDF1B2368F8B213
:10CF0800997CBDE8F04118F0F1B9BDE8F08100BFA7
:10CF1800871D00200B150308F40100201BF60208EA
:10CF2800C01C0020C9140308F81C0020F4CB020818
:10CF380010B50E4B1B78452B17D10D4B1A7842F0C4
:10CF480006021A700B4A1378032B0ED80A490B4CA9
:10CF5800086844F823000133137083680B60FBF7FB
:10CF6800DDFBBDE81040FBF795BD10BDC01C0020DF
:10CF7800D71D0020B71D0020F81C0020C41D00206C
:10CF880010B50C4B04462146D8790FF058F860B11B
:10CF9800204655210EF0B2FE48B120460EF044FF5F
:10CFA800D0F1010038BF002010BD022010BD0220C2
:10CFB80010BD00BF961D002008B50FF02FF8C0B2B5
:10CFC80008BD00002DE9F047634B644C1A78994678
:10CFD80012F0010F624D65D02078FFF7D1FF614A4A
:10CFE8002B181178604F93F8A031604E442938709F
:10CFF800336090460AD12D2B08D038B995F8A11185
:10D0080001233B7031602078FFF7D6FF98F8003095
:10D01800552B10D133682D2B0DD03B785BB1013BDC
:10D02800514ADBB21370EB1893F8A0114F4B2078DC
:10D038001960FFF7C1FF98F80030232B19D14C4B2A
:10D0480020781B689B7C013B984212DA434B0130E5
:10D05800C0B21870FFF794FF3870281890F8A03104
:10D068003360444B9B7803F00203DBB20BB1FBF750
:10D0780049FB98F800302A2B14D1207890B1374B0F
:10D088000138C0B21870FFF77BFF3870281890F885
:10D09800A0313360374B9B7803F00203DBB20BB14E
:10D0A800FBF730FB344EFCF7F7FC237832789A42D2
:10D0B80088BF337032780F32934202DD2E4A0F3B1D
:10D0C8001370DFF8C480002730783818C0B2FFF733
:10D0D80057FF281890F8A0310137102F08F8013FA2
:10D0E80007D0254B1A78224BBA181B689B7C9A42AA
:10D0F800EADB99F8003013F0010F13D01F4B1A78B0
:10D108001F4B02F08002D2B22AB122783178103255
:10D11800521A5F2105E0227831781032521A1349E9
:10D1280009689954134DAB7803F00203DBB25BB185
:10D138002078E91D652246F69553FBF733FB052059
:10D148000B212A46FBF79AFB21780E48013102226F
:10D15800BDE8F047FBF700BCD71D0020921D00205A
:10D16800EC6C0208C01C0020D81C0020A01D002068
:10D17800F81C0020E81D0020891D0020DC39002053
:10D18800F4010020F50100200302002038B505460F
:10D1980000240123A3402A78E0B29A4205D10E491F
:10D1A800102246F6D953FBF7FDFA0134042CF0D1CE
:10D1B800043C0A4BE0B2E3189A782B78934206D1E4
:10D1C8002BB10549102246F6F953FBF7EBFA013467
:10D1D800042CEED138BD00BFC21C0020961D0020D3
:10D1E8002DE9F041074610460D461446F3F722FB99
:10D1F800C3B28046B3B1AB4214D80B4E20212A46A5
:10D20800F019F3F7C7F82046F3F714FBC8EB050548
:10D218006D08EDB2EF1902462146F019BDE8F0415C
:10D22800F3F710B8BDE8F081F4010020F0B5154B14
:10D238000C781A1895781F46FDB100233A18927891
:10D248001A4112F0010F4FF001020DD0AC420E78D6
:10D2580003D09A4042EA060604E09A40C2F10F025F
:10D2680002EA06060E7005E09A400E78C2F10F0237
:10D2780032400A700133042BE0D10B7803B90C70EB
:10D28800F0BD00BF961D002031220023017819410E
:10D2980011F0010F02D00449C9188A75013301320F
:10D2A800042BD2B2F2D17047F401002070B57D4B47
:10D2B800044631B11B78532B40F0F280533B037086
:10D2C80070BD1A78302A35D1774A53785BB1774BDD
:10D2D80077491B78182000FB03135B7913F0100FB4
:10D2E80001D001235370734B20781978014013D073
:10D2F8009278002A40F0D4801978114111F0010F7A
:10D3080006D0012191402078C1F10F010140217020
:10D318000132042AF0D143E01A780A4112F0010FD1
:10D3280004D001228A402078024322700131042966
:10D33800F2D135E0A2F13101C9B203293AD85A49EC
:10D348004A785AB1594A5A481278182505FB0202F8
:10D35800527912F0100F01D001224A701B78554AF9
:10D36800313B1278DBB21A4112F0010F00F09880BD
:10D37800227852FA03F010F0010F0BD089780029B7
:10D3880040F08E80013111FA03F3C3F10F0303EA71
:10D39800020204E0012111FA03F343EA02022270B7
:10D3A800002112224448F2F7F5FF2046BDE87040FC
:10D3B800FFF7ECBE132A0CD0552A17D13B4B3C4A39
:10D3C8001B78182101FB03235B7913F0200F03D18D
:10D3D80070BD354B01225A7000202146FFF726FF09
:10D3E800344B9B78002B5BD0002051E0142A0CD0E2
:10D3F8002A2A17D12D4B2E4A1B78182101FB03230B
:10D408005B7913F0200F03D170BD274B01225A70AE
:10D4180001202146FFF70AFF264BDB78002B3FD07F
:10D42800012035E0152A0CD0232A17D11F4B204A9A
:10D438001B78182101FB03235B7913F0200F03D11C
:10D4480070BD194B01225A7002202146FFF7EEFEEB
:10D45800184B1B79002B23D0022019E0162A0CD078
:10D46800442A1DD1114B124A1B78182101FB0323B2
:10D478005B7913F0200F03D170BD0B4B01225A705A
:10D4880003202146FFF7D2FE0A4B5B7943B1032004
:10D498000949102246F6F953BDE87040FBF782B9F6
:10D4A80070BD00BFC01C0020671300208A1D00202B
:10D4B8008A3A0020961D0020C21C00202DE9F04F5A
:10D4C80087B09DF840408146072C0D4605929A4644
:10D4D80037D1073C27462B78234113F0010F2CD076
:10D4E800012623B24FF000080293512031463246FC
:10D4F80033460096CDF8048004F0DAFA1B20414642
:10D50800A2194346CDF80080F5F7F8F837B911208D
:10D5180039463A4633460097F5F7F0F8534B20461C
:10D5280013F8242001276FF3000203F8242011992F
:10D53800F5F76EFF2046F6F769F90134042CCAD1D5
:10D548000DE2012C03780CD10BB90B7823B3FF2320
:10D5580000930021464B01911B780C200133029364
:10D5680016E0022C09D10BB90B78ABB10021FF23CF
:10D5780000930191029134200AE0062C0CD10BB9DA
:10D588000B784BB10021FF23009301910291652094
:10D5980004220B4604F08CFABAF1010F99F8003016
:10D5A8002BD13BB1334B0020D9790246534600902A
:10D5B800F5F7A4F82B783BB12E4B0120D97900223E
:10D5C80003460092F5F79AF80020F5F713FF99F84B
:10D5D8000030002B5BD0284B1978002957D1274BF6
:10D5E800DB78002B53D0FF2300933A2001220B460F
:10D5F8000191029104F05CFA49E063B1052C4FF007
:10D60800000102D100910F2001E000910B200A4691
:10D618000123F5F773F82B7883B1052C4FF000013F
:10D6280006D110200A4601230091F5F767F812E0A9
:10D638000C200A4601230091F5F760F8022C25D04A
:10D64800032C01D10E4B02E0042C02D10D4B1F78A4
:10D658001DE0052C01D10C4BF9E7012C01D1044B3D
:10D66800F5E7062C0CBFFF27002710E09E190020C5
:10D678006B1A0020961D00208C19002067130020CB
:10D68800B01F002067560020E33B0020FF2799F8D1
:10D698000030002B00F0B580934B944E1A789846D2
:10D6A80002F02002D2B262B1317811F0010108D142
:10D6B800FF230093282001220B460191029104F0D8
:10D6C800F7F998F8003003F01003DBB26BB131784A
:10D6D80001F00201C9B241B9FF23009329200122B8
:10D6E8000B460191029104F0E3F998F8033013F026
:10D6F800010F0DD0317801F00401C9B241B9FF23FF
:10D7080000932A2001220B460191029104F0D0F9DE
:10D7180098F8033003F00203DBB26BB1317801F003
:10D728000801C9B241B9FF2300932B2001220B46FF
:10D738000191029104F0BCF998F8033003F0040356
:10D74800DBB26BB1317801F01001C9B241B9FF23E6
:10D7580000932C2001220B460191029104F0A8F9B4
:10D7680098F8033003F00803DBB26BB1317801F0AD
:10D778002001C9B241B9FF2300932D2001220B4695
:10D788000191029104F094F911F0E0F868B1317850
:10D7980001F04001C9B241B9FF2300934920012299
:10D7A8000B460191029104F083F998F8033003F0D5
:10D7B8004003DBB26BB1317801F08001C9B241B9E5
:10D7C800FF2300934E2001220B460191029104F0A1
:10D7D8006FF9767816F0010613D14548314616F0F0
:10D7E800F4FF58B1FF230093731C00211BB202936E
:10D7F800752001220B46019104F05AF90136702E6A
:10D80800EBD1119B3B4A19783B4B51B199F8001069
:10D8180011702A781A702B780BB1542005E0522029
:10D8280003E011702A7853201A7004F00BFD119B45
:10D8380000261A78314B1A7099F80030334113F0EA
:10D84800010F2DD03146059816F0BFFF0122014681
:10D8580028B933B2019000920293104605E00021E6
:10D8680033B200920191029324200B4604F020F970
:10D87800BAF1010F05D1224B8020DA790521013256
:10D8880008E0022C07F1010202D18020072101E003
:10D89800802006213346F6F7F7FA3046F5F78AFF77
:10D8A8002B78334113F0010F55D000214FF0010BB5
:10D8B80033B2029302205A460B46CDF800B00191CC
:10D8C80004F0F6F8DA45DFF83C801DD118F8263068
:10D8D80013EA0B0332D10A4A0520D179009359443F
:10D8E80006EB0B0228E000BFDC3900205D1B00209E
:10D8F8007C190020D6190020D71900207B1B002096
:10D90800961D00209E19002018F8263013F00103F8
:10D9180014D1022C0CD1134B1B7803F02403042BD5
:10D9280004BF114B83F800B000230093072001E0E7
:10D9380000930620791C721CF4F7E0FE119930461A
:10D94800F5F766FD3046F5F761FF18F826306FF3F6
:10D95800000308F826300136042E7FF46DAF07B0B7
:10D96800BDE8F08F841B0020601300202DE9F041F2
:10D9780080460E46174646F2BF75002438462146B3
:10D9880016F023FF88B1294608220B4804F023F833
:10D998000948414616F0C6FE074816F0E9FE20B9C8
:10D9A8000123A34032781343337001340835042C23
:10D9B800E4D1BDE8F08100BF731B00202DE9F043DE
:10D9C80087B08046894604A847F2E911082204F086
:10D9D80002F8002440462146E7B216F0F6FE002879
:10D9E80043D03846F4F7C4FB0025661C024631468E
:10D9F80011202B460095F4F781FE012321462A4683
:10DA08000420FF080095F4F779FE4BF2DF50381830
:10DA180003F0D0FF04F00703C1B2194111F001016E
:10DA28004FF002024FF001030AD00092019336B280
:10DA38007720294692182B46029604F039F814E00C
:10DA48000092019336B2232004220B46029604F07A
:10DA58002FF8B9F1000F08D004A8214616F0B5FE3A
:10DA680018B10548214616F09AFE0134402CB1D170
:10DA780007B0BDE8F08300BFB31900202DE9F74FC8
:10DA8800174698463B7805460C469DF830909DF819
:10DA980034B09DF83820DFF8B8A043B102EA030398
:10DAA8003B7009789AF800208A18D31A03702378F3
:10DAB80083B122482146F5F755FE21491F4816F043
:10DAC80031FE1E480121FFF779FF1C4841462246D6
:10DAD800FFF74CFF1B4B00261E70297843F6FB20EE
:10DAE80003F05EFF494646F2CD6003F059FF204639
:10DAF80039464A46F5F734FC134B42461E713946FF
:10DB08004B462046CDF800B00195FFF7D7FC2846D4
:10DB1800F8F730FB2B780D480D498AF80030F5F7F7
:10DB280021FE11F053FF88F800603E7026702E70B9
:10DB380003B0BDE8F04F04F08FBA00BF7C1B002093
:10DB4800CE190020D41D0020671300205F1B002081
:10DB58008C19002010B50B4B0B4C024603CB2060F0
:10DB680061600A48114616F0FEFD2146074816F086
:10DB7800D9FD064816F0FCFDD0F1010038BF0020A1
:10DB880010BD00BFB02D0020691B0020731B0020B2
:10DB980010B50A4C637C4BB100200949FAF7B6FE70
:10DBA800084B1B78432B01D1433B6374607C20B93D
:10DBB8000549BDE81040FAF7A9BE10BDC21C0020F7
:10DBC8005DF60208C01C00203CF60208034B1A78D8
:10DBD80001321A7001230370704700BFD41D002062
:10DBE80010B50C48FAF738FE0B4A002414700B4A9B
:10DBF8000B4B14700B4A5C7114700B4A1C71147037
:10DC08000A4A5C7014700A4A1470FAF743FF094B09
:10DC18001C6010BDE81D0020961D0020C11C0020BE
:10DC280067130020D81D0020E51D0020FC1C0020E3
:10DC3800D41D0020F81C00202DE9F04F9B4B9C4F71
:10DC480093F800903B68DFF8BC829C7C994BF022EB
:10DC58001A7098F800308BB00D2B3D46464643D1DC
:10DC6800202195486FF02F02F2F794FB934B93F81D
:10DC780005C0BCF1010F02D9002091492FE01AD14B
:10DC880000245C718F4A904B90499148914D0470E3
:10DC98001C7014700C70CDF800C001942D7802959A
:10DCA800FFF7ECFEFAF7F6FE8B483C600BB0BDE8D8
:10DCB800F04FFAF7D1BD89488449F5F753FD884BF1
:10DCC800884A03CB884B10601B785160532B5FD177
:10DCD80098F800308549013388F8003000200BB0EF
:10DCE800BDE8F04FFAF712BE092B0FD17E4B1B7817
:10DCF800532B3DD17E4B00221A700D2388F800303B
:10DD08007C4B1A7842F006021A7089E20E2B37D142
:10DD1800754B1B78532B2BD17749704816F002FDB1
:10DD28006E48FFF717FF044640B198F80030052207
:10DD3800013B88F80030614B5A7171E2082246F2C3
:10DD4800CE61684803F047FE66496C4816F00BFD43
:10DD5800012300935F4B01941B785D4802935B4954
:10DD6800584A594BFFF78AFEFAF794FE3C6057E28F
:10DD7800232B40F055820BB0BDE8F04FFFF730BFC2
:10DD880033B95F4B1A781AB901321A7011F01EFEB6
:10DD9800631E48BFA31DDB10013303FB09F91FFAFB
:10DDA80089F909F5CC47A9F59449A9F12109514BFD
:10DDB800CDF81C901A78CE3712F0010F4C4C00F0B9
:10DDC8002381494B1A789946432A40F0CC8033780E
:10DDD8000D2B40F0C8804148217816F0F6FC002849
:10DDE80000F0C1803F48217816F0EFFC002840F091
:10DDF800BA80079920780FFA81FB0BEBD00003F06B
:10DE0800D9FD23784FF0010A03F007020AFA02FA53
:10DE1800DFF8F4805FFA8AFA10EA0A0FC8F80000FF
:10DE280027D0264BDB78002B40F09D80294BD879F2
:10DE3800F8F7FEF8002800F09680D8F80010CAF12C
:10DE4800FF0A20780AEA0101C8F800100BEBD0009D
:10DE580003F0A6FD20780FFA87FB0BEBD00003F048
:10DE6800A9FD00EA0A012078C8F800100BEBD000E1
:10DE780064E00FFA87FC0CEBD300CDF814C003F074
:10DE880099FD10EA0A0FC8F800003FD140EA0A01DC
:10DE9800059A2078C8F8001002EBD00003F080FD46
:10DEA8002178164816F07BFC5DE000BF871D002036
:10DEB800F81C0020E31D0020040200206713002046
:10DEC80002F70208D81D0020C11C0020E51D002013
:10DED800FC1C0020961D0020E81D00207C1B002053
:10DEE800B02D002074190020C01C0020C8F70208BB
:10DEF800921D0020D71D0020C3190020CE19002034
:10DF080028140020D41D0020A01D0020914BDB7890
:10DF180023B9914BD879F8F78BF8B0B9059B2078DD
:10DF2800CAF1FF0A03EBD00003F044FD8B4A00EA74
:10DF38000A01059B2078116003EBD00003F030FD47
:10DF48002178874816F036FC0DE020780BEBD000DE
:10DF580003F030FD40EA0A012078C8F800100BEB06
:10DF6800D00003F01DFD99F80030232B10D12A684A
:10DF78002378927C013A93420ADA7A4A0133137081
:10DF8800794B9B7803F00203DBB20BB1FAF7BAFBCB
:10DF980099F800302A2B0CD1237853B1714A013BF0
:10DFA8001370714B9B7803F00203DBB20BB1FAF7E5
:10DFB800A9FB99F80030552B12D129682278897C61
:10DFC800684B08398A4201DA083200E000221A70E8
:10DFD800654B9B7803F00203DBB20BB1FAF792FBB7
:10DFE80099F80030442B0FD122785E4B072A9CBF4A
:10DFF8002A68927C083A1A705B4B9B7803F00203FC
:10E00800DBB20BB1FAF77EFBFBF746FD574A2378E4
:10E0180011789246994288BF137012780F32934252
:10E0280002DD524A0F3B13702B684FF0000B93F838
:10E038001280CDF818B0B8F10F0F9ABFC8F12008B8
:10E048005FFA88F84FF0100831784FFA8BF30D29F2
:10E0580005D19AF800209B18DB10454A04E09AF88D
:10E0680000209B18434ADB10D35C9AF800200593E4
:10E078004FFA8BF39A180D2902F007094FEAE202CA
:10E0880002D13D49895C0691DDF81CC004930FFA62
:10E098008CF0101803F08EFCC0B2049B08909AF81C
:10E0A80000003AB2181802EBE00003F083FC327863
:10E0B800049B09929AF80020C0B29A1846E0059B82
:10E0C800DDF824C043FA09F12C4B01F001010029C5
:10E0D8000CBFA521DB21BCF10D0F03F8081014D1EA
:10E0E80027494FEAE20C11F80C1041FA09F111F036
:10E0F800010F08D0DDF818C04CFA09F111F0010F32
:10E1080003D0582110E02D210EE0DDF820C04CFA94
:10E1180009F111F0010F01D0502105E040FA09F191
:10E1280011F0010F02D0542103F8081009F1010978
:10E138005FFA89F90BF1010B08F101080132B9F115
:10E14800080F5FFA8BFB5FFA88F81BD0B8F1200F35
:10E15800B5D124E067130020961D0020A01D0020E3
:10E16800CE190020921D0020E81D0020891D0020E6
:10E17800C3190020231A002074190020F40100207C
:10E188007C1B0020B8F1200F09D09AF800304FFA14
:10E198008BF2D2182B689B7C9A42FFF655AF224926
:10E1A8000B7813F0010F17D02B68204A9B7C12784C
:10E1B8000F2B02F0800298BFC3F11003D2B294BFB4
:10E1C800DBB2002342B122789AF800101032521ABA
:10E1D8001749CB185F219954164EB37803F0020300
:10E1E800DBB25BB12078F11D652246F69543FAF75C
:10E1F800D9FA05200B213246FAF740FB2B689B7CA5
:10E208000B2B0DD9B37803F00203DBB243B12178AD
:10E218000948013102220BB0BDE8F04FFAF79CBB68
:10E228000BB0BDE8F08F00BFD71D0020DC390020FF
:10E23800F4010020E81D0020F50100202DE9F0433D
:10E24800002387B08DF817307C4B1B78012B00F02A
:10E2580070827B4B1A78984672B17A4BDB78002B28
:10E2680040F06782784C2378002B40F0B580FAF7AD
:10E2780011FC09232370AFE0734B19781C46082959
:10E2880000F2AA8071490978232913D11A70FAF784
:10E2980001FC6F496F4A0B7853B16F48013B047812
:10E2A800DBB244F0060404700B706C4951F823305B
:10E2B8001360AFE2684B1A7812F0010F04D1012104
:10E2C8000A438DF817101A70F4F74CFE28B9237812
:10E2D8001BB90DF11700FFF779FCF4F751FE30B9BF
:10E2E8002378012B03D10DF11700FFF76FFCF4F72A
:10E2F80055FE30B92378022B03D10DF11700FFF733
:10E3080065FCF4F757FE30B92378032B03D10DF1E0
:10E318001700FFF75BFCF4F75BFE48B9F4F784FEDF
:10E3280030B92378042B03D10DF11700FFF74EFC09
:10E33800F4F7AEFE30B92378052B03D10DF11700A1
:10E34800FFF744FCF4F798FE30B92378062B03D185
:10E358000DF11700FFF73AFCF4F748FE30B92378BF
:10E36800072B03D10DF11700FFF730FCF4F74CFE33
:10E3780030B92378082B03D10DF11700FFF726FCDD
:10E388009DF8173043B32378082B23D8DFE803F030
:10E3980005080D101316191C1F000020304901E054
:10E3A80030490020FAF7B2FA16E000202E49F9E7C2
:10E3B80000202E49F6E700202D49F3E700202D49DB
:10E3C800F0E700202C49EDE700202C49EAE700207F
:10E3D8002B49E7E7FAF75EFB1B4F3B783D46092BD5
:10E3E80040F0B2801C4E194F317811F0010153D121
:10E3F800244C12222046F1F7CDFF01236374224AF0
:10E4080098F80030137003B96374637C13B11F4B21
:10E4180000221A70FFF7BCFB1B48617CFEF746FF21
:10E42800337803F0FD0343F001033370184B1A7877
:10E4380082B33A7000221A702EE000BFE31D00205C
:10E448008C19002067130020D41D0020C01C002058
:10E45800B71D0020F81C0020D71D0020C41D002077
:10E46800AEFC02088DFC0208CFFC0208F0FC020892
:10E4780011FD020832FD020853FD020874FD02086E
:10E4880095FD0208C21C0020FC1C0020601300201F
:10E498008C1D002030233B703B78884E13B973786D
:10E4A800102B4DD1DFF86492854CFFF771FB84483F
:10E4B80099F81110FEF7FAFE237823B100201021F5
:10E4C8004A46FEF78DFE98F8003024787D4A24EA03
:10E4D800030111707C4A23EA040111703A78A2F111
:10E4E8005200C0B2012803D97078744F10280CD19B
:10E4F800002373701CB911B10133009311E1042397
:10E5080073712B7801332B701AE0432A18D1BBB9E9
:10E51800FC78ACB96D4BD879F7F78AFD38B96C49F6
:10E52800FAF7F4F905237B7108332B7004E02046D1
:10E538006849FAF7EBF97C71674A684B1A6069E138
:10E548005F48FEF7A1FE65E10A2B31D15D4809F06D
:10E55800BDFCC6B2594C36B36379042B02D10020F6
:10E568005F4903E0022B04D15E490020FAF7CEF997
:10E5780002E00BB904336371314602225A48FAF7B4
:10E58800EBF95A4B1E78232E00F0D3803046FAF769
:10E5980079FA002800F03E81312E40F03B812B783B
:10E5A80001332B7002E03B7801333B70042332E0E7
:10E5B8000B2B32D1434809F06FFCC6B23F4C36B33F
:10E5C8006379042B02D10020494903E0022B04D1CE
:10E5D80048490020FAF79AF902E00BB9043363714D
:10E5E800314602224048FAF7B7F9404B1E78232EED
:10E5F80000F09F803046FAF745FA002800F00A81BB
:10E60800312E40F007812B7801332B7002E03B78E4
:10E6180001333B7008236371FCE00C2B40F0FA8057
:10E62800284809F01FFC0021C4B2264809F0F0FB75
:10E63800002C6DD0214E33792BB9BE2016F0B2FED6
:10E6480033790133337173791C4A092B02D90020BD
:10E658001F4915E010D11D4B00241C705471264B26
:10E66800194A1849164801251C7014700C7004705A
:10E678000095019402949EE0082B04D11F490020C4
:10E68800FAF744F911E0062B02D100201C49F7E7FC
:10E69800042B02D100201B49F2E7022B02D10020F3
:10E6A8001949EDE70BB9083353717379082B3CD836
:10E6B8000D4821460222FAF74FF936E06713002089
:10E6C800FC1C0020E51D0020D81D0020961D002000
:10E6D80002F702087EF60208906E0208F81C002075
:10E6E80086F70208A7F70208F4010020C01C0020E2
:10E6F80044F7020865F70208C11C00209FF60208CB
:10E70800C0F60208E1F6020823F70208C21C00203E
:10E71800012542484249434A2B460095F5F7D4F96A
:10E728000095414B01941B7840E0404F3C78232CE6
:10E7380002D1FFF755FA6DE02046FAF7A3F9002851
:10E7480068D0303CE4B2631EDBB2012B3C7039D890
:10E75800022C354D1ED1E879F7F76AFC002838D02D
:10E768002E48FFF7F7F9002833D1082246F2CE6188
:10E778002F4803F030F929492D4815F0DEFF2C49C0
:10E78800082246F2CE6003F020F92949294815F0FD
:10E79800EAFF06E0012321482149224A0093F5F7C0
:10E7A80093F901230024009301942B7802932248C3
:10E7B8001C49224A1A4BFFF761F9FAF76BF9204B0B
:10E7C8001C6027E0032C25D1174BD879F7F730FCCC
:10E7D80010B90C2373711DE000241048214615F070
:10E7E800F4FF28B1E02016F0DDFD204616F016FEF5
:10E7F8000134402CF1D1134A0023137073712B7824
:10E80800114A01332B700E4B1A60104B1A7842F0E4
:10E8180006021A7007B0BDE8F08300BF7C1B002019
:10E82800C11C0020E51D0020961D0020C01C0020F2
:10E8380074190020CE190020FC1C0020D81D0020CF
:10E84800F81C0020921D0020906E0208D71D0020A1
:10E8580088234B43054A03EBD003D35C00F0070041
:10E8680053FA00F000F00100704700BF840D00204B
:10E8780070B504461646157839B912E00135EDB27F
:10E8880028462146FFF7E4FF48B9202DF6D970BD88
:10E89800013DEDB228462146FFF7DAFF08B13560A1
:10E8A80070BD002DF4D170BD064B38211B780322B2
:10E8B80001FB0031044844230370C9B2173BC370FD
:10E8C800FAF74AB8921D0020F4010020012802D06E
:10E8D800022806D102E01D20044904E01D20044955
:10E8E80001E004491D20FAF711B800BFA9EF02089A
:10E8F80088EF0208CAEF0208037809680F4A03EB99
:10E908000310401802EBC00050F8240C0C49884250
:10E918000FD1882101FB03239A68A0F59C63063B6D
:10E928009A4208D0A0F598600538101A18BF01203F
:10E938007047002070470020704700BF840D0020FA
:10E9480067EF020803780A6803EB0313D318084A31
:10E95800053B02EBC3035968064A914205D1187A70
:10E9680009288CBF0020012070470020704700BF95
:10E97800840D002067EF02082DE9F04F984B994F5E
:10E98800F0221A703B6889B09C6847F2F373E11A69
:10E998004C4244EB0104DD3A6243934B9D5C03EB2C
:10E9A8000208C5F30005EEB23A46002E2CD13046D7
:10E9B8008E49F9F7ABFF8E4B1B78232B41F02A8247
:10E9C80098F8013066F3041388F80130FAF762F812
:10E9D800884B1A7842F006021A70874A1378013B6E
:10E9E800DBB21370854A52F823303B60844B1D70AC
:10E9F800844B1D70844B1D70844B1E60844B1D70AE
:10EA0800844B1D7001F006BA814D95F80090B9F15C
:10EA1800000F0CD04FF43661614309F1FF30342305
:10EA280003FB00137C49CB181B798DF81F307B4BF7
:10EA38001E787EB17A4E2046317810F06BFE0028A1
:10EA480040F05C8475493070087007460646804679
:10EA580000F05BBC6D490B688B46A3F112000328DC
:10EA680009D9A3F11601032909D9A3F11A01032928
:10EA780009D9374605E037464FF0010805E0374623
:10EA88000126B84601E00127B046594909785329BB
:10EA980040F0D581B9F1000F3AD172226243614941
:10EAA800885C10F0020F0AD0002B41F0B3810133CB
:10EAB80063F383008854CBF8003001F0ABB95A4BAC
:10EAC800997989B120464A4610F00CFEFF2801F0DA
:10EAD800A18101302870CBF80090F9F7DBFF2046C0
:10EAE800FFF7E2FE01F096B9DFF8FCC0132202FB43
:10EAF80004C25178204669F3041151704B4A02212F
:10EB080082F80090039310F093FD0122039BCDE25D
:10EB180009F1FF312046C9B210F0FCFD002840F091
:10EB28008B80DFF810B1DFF8EC909BF80020012310
:10EB380032B98BF80030324B89F800201A70E4E3C0
:10EB480005900393F9F7A6FF05988BF80000039B3F
:10EB580089F80030364A835C9246A3F13001C9B285
:10EB6800092904D9413BDBB2052B01F2538101305D
:10EB78000A28EFD14FF0000847460AEB480015F085
:10EB880059FE7B080237FFB20A2F294E0AF8030004
:10EB980008F10108F1D1304611F0A8FA002801F077
:10EBA8003981304611F010F80746002841F03281CB
:10EBB8001D4B3046997911F0A8FA002801F02A81F6
:10EBC8002978337901392046C9B202220097019683
:10EBD80011F0EEFA022389F8003001F01BB900BFEA
:10EBE800E31D0020F81C0020E6390020F7E00208A9
:10EBF800C01C0020D71D0020B71D0020C41D002008
:10EC0800DD1C0020061D0020871D0020A01D0020FF
:10EC1800921D0020891D0020503D0020D41C00209A
:10EC2800881D00201054002067130020D61D0020E6
:10EC3800B81D0020931D0020DBF80030DFF8089392
:10EC4800202B27D0212B23D14FF436626243297819
:10EC58003420013900FB0122AC489DF81F301218FE
:10EC68004FF0000B20460192C9B20322CDF800B044
:10EC780011F09EFAF9F70EFF2A78A54B013AA5483C
:10EC88001A701423C9F800B085F800B003703CE38B
:10EC98001E2B03D10133C9F8003019E31F2B18D1FB
:10ECA8004FF43662624329783420013900FB01228F
:10ECB80096484FF0000B121801929DF81F3020461D
:10ECC800C9B20622CDF800B011F072FAC9F800B046
:10ECD800FEE29A1F062A0ED88F4B1A7819462AB9CF
:10ECE80001321A708D4B1A788D4B00E3012A40F0DF
:10ECF8000C830223A1E1A3F10D02042A3AD8894921
:10ED0800D3B291F800C095F800E08048864ABCF17B
:10ED1800000F1ED04FF0000C81F800C011784FF49E
:10ED2800366262430EF1FF3E0CF1340C0CFB0E22EE
:10ED38008018C0184174382000FB04EE5FFA8EF08A
:10ED480000EB800000F5F8401B30C01802F028FEE8
:10ED5800DBE24FF0010C81F800C04FF436616143EB
:10ED68000EF1FF3E0CF1330C0CFB0E1E7044C31861
:10ED78005B7C59E0A3F112020B2A4CD86B4A297824
:10ED88001078002845D000201070A3F1120938220D
:10ED98004B1E02FB0433203ADBB2534303F5FC431A
:10EDA8005FFA89F9DFF894B14B3303EB49039BF819
:10EDB80000101846039302F0F3FD5D4A4FF4B66C59
:10EDC8000CFB04FC11781A22013902FB01C14F48DF
:10EDD800494400EB41019BF80000DFF870B18875E9
:10EDE800039B9BF80010581C0492CDF814C002F045
:10EDF800D7FD4F49049A0B78DDF814C0013B02FB9C
:10EE080003C2424B4A4403EB42029BF80030D375DD
:10EE18007BE2012308E0DFF8209199F800302BB954
:10EE2800012289F80020434A13706EE2F9F732FE96
:10EE3800002389F800302046FFF736FD65E24329B4
:10EE48004BD1354A1278002A40F05F82354A127851
:10EE5800002A40F05A82B9F1000F00F05682364A73
:10EE68001278002A40F05182212B30D01F2B30D04D
:10EE78002E4B1978012919D9B8F1000F02D1002FAA
:10EE880000F043822D4B02391A7852FA01F010F043
:10EE9800010F4FF0010004D010FA01F122EA01023B
:10EEA80025E210FA01F141EA020220E200F02D8287
:10EEB80009F1FF312046C9B210F02CFC20B9204BD3
:10EEC8001B78002B40F0218200232B7000E22023C6
:10EED80000E01E23CBF80030FAE1232940F09680A9
:10EEE8000D4B1B78002B40F010820E4B197800292F
:10EEF80040F00B82104BB9F1000F50D01A783AB39A
:10EF08000C480F2A01700F48017042E1503D002063
:10EF1800881D0020D41C0020D61D0020861D00203E
:10EF2800E41D00209F1D0020541E00208B1D002082
:10EF3800921D0020DD1C0020871D0020851D00205B
:10EF4800931D0020061D0020A01D0020D51D0020B7
:10EF580009F1FF312046C9B210F0DCFBB0B19A4A82
:10EF680013787BB1B8F1000F01D0042B08D90EB18A
:10EF7800012B05D9002F00F0C881042B00F2C281B3
:10EF8800013351E79DF81F000121F6E08F4B1A78F5
:10EF9800511EC9B208296FD801321A706CE0DFF827
:10EFA8006CC2132101FB04C1487869F3041048704E
:10EFB800022120460492039310F03AFB08F034FE35
:10EFC800F9F768FD8249087840F006000870814822
:10EFD80001780139C9B201707F48049A50F82110AC
:10EFE80011607E4A82F800907D4A82F80090039B67
:10EFF800CBF8009083F800907A4B85F8009083F85E
:10F008000690794B83F8009000F004BF2A2936D186
:10F01800764B1B78002B40F07881754B1A78002AC4
:10F0280040F0738173490B784BB16C48012B027027
:10F038006B48027040F26981013B0B7065E1B9F1E0
:10F04800000F00F0628109F1FF312046C9B210F0CB
:10F0580061FB58B15C4A137823B1012B40F255810A
:10F06800013BE1E69DF81F00002186E0574A13782E
:10F07800012B01D9013B13700022584B37E1442979
:10F0880040F08D80594A1278002A40F03E81B9F14B
:10F09800000F0DD1534B9A79511EC9B2012901D8DD
:10F0A800013203E0032A40F03081023A9A712CE1E0
:10F0B800504A1278002A40F02881444A1278002ADF
:10F0C80040F023814A4A1278002A58D13E4B1B78D7
:10F0D800012B09D9002E00F01881474B1A78072A0E
:10F0E80000F212810132AAE019D1B8F1000F0BD059
:10F0F800424A032011789846013191FBF0F000EB69
:10F108004000091A117000E1002E00F0FE803B4A11
:10F118001E461178013101F003011170F5E0314B01
:10F12800204699794A4610F0DDFAFF2800F0ED8074
:10F13800DBF80030212B00F0E8801F2B00F0E58081
:10F14800013028702046FFF7AFFB4FF43662624368
:10F1580029783423013903FB0123294A9BF800004D
:10F16800D31893F8049049468DF81F90FFF770FB69
:10F178000146002840F0AC804846224AA6E00D2B04
:10F188000BD19DF81F0010F077F930B11E4B1A789B
:10F198001F2A00F2BA800132A9E00120AAE055290D
:10F1A80040F0B380114A1278002A40F0AE80B9F1DD
:10F1B800000F2DD10B4B9A79012A01D9013A75E735
:10F1C80040F0A380032271E78B1D0020931D0020CF
:10F1D800D71D0020B71D0020C41D0020DD1C002005
:10F1E800061D002067130020891D0020D61D002061
:10F1F8009F1D0020871D0020851D0020D51D002093
:10F20800503D0020A01D0020541E0020E63900209B
:10F21800894A1278002A78D1884A1278002A74D14B
:10F22800874A1278002A56D1864B1A78012A08D9BB
:10F23800002E6AD0844B1A78012A65D9013A1A70CF
:10F2480062E012D1814B197811B1013919705CE073
:10F25800B8F1000F03D002211970904655E0002E36
:10F2680053D00321197016464FE0B9F1010F4CD95C
:10F27800774BA9F1020220469979D2B210F040FAF0
:10F28800FF2842D0DBF80030DFF8D091212B3CD0AA
:10F298001F2B3AD0013028702046FFF705FB4FF4AA
:10F2A8003662624329783423013903FB0123694A12
:10F2B80099F80000D31893F804B059468DF81FB098
:10F2C800FFF7C6FA014618B958464A46FFF7D0FA7A
:10F2D800F9F7E0FB19E00D2B0BD19DF81F0010F09A
:10F2E800CBF830B15C4B1A78012A0ED9013A1A7062
:10F2F8000BE0FF2058490FF0DDFF06E000273E46EF
:10F30800B84602E0012700E001262978DFF8989145
:10F31800002940F0CB8099F8003013F0010205D1A4
:10F3280043F0010389F800304C4B1A600025204651
:10F33800294610F06FFC30B172236343484AD15C10
:10F3480041F00201D1540135382DF0D13A356543E9
:10F35800434E735D13F0020F43F3400015D03F4C4A
:10F36800206810B93F4900F0C1BC00203E49F9F7B8
:10F37800CDFA735D13F00C0F43F3810540F04A8515
:10F38800F9F788FB256000F045BD314DAB79A3B195
:10F39800012B01D1354906E0022B01D1344902E0A5
:10F3A800032B02D13349F9F7B1FAA979204610F0B5
:10F3B800E3F9022201463048EDE114B920462F490D
:10F3C80001E02F491846F9F7A1FA2E4803786BB9DE
:10F3D8002D490A222D48F1F7B3FA2D49132303FBCF
:10F3E80004135A7842F010025A7004E02748294959
:10F3F8000A22F1F7A5FA284D3821022205F11E004C
:10F40800F9F7AAFA204610F0DBF90222014605F1C5
:10F418001900F9F7A1FA214B00221A70204B1B782A
:10F4280003F08003DBB2002B00F0F4841D4B1B8833
:10F43800EB8100F0EFBC00BF871D0020931D00206A
:10F448009F1D00208B1D0020851D0020D51D00203C
:10F4580067130020503D0020541E0020A01D0020EE
:10F468001054002039E102085AE1020862E2020859
:10F4780083E20208A4E20208120200209CE10208CA
:10F4880020E20208D41C0020C5E20208FA0100208C
:10F49800E6390020E6E20208F4010020891D002078
:10F4A800DC39002099540308D71D00200139204673
:10F4B800C9B210F02FF9002800F0F483954B93F8A7
:10F4C80000B038230BF1FF3B03FB04BB99F8003075
:10F4D8005FFA8BFB13F0010F03D08F4A1378002BD0
:10F4E80041D08E48F9F7B8F90BEB0B1101F5E8415B
:10F4F80010228B483B3102F06EFA884B11229A7128
:10F50800884B1B6813B91020874921E0012B02D1D1
:10F51800102086491CE0022B02D11020844917E0F4
:10F52800052B02D11020834912E01E2B02D1102096
:10F5380081490DE01F2B02D11020804908E0202BC3
:10F5480002D110207E4903E0212B03D17D491020F0
:10F55800F9F7DCF999F800306F4843F0010389F8AE
:10F56800003000230370784B1A78002A00F0AB8033
:10F578000BEB0B1B0BF5E84909F13B09102273480B
:10F58800494602F028FA00229346704B995C41B133
:10F598000BF1010B5FFA8BFB0132BBF1100FF4D1B9
:10F5A80007E06A49C2F1100201EB0B002021F0F7D5
:10F5B800F1FE654A107858450BD90138484402F0E5
:10F5C800F9F930B9604B202118780138484402F025
:10F5D800E7F9DFF894B19BF8003018460393F9F780
:10F5E80051FADC46039BDFF878B110B9432B44D1BC
:10F5F80001E0432B05D100238BF800304FF0200A9F
:10F6080030E05348534A90F800E053499E450ED1E4
:10F61800AEF1300E0A20137800FB0E1E0133DBB268
:10F628001370734493F8AD307BB913700DE0037019
:10F638009BF800304FF0000E82F800E02BB14248F2
:10F6480003780F2B01D80133037040238BF8003067
:10F6580013789CF800200A20303A00FB0211C918E0
:10F6680091F8ADA03849394A08785146013802F86E
:10F6780000A0484402F094F90FE0384B1B7803F0DF
:10F688008003DBB24BB19BF8003033B92E482F49C9
:10F698000378FF22CB1803F8012C9BF8003013B134
:10F6A8002F4A013B13709BF80030012B10D1264ADA
:10F6B80013780F2B01D801331370264A00238BF8D7
:10F6C8000030137004E004200C21144AF9F7D6F82E
:10F6D800144A13689346002B48D14FF436626243AC
:10F6E80029783424013904FB01241E4AA4186178BE
:10F6F800164AC1F3C30109B93F2004E0994201D970
:10F70800DB2000E0A5200133DBB2907501320A2B23
:10F71800F1D17FE3921D0020891D0020E81D002003
:10F72800EF1D0020A01D0020E3EE0208CDE3020833
:10F738000FE40208D5E402087AE502089BE502080E
:10F74800BCE50208DDE50208871D0020F401002061
:10F75800DA1C0020061D0020EC6C0208DC390020B1
:10F76800DD1C0020583D0020C01C0020012B15D1B5
:10F778004FF4366363432A783424013A04FB023495
:10F78800AB4BE418637813F0070300F043831421AC
:10F798005943A8488322F9F7DFF83BE3022B26D127
:10F7A800A54A9DF81F30882101FB03232978A34A25
:10F7B800D87901390623202502F8015950FA03F5B2
:10F7C80015F0010F10D04FF436656543342606FB5B
:10F7D80001559B4E7519ED791D4115F0010F01D0AA
:10F7E800DB2500E0A5255570013BE4D212E3032B8D
:10F7F80013D14FF4366363432A783424013A04FB67
:10F8080002348F4B1C19237A13F0010F02D01020F9
:10F818008C496BE210208C4968E2042B13D14FF419
:10F82800366363432A783424013A04FB0234844B58
:10F838001C19237A13F0020F02D01020834955E2D5
:10F848001020834952E2052B15D1162700262B7864
:10F858003422013B53434FF4366202FB0433784AA7
:10F868007C49D318985DC919013614F0C9FF0237CD
:10F87800052EECD1CEE2991F062900F2FF809DF8F3
:10F888001F206D4F02EB0210411807EBC101C96838
:10F89800714801F1100651F804CBB14240F804CB8D
:10F8A800F9D19E1FF6B202EB02129219013207EB50
:10F8B800C202507A92F80AC0684A297813789046AA
:10F8C80073B94FF4366363433422013902FB0131C3
:10F8D800634BCA5E634B024102EA0C021A7011E0E4
:10F8E800022B0FD1604B01391B784FF000090093B0
:10F8F8002046C9B204223346CDF8049010F058FCD3
:10F9080088F8009098F80030012B29D1574BDFF880
:10F91800589193F800A05046F9F7B4F810B9BAF125
:10F92800430F1AD10DF11F005149FFF70BF810B121
:10F93800002389F800309DF81F30DBF8002003EB26
:10F9480003139B1807EBC303504699F8001013F8EC
:10F95800202CFAF7C1F889F8000099F800A003E014
:10F9680013B9404B93F800A0BAF1090F07D9BAF1BF
:10F97800630F8CBF4FF003094FF0020901E04FF00D
:10F9880001099DF81F3003EB03139E1907EBC60707
:10F99800FB685A7BE02A02D12E4A202151779A7BB4
:10F9A800E02A02D12B4A20219177DA7BE02A02D182
:10F9B800284A2021D17798F800200ABB4FF43662F4
:10F9C800624329783424013904FB0124184AA41815
:10F9D800A27812F0080F1BD05A7BE02A02D11D4AE8
:10F9E8003F2151779A7BE02A02D11A4A3F21917729
:10F9F800DB7BE02B40F00E82164B3F22DA7709E2E0
:10FA08001C4B1B7803F08003DBB2002B40F0028212
:10FA18000DF11F001649FEF76FFF18B15046FEF7AB
:10FA280055FFF7E114485146C9EB00004A46B2E6D3
:10FA3800583D00200F020020840D002013020020F2
:10FA4800503D002072E4020893E4020838E50208F9
:10FA580017E50208F401002004020020D61D00204A
:10FA6800553D0020861D0020E41D0020C01C0020FC
:10FA7800A01D0020DC39002014020020A3F10D0293
:10FA8800042A31D89DF81F30D6B2222202FB036324
:10FA9800984A02EB83035F6C3846F0F7CBFE394691
:10FAA80002469548F0F74CFF944B1B786BB1944B8A
:10FAB8001B7803F08003DBB21BB19248202102229D
:10FAC800EDE0914B8F4819780CE04FF436636343AF
:10FAD8002A783424013A04FB02348C4B89481C19D7
:10FAE800A619717C822256E6123B0B2B00F29281FA
:10FAF8009DF81F20DBB2222101FB02317D4A16311D
:10FB080052F821207C4902F110008A4652F804CBB1
:10FB1800824241F804CBF9D1DFF83092DFF830B2F5
:10FB28002FB199F80020012A15D1013209E096B1C8
:10FB380099F80020012A07D97549097803290AD1BB
:10FB4800013A89F8002006E005D1714909780329AE
:10FB580008BF8BF8002099F800209AB94FF4B661D5
:10FB68004C432A781A21013A01FB0244674AE318F8
:10FB7800083302EB43039A798BF80020DA79644B57
:10FB88001A7047E1634C202104F118000822F0F7AD
:10FB980001FCB8F1000F00D1AEB15D4D2B78012BFF
:10FBA80001D15D4A01E04BB95C4A1368236153688F
:10FBB800CAF80430B8F1000F21D00BE0022B0CBFBB
:10FBC800574A584AF1E7584A136823615368CAF8F4
:10FBD800043019E19BF800004E4A3121002350FA05
:10FBE80003F515F0010F01D0117701E02D251577E8
:10FBF800013301310132042BC9B2F0D12FE0002EBC
:10FC080000F00281202108224848F0F7C3FB3D4854
:10FC18009BF800108222F8F79FFE394B1B7803F0FF
:10FC28008003DBB21BB199F80030012B02D82B7886
:10FC3800032B21D1202102223248F0F7ABFB1BE035
:10FC480050FA03F515F0010F01D0117701E02D25C9
:10FC58001577013301310132042BC9B2F0D1284B99
:10FC68001B7803F08003DBB233B199F80030012B25
:10FC780002D9E4182023A376214B1B7803F08003D4
:10FC8800DBB2002B00F0C68099F80030012B40F061
:10FC9800C180002F40F0BE80174820210822F0F7CD
:10FCA80079FBB7E099F80030214D13F0010F04BF3C
:10FCB80043F0010389F800302E78002E4AD12D2117
:10FCC8000A221C48F0F766FB04201B49F8F71EFEC1
:10FCD8001A4B1B78012B02D11020194906E0022B80
:10FCE80002D11020174901E017491020F8F70EFE3D
:10FCF80090E000BF840D0020040200209F1D00201A
:10FD0800DC39002012020020541E0020503D002043
:10FD1800D51D0020F40100201DEE02083EEE020869
:10FD28005FEE020880EE020899ED02080C0200203E
:10FD3800931D0020B81D00200CF00208891D00202A
:10FD4800F6E40208B4E40208D5E402088B1D00209A
:10FD5800851D0020314B1C782046F8F793FE304B68
:10FD6800304A00282AD0304F30493878A04216D17E
:10FD780030380C782E4E00EB80073C19345D04B9FE
:10FD88000C700F7800EB8000C4190137FFB2C0195E
:10FD98000F70315C345D59B92448017008E00120C6
:10FDA800087019783C7019B1092E9CBF36182E704E
:10FDB8002978511801F8014C40211970197811B1AE
:10FDC8001748013901701978012909D129780929B9
:10FDD80002D818480131017000211970134B1970AD
:10FDE8001168154BC3F816105168C3F81A10128918
:10FDF800DA83124A127802F08002D2B252B12A781B
:10FE08009B1820225A7505E09BF800000A4A312108
:10FE1800002315E709B0BDE8F08F00BFC01C002023
:10FE2800DD1C0020B81D0020DA1C0020061D002063
:10FE3800EC6C0208931D0020F4010020DC3900203E
:10FE48001FB5044611B100200B4901E008460B49D3
:10FE5800F8F75CFD217810220139C9B201EB0111D4
:10FE680001F5C2414831684601F0B5FD1020014650
:10FE78006A46FDF7B5F91FBD04CE020846CE020852
:10FE88000B4B1B78442B06D0552B037801D013B1AC
:10FE98007047013B01E003780133037003780BB925
:10FEA800203302E0212B01D1203B0370FFF7C8BFAC
:10FEB800C01C00202DE9F74FDFF8C881DFF8D4A176
:10FEC80098F80030554643F0010388F800309AF856
:10FED8000130624C23F07F039B46D3B10020604978
:10FEE800F8F714FD5F482A21F0F7D2FA18B1217803
:10FEF8008222F8F731FD2278002A40F0AB802B6887
:10FF080062F3CF332B60584B1A7842F003021A7011
:10FF1800A0E0DFF85491237099F800304E4603F0C2
:10FF28000202D2B20192514F002A40D013F00108C8
:10FF380013D058464E49F8F7E9FC3B78232B20D1DB
:10FF48004C4B4D4A4D481A600121FFF779FF337831
:10FF580003F0FE036BF3410312E040464849F8F70B
:10FF6800D5FC3B78232B0CD1424B434A43481A60BB
:10FF78000121FFF765FF337868F3000368F3410355
:10FF880033703B782A2B65D1337803F0FE036FF387
:10FF9800410333702B6843F400432B600F23237015
:10FFA800364B187803B0BDE8F04F0DF05DBF0DF08B
:10FFB8009FFE054600282DD001213048FFF760FF3D
:10FFC8003B78532B12D13378019A03F0FD0362F387
:10FFD80000033370DAF8003043F40043CAF8003005
:10FFE8000F232370254B18780DF03EFF3B78232B09
:08FFF80030D13378002203F040
:020000040801F1
:10000000FD036FF3000333701E4B1A70F8F746FDC3
:100010001E4A137843F00603137015E01C49F8F7E5
:1000200079FC3B78232B19D199F8003065F3410313
:1000300065F3000389F80030F8F730FD98F80030D8
:1000400043F0060388F80030124A1378013BDBB214
:100050001370114A52F82320084B1A6003B0BDE810
:10006000F08F00BF7257002088CE0208F4010020F4
:10007000633B0020C01C0020A9CE0208F81C002011
:10008000AC6E0208921D0020CACE0208D71D0020C7
:10009000EBCE0208B71D0020C41D0020DC39002073
:1000A0002DE9FF412C4D2D4C2B7843F001032B7093
:1000B000217801F00401C9B211B92948FFF7E4FE23
:1000C000284E3378232B21D12378274F13F00408AF
:1000D0000AD0224A6FF382031370244B20483B60FE
:1000E0000021FFF7B1FE11E0F8F7D8FC2B78204A89
:1000F00043F006032B701378013BDBB213701D4AEB
:1001000052F823303B60164B83F800803378532B32
:100110001FD12378052243F004032370104B1649A6
:100120001C78013CE4B204EB840000F5CA4088303E
:1001300001F04FFC00201149F8F7ECFBFF230021F0
:1001400000930134162004220B460191029401F021
:10015000B3FCBDE8FF8100BFD71D0020633B00203A
:10016000921D0020C01C0020F81C0020C86E020850
:10017000B71D0020C41D0020E46E020867CE0208EF
:100180002DE9F041984B04469A7812F0010F00F0E7
:1001900017811B88002B40F01381944D95F8203077
:1001A0003F2B40F2D780012C14D1914B1B7803F0E8
:1001B0000203DBB2002B00F0C48095F820208B4BAB
:1001C000402A03D1013283F82020FBE0482283F843
:1001D0002020B6E0022C03D1482385F82030B0E07F
:1001E000844E337803F02002D2B28AB195F82020F1
:1001F000402A0DD1032C0BD07F4B804A03F1100114
:1002000053F8040B8B4242F8040BF9D1412395E0DB
:1002100003F01003DBB28BB195F82030412B0DD1E8
:10022000032C0BD0764B754A03F1100153F8040BE5
:100230008B4242F8040BF9D142237FE0F37813F0AC
:10024000010F0FD095F82020422A0BD16D4B6B4A3D
:1002500003F1100153F8040B8B4242F8040BF9D15F
:1002600043236BE003F00202D2B27AB195F820206A
:10027000432A0BD1644B614A03F1100153F8040B7C
:100280008B4242F8040BF9D1442357E003F00402F7
:10029000D2B27AB195F82020442A0BD15B4B574A51
:1002A00003F1100153F8040B8B4242F8040BF9D10F
:1002B000452343E003F00803DBB28BB195F820300F
:1002C000452B0DD1032C0BD0514B4C4A03F110019F
:1002D00053F8040B8B4242F8040BF9D146232DE06E
:1002E0000EF038FBA0B14B4B1B788BB195F820304A
:1002F000462B0DD1032C0BD0474B404A03F1100184
:1003000053F8040B8B4242F8040BF9D1472315E054
:10031000F37803F04003DBB29BB195F82030472B14
:100320000FD1032C0DD03D4B344A03F1100153F88B
:10033000040B8B4242F8040BF9D1482385F8203096
:1003400078E095F820300133DBB2472B85F8203078
:100350007FF629AF95F82060472E04D9234B00265D
:1003600083F8206001E00136F6B206F14007FFB2E3
:1003700012E02B48314614F02CFA08B1032C04D1BA
:10038000284B9B5D23B1032C02D185F820600FE040
:100390000136F6B2BE4203D03F2EEAD9402E07D135
:1003A000214B1E221A70402385F82030BDE8F081D1
:1003B00095F820001149652246F69543F8F7F6F9BD
:1003C000012C37D1194B0D4A03F1100153F8040BDE
:1003D0008B4242F8040BF9D1044B93F820303F2BA9
:1003E0003CD9002012493EE0E81D0020F401002025
:1003F0008D190020DC3900203CD50208EF1D0020BB
:100400005DD502087ED502089FD50208C0D5020836
:10041000E1D50208443D002002D6020844D6020875
:10042000231A0020D9190020941D00203C3803080D
:10043000FAD40208104BD87800F02000C0B220B1E6
:10044000022C06D000200D490DE0032C01D10C49EF
:1004500009E00C4B93F820303F2B02D800200A49CA
:1004600001E00A490020F8F755FA1020084A014631
:10047000BDE8F041F8F706BADC39002015CC0208D7
:100480001BD50208F4010020B8D4020823D60208C4
:10049000E81D002010B5F8F701FB084B1B7803F0AE
:1004A0000403DBB22BB106490020BDE81040F8F789
:1004B00031BA0220BDE81040FFF762BE8D1900205E
:1004C000EAD2020870B5224B06461B78214CF3B9DC
:1004D000257819E02048294614F07BF978B1236883
:1004E0009D4202D9FF2E02D007E0FF2E02D19D428D
:1004F00008D202E036B91DB913B9256012E00EB971
:10050000013500E0AD19EDB23F2DE3D90AE0013B22
:100510002021124810222360EFF740FF00201049ED
:10052000F8F7F8F90F48F8F79BF946F69543207865
:100530000D496522F8F73AF9084D216805F11000D8
:1005400001310222F8F70CFA2D23AB7470BD00BF05
:10055000871D0020A01D0020FE1C0020F4010020AB
:10056000B8160308E81D0020EF1D0020F8B5594B10
:10057000F02259481A700378044613F00E051DD175
:10058000564A43F00203156000F8013B14F0C6F828
:100590002C46534BE35C1BB15248214614F003F93F
:1005A0000134402CF5D1504B01221A700FF012FA91
:1005B0004E4B1A7842F001021A70F8BD13F00C0588
:1005C00043D12E464748294614F003F908B10136B5
:1005D000F6B20135402DF5D11EB9237843F004035E
:1005E00031E0002542482946EFB214F0F2F868B134
:1005F0003B4BEB5C53B13F4B01371F700020FFF7C3
:1006000061FF237843F00803237002E00135402D99
:10061000E8D1394D3A212846EFF73EFF38B1401B6B
:10062000C0B20130281831460222F8F799F9334B4D
:100630001B78532B4CD12F4B00201870FFF742FF33
:10064000237843F008032370F8BD6FF34103037070
:1006500003F00403DBB2294D23B100202849F8F749
:1006600059F90EE02B78552B01D1FF2002E0442BE5
:1006700002D10120FFF726FF13200D21214AF8F7B0
:1006800001F92B78232B23D12478134E04F0020494
:10069000F4B9154B1C700FF09DF9337803F0FB0390
:1006A00064F3C30333700D4B1C60F8F7F7F90F4B7D
:1006B0001A7842F006021A70134A1378013BDBB233
:1006C0001370124A52F82320114B1A60094B1C7008
:1006D000F8BD00BFE31D0020FD1C0020A01D002070
:1006E000202C0020FE1C002028140020D71D0020F4
:1006F0008E190020871D0020F4010020C01C00205E
:10070000FE270308E81D0020B71D0020C41D00209F
:10071000F81C002070B505460C4616463BB1430058
:100720004BF2B94018184018114601F03DF9054B3D
:10073000182202FB0535F3092C1906F07F066370B9
:10074000E67070BD8A3A002038B510B3A0F14103BD
:10075000DBB2432B1FD9C50900F07F040BD0052C59
:1007600019D90021601E0A460AF028FCD0F10100C8
:1007700038BF002038BD042C0FD9601EC0B22946F6
:100780002A460AF0A7F850B9102C8CBF002001208F
:1007900038BD012038BD002038BD284638BD284668
:1007A00038BD0000F7B5604C312323745F4F01332F
:1007B0002376053B637463763B784BF2B9405B006C
:1007C000181801F0FBF8C0B220F07F0200F07F01A2
:1007D000D2B28DF804108DF8002004F1120359B93B
:1007E000534A04F115001188927861829A70202191
:1007F0000222EFF7D3FD0CE0D20904EB8202526A29
:1008000010886082927804F115009A700222F8F73D
:10081000A7F83878400000F53440BA3001F0CEF83F
:10082000C0B220F07F0300F07F01DBB28DF805102D
:100830008DF801303F4851B93D4B20311A889B78E3
:100840006283837002220330EFF7A8FD0BE0DB091F
:1008500004EB83035B6A1A8862839B7802228370AD
:100860000330F8F77DF8344B1B7813F0010F5AD0A2
:10087000324D02A92A788B1813F8041C13F8086C5F
:100880002F4B1B78232B04D1002A41D1223B2B7004
:100890003EE02A2B04D1002A3AD0013A2A7037E0F0
:1008A000552B46EA010611D10DE02B7802AAD31888
:1008B000013E13F8081CF6B23046C90913F8042C9F
:1008C000FFF742FF98B9002EEFD121E0442B19D158
:1008D00015E02B7802A9CB18013613F8081CF6B2E4
:1008E0003046C90913F8042CFFF72EFF38B1134B1B
:1008F0003878197832460123FFF70CFF08E0872E7D
:10090000E7D905E0532B03D1533B2B70F9F7C8F817
:100910000C4B1B7803F08003DBB223B12B78202231
:10092000023304F83320FEBDF4010020871D0020AF
:10093000FB3303080E020020D71D0020921D00206B
:10094000C01C0020DC390020024800210922EFF7FA
:1009500025BD00BFA51D002070B50A46002405E096
:100960001B19811A2A2501345D54E4B20E4D0F4B38
:10097000295D09B19442F3D1801A00191818202179
:10098000121BEFF70BFD0A4B1E785EB1432E04D10C
:100990000CB1013CE4B200232B553046F8F776F851
:1009A00000B12E5570BD00BFA51D0020F401002030
:1009B000C01C002038B5184C184DA07800F010006D
:1009C000C0B250B91649F7F7A5FFFFF7BDFF23687E
:1009D00043F4801323600F232B702A782AB92368ED
:1009E000FF2062F31453236038BD0E48C5792DB93A
:1009F0001C200821FFF7B0FF284638BD23680A49AC
:100A00006FF3145308222360EFF748FF00280CBF50
:100A10000120FF2038BD00BFDC390020E61D00208A
:100A20004DD30208A51D00205C530308F0B55C4CB3
:100A300085B0667806F01006F6B2002E3ED1594B0E
:100A40001A78594B013A53F82230584A934204D14C
:100A5000574B1A7842F0020207E002F11C018B4268
:100A600008D1534B1A7842F00402022161F3C70205
:100A70001A7019E03832934216D1FFF79BFF002815
:100A800000F08C8001284A4D06D12B78022243F0D9
:100A9000010362F3C70306E030464649F7F73AFF21
:100AA0002B7866F3C7032B70434B1A7842F0010290
:100AB0001A70236843F4805323606FE03C4D2B7819
:100AC00013F0F80606D03D49002005B0BDE8F0401F
:100AD000F7F720BF13F0070F41D003F00202D7B29F
:100AE0004FB11220314610F0ABF8FF23009301966E
:100AF000029643202AE003F00406F6B2A6B1394676
:100B0000384610F09DF8382102200EF077FC09F0ED
:100B10000BFD0DF019F9FF23009301970297442074
:100B2000394604223B4614E013F0010F13D0012193
:100B300043F6206010F084F83046F5F7E7FA204BD2
:100B400045201E80FF230093019602963146042221
:100B5000334600F0B1FF00201A49F7F7DBFE2B788F
:100B600003F0FA036FF341032B70174B1B78232B11
:100B700014D123686FF30C332360F7F78FFF0E4B0C
:100B80001A7842F006021A70064A1378013BDBB26B
:100B90001370054A52F823200C4B1A6005B0F0BDC3
:100BA000DC390020B71D0020C41D0020EC6E0208B7
:100BB000F45400206ED30208D71D00209A2B03089E
:100BC000D61C0020792B0308C01C0020F81C002034
:100BD0001FB50446F5F786FBA8B14B2001F036FBA4
:100BE000FF2300930121FF3B0193392004220B4690
:100BF0000134029400F060FF064B01205A7842F065
:100C000004025A7004E0044B1888003818BF012011
:100C100004B010BD503B002088570020F0B5204E96
:100C20000024337A0546013385B00F463372102015
:100C30002146012223460094F1F764FD55B9FF23B4
:100C400000934F20294604222B460195029700F07D
:100C500033FF0EE0012D0CD1FF23009350202346DB
:100C6000214604220194029700F026FF337A013BCB
:100C70003372337A052B11D1FA330121002400930A
:100C800027200B4604220194029400F015FF044B28
:100C90001C7205B0BDE8F04001F0AABA05B0F0BD85
:100CA000961D0020074B182202FB00335B7913F0DE
:100CB000100F05D0044B173ADA715A7009329A7046
:100CC000704700BF8A3A0020671300202DE9F04FDB
:100CD0009A4B87B01A78074699461AB1012A40F014
:100CE000E68130E0964B1A68964B9A4200F0E1811B
:100CF000F4F776FF944B5B7803F00203DBB253B951
:100D0000924B5B7803F08003DBB223B901F096FAD3
:100D100008B909F009FC8E4B1A686FF310421A608B
:100D20008C4B1878F7F7B2FE002800F0C281FFF76D
:100D30000BFE894B3C221A70F7F7F4FC99F800304F
:100D4000013389F80030844B1C7874B9834B791CCB
:100D50001A78204664F3C30264F304121A70C9B20D
:100D6000FFF75CFF89F80040A3E17D4D384609F0AC
:100D7000FBFBF7F7CBFC00207A49F7F7CBFDDFF858
:100D8000F4812B78AA46434413F8313C23B91B2045
:100D90000621FFF7E1FD8CE1704A0B21137804A8CE
:100DA000C3F3C004C3F3001603F0F7036FF3041397
:100DB0001370002389F80030062200F010FE2A7814
:100DC000414604A8303AEFF70FFA804628B14FF0B9
:100DD00000084FF0120945462AE04AF26B7000F015
:100DE000EDFD0028F3D0604D85F80880F5F760F838
:100DF0000446002840F05D815C4A514B21461A6050
:100E0000FF2300930190029004220820234600F063
:100E100053FE012223460E2021460094F1F772FC76
:100E2000534B1A7842F004021A700123AB7140E16F
:100E30004946062204A800F0D2FD9AF8002004A832
:100E40004C49303AEFF7D0F9002840F0218128468C
:100E5000FFF7BEFE002840F02C81DFF80CB1012125
:100E60008BF808002846F5F731F88146F5F720F8A9
:100E7000DA46002840F0B58048463F49EFF792FB3C
:100E8000B0B901F0EDF82E4B14B916B93B4A23E086
:100E900036B13B4A1A603B4B1A786FF3410205E0CA
:100EA000394A1A60374B1A7866F341021A70D7E054
:100EB00048463649EFF776FB20B148463449EFF70C
:100EC00071FB70B9002C40F0F480002E40F0F180EE
:100ED00001F0C6F82F4A1A4B1A603846FFF7E2FEB7
:100EE000BEE048462C49EFF75DFB50B94AF2697005
:100EF000012100F059FD164A136843F400531360B2
:100F0000E0E748462549EFF74DFB38B9002C40F0A3
:100F1000D080002E40F0CD80214A0CE04846214987
:100F2000EFF740FB002841D1002C40F0C280002E9A
:100F300040F0BF801C4A024B1A6091E0F41C002074
:100F4000F81C0020406F0208C63300205F3B0020E1
:100F5000DC390020C01C0020E61D0020A41D00205C
:100F6000DC1C0020F4CB0208961D00205C6F0208F8
:100F7000F1250020A51D0020E5540308A8710208F2
:100F800030730208D71D00204C7302086154030817
:100F9000F1560308687302089C5403089E54030822
:100FA000A0730208AE560308F4730208484642498B
:100FB000EFF7F8FA002853D101F052F83CB13F4A5C
:100FC0003F4B1A603F4B1A786FF3410270E0002EDE
:100FD0006FD03D4A3A4B1A603A4B1A7864F341029B
:100FE00066E048463449EFF7DDFA064620B901F0DD
:100FF00037F8002C5DD01BE048463449EFF7D2FAB1
:10100000002856D048463249EFF7CCFA38B9002CC0
:101010004FD1304A2A4B8BF807501A6049E04846B6
:101020002D49EFF7BFFA064650B9A4B101F018F800
:10103000224A234B1A60234B1A7866F3410237E0A9
:1010400048462649EFF7AEFA20B148462449EFF763
:10105000A9FA00B96CBB234A194B1A6001F000F8D9
:1010600008F56A507C308AF8075000F0A7FC8AF82F
:1010700000009AF8070000F5D640693000F09EFCA9
:101080008AF801001848F5F759F8202D11D108E029
:101090000135EDB2202D08F1010809F107097FF4AF
:1010A000C7AE791C0020C9B2FFF7B8FD01E00022ED
:1010B0001A7007B0BDE8F08FA05403084C73020803
:1010C000F81C0020D71D0020307302089E5403082E
:1010D000AE560308F4730208E5540308615403088C
:1010E0009C54030810740208961D002010B5214876
:1010F000214903680A789C7B944203D99C8914F0A7
:10110000200F18D09A8912F0800F01D105E01C3B06
:101110009A8912F0400FFAD000E01C3303600023DC
:101120000B7003689B8913F0200F16D0134BDA79EC
:10113000114B1A7011E00132D2B20A70986843F66E
:101140000953984209D101E00132D2B2162A03D8DC
:101150000B4853B29840F7D40A700A4A136843F414
:1011600080731360F7F7DEFA074B1A7842F0060235
:101170001A7010BDF81C0020871D0020961D00204D
:1011800000060088DC390020D71D002010B5234957
:10119000234A0B78D3B11068848914F0200F15D13D
:1011A000013BDBB20B70846843F60952944228D1AC
:1011B00004E013B1013BDBB200E0837B162B03D8C4
:1011C000184C5AB29440F4D40B701AE01368988902
:1011D00010F0400F01D106E01C33988910F0800F09
:1011E000FAD0136002E00E481C3B036013689A7B40
:1011F0000A709B8913F0200F03D00B4BDA79074B51
:101200001A700A4A136843F480731360F7F78AFA76
:10121000074B1A7842F006021A7010BD871D002095
:10122000F81C002000060088961D0020DC390020F4
:10123000D71D0020084B1A68084B9A4204D003F5CA
:1012400080630C339A4205D1054B1878003818BFDB
:101250000120704700207047F81C0020406F0208F2
:101260008C190020074B084A1B68934202D0383281
:10127000934205D1054B1878003818BF01207047FC
:1012800000207047F81C0020F47302088C1900201D
:101290002DE9F04F814B824D1970A0F11103DBB2A3
:1012A000012B87B00E46287006D8122801D11138BC
:1012B00000E00020F4F788FF2B78522B0DD1F1F7D6
:1012C0003BFF28B9F1F72CFF10B9F1F74DFF20B122
:1012D000744B1A7842F008021A70734B734C1B78E7
:1012E000002B2FD12168724A91422BD0714A236082
:1012F0001370714A71481178037063F3C30163F38B
:10130000000163F3071111706D4A117863F3010155
:1013100011706C4A117863F3C50111706A4A137039
:101320006A4A117863F3410163F3000163F38201B8
:101330001170674A116863F30C311160654A1370CC
:10134000654A93712368002B40F05F81604F7B7882
:1013500003F02003DBB273B1604B93F80080B8F167
:10136000000F08D14AF26970414600F01DFB3B684E
:1013700068F34D333B605A4B187810F01E0002D0D2
:101380000020584907E0544B93F808909846B9F16B
:10139000000F05D0544907B0BDE8F04FF7F7BABACF
:1013A000524F97F801B0BA46BBF1000F2DD0BBF1F8
:1013B000070F15D94E48F7F753FA4E49B87865220A
:1013C00046F69553F7F7F2F93878072310F0030043
:1013D0007B700EBF484948464849F7F79BFA0CE036
:1013E000BBF1020F09D84248437823B1F7F738FA26
:1013F00087F80190B4E202237B7010203C4A01463A
:1014000007B0BDE8F04FF7F73DBA3D4FBB795BB190
:1014100087F806B000F034FC8E20594601225B4666
:10142000CDF800B0F1F76EF90020F1F7E7FF224A9E
:1014300020491378334843F00603137000230B70E0
:10144000314923600B7088F8033088F8013003704D
:10145000183303FB06FC2D49934611F80CC089464E
:101460001CF0080F04D130460593FFF72FFC059BB5
:1014700003FB06935B7913F0100F04D02A78133A1C
:10148000D2B2032A46D913F0200F79D02B78442BFF
:1014900040D03DD8232B3DD02A2B3AE08A1D002096
:1014A000C01C0020CB190020E31D0020F81C0020E8
:1014B000906E0208B71D0020D71D0020921D00204D
:1014C000D91C00208D1D0020951D0020A41D00208A
:1014D000DC390020E21D0020671300208C19002059
:1014E0007157002057CC0208B6FD02088F1D00205E
:1014F000E81D0020EF1D00205FCD02083ECD020850
:10150000961D00208C1D0020871D00208A3A002097
:10151000552B35D18C4B1B78002B31D18B4B93F84D
:101520000090B9F1000F2BD143F6DB2000F046FA12
:10153000012825D11F23FB7188F8030043F61B30D7
:1015400000F03CFA3870F87900F5D640693000F0C8
:1015500035FA78707E48F4F7F1FD9BF8003030469C
:1015600069F341038BF8003008F0FEFFF7F796FAB5
:10157000784B79482360794BC3F800902B7803703F
:101580002B78432B0AD1714B1B783BB9013388F878
:101590000330734B3046236008F0E6FF2878173895
:1015A000C3B2072B27D86F49FF220AF091FD9AF8A2
:1015B00000106D4B60F301018AF8001001F0030187
:1015C000022918D00122032041B1009001929B789A
:1015D00068309B1802930021033206E000900192CC
:1015E0009B786C200133029304220B4600F064FACE
:1015F000FF238AF8013098F80730002B00F0B08103
:1016000052232B70594B0022DA712268544B9A42B4
:1016100050D12878A0F14303DAB2122A22D8544AD2
:101620005BB29A401ED5432840F09A81464B1B7806
:10163000002B40F0958100F01DFD4E4B48B11A780B
:1016400003201109013191FBF0F000EB4000091A71
:1016500004E01A781109013101F0070161F3071262
:101660001A707DE1F7F712FA002823D0414F3A783B
:1016700012F0F00308D163F307123A7023603E4B77
:101680001A7842F008020EE0102B13D100F0F2FCA1
:1016900080B13B786FF307133B7000232360364B18
:1016A0001A7842F0100230461A7007B0BDE8F04FC9
:1016B000FFF70CBB314B1E211A78264F61F346020F
:1016C0001A702B78232B1CD12368BB4219D12C4BC9
:1016D000182202FB0636737913F0100F11D0294B34
:1016E0001B7873B11A4EF7F7D9F9FCF77DFAF07948
:1016F00000F56A507C3000F061F93070AA20F1F7F3
:101700007DFE1C4E337813F0010F43D02368BB429B
:101710000BD01D4A934208D0FFF78CFD28B9FFF784
:10172000A1FD10B9AA30F1F769FE2268174B9A4261
:1017300002D10020F1F762FE2B78522B40F0D580C9
:101740005322134BC9E000BF8C190020F41C002069
:10175000961D0020107402088C1D0020C41D00205E
:10176000406F0208911D00208F1D0020671300208C
:10177000002000C0D71D0020A41D0020551E002001
:101780008A3A0020B71D0020906E020848740208B3
:10179000C01C00202368BB420BD0734A934208D080
:1017A000FFF748FD28B9FFF75DFD10B9AA30F1F742
:1017B00025FE2B78552B1ED1FFF7E8FC33786B48BC
:1017C00043F0060333708378694F03F00203DBB202
:1017D0004BB1F7F745F823681868FAF7C7F93B7873
:1017E0006FF341033B706348837803F00203DBB27D
:1017F0000BB1F7F735F82B78442B1ED1FFF776FCA9
:1018000033785A4843F0060333708378584F03F017
:101810000203DBB24BB1F7F723F823681868FAF735
:10182000A5F93B786FF341033B705248837803F08E
:101830000203DBB20BB1F7F713F82B78522B09D167
:101840003378002243F0010333704B4B1A704B4B3B
:1018500045321A704A4B00271F702B78232B44D136
:10186000484B42481F70484B1F70F6F7F9FF41483C
:10187000F6F7F6FF3378454943F0060333700B78EB
:101880003B4A002B2BD0424A013B1770414ADBB246
:101890000B7052F8233023603F4B1A7812B11F703F
:1018A0000EF098F823683D4A9B68934202D109F0F4
:1018B000AFFE1AE002F59A718B4203D002F5E07197
:1018C0008B4204D10120014606F0BAFF0DE002F57B
:1018D000EE72934209D1324B00221A7005E0117862
:1018E00063F30711117023603AE02E4BDB7813B1DC
:1018F0000020F1F783FD23681F7B17F00F0702D14B
:10190000FBF71AFB1BE0012F02D1F8F777FA16E07C
:10191000022F02D1F9F7E0F911E0082F05D84FF0B6
:101920009C53BB4001D5F9F79DFC042F03D12368DC
:101930009B69984703E0052F01D1F8F74BFF3378F7
:1019400003F00203DBB21BB123681868FAF70EF943
:1019500033786FF3410333702B780BB1084A13705F
:1019600007B0BDE8F08F00BF906E0208E81D0020B0
:10197000D71D0020081D0020921D0020C01C002043
:10198000DA1C0020951D0020E21D0020B71D00205C
:10199000871D0020C41D0020281400206474020844
:1019A000071D00206713002007B502AB03F8011DD7
:1019B00019460122002305F09DFB0EBD07B500234B
:1019C00002A901F8013D012205F0FCFB9DF807008A
:1019D0000EBD08B5002305F08DFB002008BD0346B1
:1019E00010B508461446194605F0ECFBE0B210BDF0
:1019F00010B50346002484540846194605F0E2FB5E
:101A0000204610BD37B50546002400E014460122EB
:101A100060190DF1070105F0D5FB9DF80730621C38
:101A2000203BDBB25A2BF1D920463EBDF8B500254C
:101A30002C461E4B1C21585D01FB0431400000F573
:101A400074506630043102220134FFF7C2FF1C35A6
:101A50005C2CEED143F6C43420B204220534144980
:101A6000FFF7B7FFA4B243F6D8339C42F4D1002568
:101A700049F668572C4615E007EB460004EB440195
:101A800000B259180222FFF7A4FF0136F6B2094B43
:101A90005A199278B242EFD8013480370335142CAA
:101AA000BFB201D00026F2E7F8BD00BF5C9F02087C
:101AB000635403086CA902082DE9F3470446154650
:101AC0008A46022243F61E610DF106001E46BDF94C
:101AD00030909DF828809DF82C70FFF780FF2F4BE9
:101AE0002F499A78BDF906008A705A7800EBC00039
:101AF000CA701A7900F578500A715A7920304A7103
:101B00009A791B7845EAC6158A710C7081F80190A4
:101B1000CB710D7200B20922FFF75BFF1EB1214BA2
:101B20001A8801321A80BDF8063001339BB2B3F532
:101B30007A7FADF8063002D30023ADF806300222DA
:101B40000DF1060143F61E60FFF743FFBDF80600E6
:101B5000154B188000B200EBC00000F5785000F182
:101B60002005283000B2FFF729FF10F0800F03D0C6
:101B70000C4B1A88013A1A8028B20021FFF714FF93
:101B80000A4B03F8148003EB44046770BAF1000FAA
:101B900002D00120F4F7BAFABDE8FC87FC5400201B
:101BA000AE1D0020D61C0020C43300205931002077
:101BB0002DE9F743314B1D78303DEDB2C5F10606F6
:101BC000F6B23EB305F11207202413E008F1010834
:101BD0000FFA89F000215FFA88F8FFF7E5FE09F1B6
:101BE0000109B0451FFA89F9F0D1013C0737E4B289
:101BF000BFB21CB1B9464FF00008E7E70B3501341E
